:10000000FCFB0220D101000059BC010011BC010021
:1000100011BC010011BC010011BC010011BC0100A8
:1000200011BC010011BC010011BC010059BC010050
:1000300059BC010011BC010091D10100E1D30100C4
:1000400059BC010059BC010059BC010059BC010058
:1000500059BC010059BC010059BC010059BC010048
:1000600059BC010059BC010059BC010059BC010038
:1000700059BC010059BC010059BC010059BC010028
:1000800059BC010059BC010059BC010059BC010018
:1000900059BC010059BC010059BC010059BC010008
:1000A0004DB5010061B501004DB60100DDB601009E
:1000B00059BC010059BC010059BC010009D501001F
:1000C00059BC010035D6010059BC010061D70100BF
:1000D00059BC010059D8010059BC010025B50100E7
:1000E00059BC010059BC010059BC010059BC0100B8
:1000F00059BC010059BC010059BC010059BC0100A8
:100100003109FF1F59BC010059BC010059BC010055
:1001100059BC010095C3010059BC010059BC010044
:1001200059BC010059BC010059BC010059BC010077
:1001300059BC010059BC010059BC010059BC010067
:1001400059BC010059BC010051D9010059BC010042
:1001500059BC010059BC010059BC010059BC010047
:1001600059BC010039B5010075B5010059BC010049
:1001700059BC010059BC010059BC010059BC010027
:1001800059BC0100D5B4010059BC010059BC0100A3
:1001900059BC010059BC010049DA010059BC0100F9
:1001A00059BC010059BC010059BC010089B50100CE
:1001B00059BC010059BC010059BC010059BC0100E7
:1001C00059BC010059BC010059BC010059BC0100D7
:1001D0005C4B4CF2205210B51A804DF628121A8052
:1001E00000BF00BF1BF03CFD574B4FF030621A6060
:1001F000564A9A60564ADA60564B4FF470021A60BB
:10020000554B564A1A60564B1A78110703D51A787F
:1002100042F008021A70534B5349AA221A70534AEB
:10022000534B8B4204D252F8040F43F8040BF8E707
:10023000504B514900228B4202D243F8042BFAE77B
:100240004E494F4A002352F8230041F8230001335E
:10025000742BF8D14B4B4C4A802103F8011B93427D
:10026000FBD14A4B454A1A60494B8A221A70A3F5C2
:10027000805324225A70A0221A709A799207FCD5D2
:100280009A79D406FCD4434A937903F00C03082BE3
:10029000FAD1414B60221A7002331A78802AFCD1BD
:1002A0003C4B01221A715D225A719A799006FCD555
:1002B0009979384A4906FBD5384B394919600021EC
:1002C000596020231370937903F00C030C2BFAD19F
:1002D000344B354A1A60354A354C136813F4807331
:1002E00003D123604FF4A8531360324B324A1A6093
:1002F00000225A60072243F8042C304AC3F80C2D20
:1003000062B61BF09FFD2368DA0705D52C481BF069
:1003100087FD2C4B2C4A1A602C4B1B785B0609D5A9
:10032000284C294B22689A4204D125481BF078FDBD
:10033000002323601DF0ACFE1BF098FC1BF0C8FBF3
:10034000FEE700BF0E20054030800440823F0400DD
:100350000100002B88ED00E0002008E0030000858C
:1003600002D0074000E007407016FF1F904F0200C8
:100370003009FF1F7016FF1FDCD201200004FF1F91
:100380000000000000E400E064E400E008ED00E0AC
:10039000005006400040064001E007404480044011
:1003A0000000060204800440C010070010D0034083
:1003B00014D0034014E000E01FBF02000000202022
:1003C00083150C661CE00340A5C3945A00F0074057
:1003D000FFFFFFFFFFFFFFFFFFFFFFFFFFFFFFFF2D
:1003E000FFFFFFFFFFFFFFFFFFFFFFFFFFFFFFFF1D
:1003F000FFFFFFFFFFFFFFFFFFFFFFFFFFFFFFFF0D
:10040000FFFFFFFFFFFFFFFFFFFFFFFFDEF9FFFF23
:1004100010B5054C237833B9044B13B10448AFF33E
:1004200000800123237010BD7016FF1F0000000024
:100430008C4F0200084B10B51BB108490848AFF3B8
:1004400000800848036803B910BD074B002BFBD0A0
:10045000BDE81040184700BF000000007416FF1FE1
:100460008C4F02007016FF1F00000000704700BF95
:10047000704700BF034B586810B103681B681847EA
:10048000704700BF48CD0120034B986810B1036846
:100490001B681847704700BF48CD0120034BD86840
:1004A00010B103681B681847704700BF48CD012092
:1004B000034B186910B103681B681847704700BFE9
:1004C00048CD0120034B586910B103681B681847D9
:1004D000704700BF48CD0120034B986910B10368F5
:1004E0001B681847704700BF48CD0120034BD869EF
:1004F00010B103681B681847704700BF48CD012042
:10050000034B186A10B103681B681847704700BF97
:1005100048CD0120034B586A10B103681B68184787
:10052000704700BF48CD0120034B986A10B10368A3
:100530001B681847704700BF48CD0120034BD86A9D
:1005400010B103681B681847704700BF48CD0120F1
:10055000034B186B10B103681B681847704700BF46
:1005600048CD0120034B586B10B103681B68184736
:10057000704700BF48CD0120034B986B10B1036852
:100580001B681847704700BF48CD0120034BD86B4C
:1005900010B103681B681847704700BF48CD0120A1
:1005A000034B186C10B103681B681847704700BFF5
:1005B00048CD0120034B586C10B103681B681847E5
:1005C000704700BF48CD0120034B986C10B1036801
:1005D0001B681847704700BF48CD0120034BD86CFB
:1005E00010B103681B681847704700BF48CD012051
:1005F000034B186D10B103681B681847704700BFA4
:1006000048CD0120034B586D10B103681B68184793
:10061000704700BF48CD0120034B986D10B10368AF
:100620001B681847704700BF48CD0120034BD86DA9
:1006300010B103681B681847704700BF48CD012000
:10064000034B186E10B103681B681847704700BF52
:1006500048CD0120034B586E10B103681B68184742
:10066000704700BF48CD0120034B986E10B103685E
:100670001B681847704700BF48CD0120034BD86E58
:1006800010B103681B681847704700BF48CD0120B0
:10069000034B186F10B103681B681847704700BF01
:1006A00048CD0120034B586F10B103681B681847F1
:1006B000704700BF48CD0120034B986F10B103680D
:1006C0001B681847704700BF48CD0120034BD86F07
:1006D00010B103681B681847704700BF48CD012060
:1006E000034BD3F8800010B103681B6818477047AC
:1006F00048CD0120034BD3F8840010B103681B6878
:100700001847704748CD0120034BD3F8880010B13B
:1007100003681B681847704748CD0120034BD3F886
:100720008C0010B103681B681847704748CD012042
:10073000034BD3F8900010B103681B68184770474B
:1007400048CD0120034BD3F8940010B103681B6817
:100750001847704748CD0120034BD3F8980010B1DB
:1007600003681B681847704748CD0120034BD3F836
:100770009C0010B103681B681847704748CD0120E2
:10078000034BD3F8A00010B103681B6818477047EB
:1007900048CD0120034BD3F8A40010B103681B68B7
:1007A0001847704748CD0120034BD3F8A80010B17B
:1007B00003681B681847704748CD0120034BD3F8E6
:1007C000AC0010B103681B681847704748CD012082
:1007D000034BD3F8B00010B103681B68184770478B
:1007E00048CD0120034BD3F8B40010B103681B6857
:1007F0001847704748CD0120034BD3F8B80010B11B
:1008000003681B681847704748CD0120034BD3F895
:10081000BC0010B103681B681847704748CD012021
:10082000034BD3F8C00010B103681B68184770472A
:1008300048CD0120034BD3F8C40010B103681B68F6
:100840001847704748CD0120034BD3F8C80010B1BA
:1008500003681B681847704748CD0120034BD3F845
:10086000CC0010B103681B681847704748CD0120C1
:10087000034BD3F8D00010B103681B6818477047CA
:1008800048CD0120034BD3F8D40010B103681B6896
:100890001847704748CD0120034BD3F8D80010B15A
:1008A00003681B681847704748CD0120034BD3F8F5
:1008B000DC0010B103681B681847704748CD012061
:1008C000034BD3F8E00010B103681B68184770476A
:1008D00048CD0120034BD3F8E40010B103681B6836
:1008E0001847704748CD0120034BD3F8E80010B1FA
:1008F00003681B681847704748CD0120034BD3F8A5
:10090000EC0010B103681B681847704748CD012000
:10091000D0F89432012280F890221A6818461368A1
:10092000184700BFF8B50646044690F858700025F1
:1009300008E0042B1ED0022B26D00135082D04F12F
:10094000080416D0A0690028F7D0237F032BF0D12C
:1009500047FA05F3DA07F0D496F858302B41DB0755
:10096000EBD503681B6898470135082D04F108048E
:10097000E8D1F8BD96F858307B402B41DB07DCD539
:1009800003681B689847EFE747FA05F3D907D4D502
:1009900096F858302B41DA07CFD403681B68984784
:1009A000E2E700BF30B48369164C027F93F85830F9
:1009B0002568016982B01341019503F00103019A92
:1009C00081B14468521AA24209D3A3B981688A420C
:1009D0004FF0010334BF002201224275037502B0BB
:1009E00030BC7047002BFAD123680093009B036151
:1009F00002B030BC7047002303610375437502B039
:100A000030BC704774CE012010B4037A446859B9E1
:100A100094F85910012202FA03F30B43DBB284F875
:100A200059305DF8044B704794F85920012101FAC0
:100A300003F322EA030384F859305DF8044B70474E
:100A4000032910B5044617D004290BD0012900D082
:100A50000021201D00F094F804F10C00002100F0AA
:100A60008FF810BD0121201D00F08AF804F10C0060
:100A7000012100F085F810BD0021F4E710B54FF416
:100A800096730446013BFDD14068036801219B68D1
:100A900098470023237510BD0C4B0D4A197911702E
:100AA0001B680C4A1969131D994239BF5188138874
:100AB000D1889388084A0B44084908681BB2138000
:100AC00010B103681B681847704700BF2CCC012089
:100AD0001F8000400002FF1F38CC012034CC0120D1
:100AE000C368DA0706D55B1041688268C858825827
:100AF000C81810474168826801EB6300104700BFC7
:100B0000C368DA0706D55B1041688268C858825806
:100B1000C81810474168826801EB6300104700BFA6
:100B2000C368DA0706D55B1041688268C8588258E6
:100B3000C81810474168826801EB6300104700BF86
:100B4000C368DA0706D55B1041688268C8588258C6
:100B5000C81810474168826801EB6300104700BF66
:100B6000C368DA0706D55B1041688268C8588258A6
:100B7000C81810474168826801EB6300104700BF46
:100B80004368074ADBB211F0FF0F52F833304FF0E1
:100B9000010214BF83F8802083F80021704700BF52
:100BA000904A0200C9B200791BF09CBA08B50079DE
:100BB0001BF08AFA08BD00BFF8B590F84C33002B43
:100BC00000F0878090F8E43503B9F8BD0468D0F8E8
:100BD000D430E20081181B690D791B019BB22DB145
:100BE000CD88C5EBC5152B44C3F3CF13D0F86C6388
:100BF000CB80851833696E791B019BB22EB12D898C
:100C0000C5EBC5152B44C3F3CF1385182B818B7A05
:100C10003BB9CB884AF6A925AB4294BF00230123F8
:100C20008B720244D37A002B54D0631C0E2B88BFE6
:100C30000027044688BF3B4644F88C3B98BF1F46BC
:100C400006460025236847FA05F120469B6801F017
:100C5000010101359847042D04F10804F2D122491D
:100C600096F8D020D6F848034D2303FB0212002348
:100C7000125C86F84C3302F01F031F2B0CD012F0CD
:100C8000800FD6F8D42016BFD068102020F01000B6
:100C900043F04003D060136096F86823D6F8E0056F
:100CA0004D2303FB021300211A5C86F8E41502F0C1
:100CB0001F031F2B0DD012F0800FD6F86C2316BF28
:100CC000D168102121F0100143F04003D16013607E
:100CD000F8BDF8BD13894AF6A9218B4294BF0023C1
:100CE0000123D372A1E700BF1C46020038B5437B45
:100CF0008568023B012BEA78A97902D90223EB70BF
:100D000038BDD2B2D40629D453062CD4C9B211F0BE
:100D1000500F044612D0AB7943F05003AB71826898
:100D2000937903F0DF03937183680222DA70036919
:100D30000BB1406D98470223A5686373636D3F2B29
:100D400004D85A1C626523442A791A75AB7943F09A
:100D50005003AB71A3680222DA7038BD102352062B
:100D6000EB701BD58568002343658365AB7943F041
:100D70002003AB718368C0229A7083681A79520885
:100D800080F85C209A7942F050029A71836842227E
:100D9000DA70826803239279437338BD826893794D
:100DA00043F05003937183680222DA7038BD00BFAC
:100DB000002A31DB002B2FDB5F282DDCBF292BDC49
:100DC0005F2AF0B4A8BF5F2220EAE074BF2BA8BF5F
:100DD000BF23A242174621EAE1751E461BDBC5F17F
:100DE0000101194405EB45020C4B01EB410104EBF9
:100DF00042120137890103EB42020020AE42A8BF34
:100E0000002303DBD052C0339942FBD10134BC42F2
:100E100002F10202F2D1F0BC704700BF041A0120B7
:100E2000D0ED066AD0ED075AD0ED057A90ED037A41
:100E300030EE660A37EEC76AE5EE806AB4EEE66A1F
:100E4000F1EE10FAC0ED066A3FDD77EE267A836A8E
:100E5000C0ED057A4362002B46DDD0ED046A90EDCB
:100E6000026A76EEA66AF6EE005AB7EE005A66EE11
:100E7000255AF4EE456AF1EE10FA75EEC75AC8BF6E
:100E8000F0EE456AA5EEA67A013B436280ED037A57
:100E900090ED007AD0ED086A90ED010A37EE066A0F
:100EA00077EEC67AB0EE476AA7EEA66AB4EEC06ADD
:100EB000F1EE10FA08D5B4EEC67AF1EE10FA54BF8E
:100EC000B0EE470AB0EE460A704737EE876AB4EED6
:100ED000E66AF1EE10FA12D5836A436276EEC77ABB
:100EE000002BC0ED057AB8DC90ED026AD0ED045A13
:100EF00076EE476AA5EEA67A80ED037AC8E7436AE4
:100F0000A9E700BFD0ED037A70EE676AF5EEC06A1C
:100F1000F1EE10FA2ED43ADD90ED017A90ED025AFE
:100F2000DFED1E4A90ED006A77EE677A77EE455A5C
:100F3000F4EEE47AF1EE10FA65EEA65AD8BFF0EEC0
:100F4000647AC5EEA76A76EE857AB4EEE77AF1EEBA
:100F500010FA08DDB4EEE76AF1EE10FA54BFB0EE15
:100F6000467AB0EE677A80ED030A80ED027AB0EE41
:100F7000470A704790ED006A90ED025ADFED074A8C
:100F800090ED017A77EEC67A75EE465AD0E790ED8D
:100F9000006A90ED017AD0ED027AD6E7BD3786354A
:100FA000D0F8C030C02B70B4044637D05F2B45DD7D
:100FB000602B31D007EE903ADFED236AB8EEE77A86
:100FC0000021DFED227A27EE267A084625460FE03B
:100FD000BF2AA8BFBF22BF2BA8BFBF23A25CE35C70
:100FE00001319342B8BF1346602913D005F8013B85
:100FF00077EE877A0346FDEEE76A421C16EE900A0A
:10100000C61A012EE4DCBF2BA8BFBF230131602923
:10101000E35CEBD184F85F3070BC7047431C411E29
:10102000C13413F8010C13F8022B8242B8BF0246F8
:101030009C4201F8012FF4D170BC7047C0220021FE
:1010400070BC1DF071BB00BFABAA2A3C00000000C1
:10105000F0B4002ABDF810402DDB002B2BDB5F28FD
:1010600029DCBF2927DC5F2AA8BF5F2220EAE070C5
:10107000BF2BA8BFBF238242174621EAE1751E4657
:1010800019DB591C491B05EB45020C4B01EB4101D7
:1010900000EB42120137890103EB4202AE42A8BFC6
:1010A000002303DBD452C0339942FBD10130B84254
:1010B00002F10202F2D1F0BC704700BF041A012015
:1010C000F0B4002ABDF810402EDB002B2CDB5F288B
:1010D0002ADCBF2928DC5F2AA8BF5F2220EAE07053
:1010E000BF2BA8BFBF238242174621EAE1761D46E7
:1010F0001ADB991B4908013106EB46020B4B01EB49
:10110000410100EB4212C90103EB4202B542A8BF04
:10111000002304DBD45203F5C0739942FAD10230A4
:10112000874202F10402F1DAF0BC7047041A012090
:101130002DE9F04F864B9DB0DD6A1B681393844BFD
:10114000002D5C68064640F37D81032D56DC304659
:101150001DF0B6FB3178002959D000284FF0000E61
:10116000ACBF07466FF00047F446701E012210F82E
:10117000013F33B99FB910F8013F4FF0FF37002B03
:10118000F8D00A2B04D01F2BF1D90EF1060EEEE792
:10119000F445B8BFF44601324FF0000EE7E76C4B60
:1011A000F445986A6346B8BF734605FB03F318938A
:1011B000674B083002FB00F2D868012805FB02F7F4
:1011C0002CD0022800F04181614B1B69012B30D0EB
:1011D000022B08BFE41B5E4B139AD3F818E01B6A7E
:1011E000DFF86CC103EB0E084245134603DA189A88
:1011F00013449E4522DB1DB0BDE8F08F544B032500
:101200003046DD621DF05CFB31780029A5D1504BE2
:101210001891D86801284FEAC507D2D1189B139AB4
:1012200003EBD373A2EB63031393494B1B69012BAD
:10123000CED107EBD773A4EB6304CCE7DCF81CE05A
:10124000DCF8243073449C42D5DA2744BE45D2DA18
:101250000029D0D00A96CDF86CC00A290A9B00F06C
:1012600018861E4600220B4602E00A2B00F09283ED
:101270001F2B16F8013F88BF0132002BF5D102EB7E
:1012800042025200199605FB02F2314B9B6A083369
:1012900005FB03FE0128AEEBC50600F0858302289E
:1012A00000F0EA85139B0393294B1B7D002B40F034
:1012B000D1800EEB04030B93022D06EB0403119374
:1012C00000F07B83032D40F0FB80002900F0978124
:1012D0000A2900F09481119C039B1D4D04EB4400EE
:1012E00003EB40101A4B2D891A6AD3F81880D3F8F3
:1012F0001CB05B6A04955B44059323460133154D8E
:101300001593A1F120030230DBB205EB400008EB9E
:10131000020A6B2B04F102020C900D9200F2108372
:101320000D4A52F823301E78079300230693039B3F
:10133000DDF834E0DDF854C0119FDDF830905A1C20
:10134000023308920993184603994C46002334E06F
:10135000D4190120041A012078300200804500F3DE
:101360005981824540F35681904540F36982BB45DF
:1013700005DC059DBD42C4BFBDF810502580E34586
:1013800006DC059D654503DDBDF81050A4F8C0508E
:10139000F34506DC059D754503DDBDF81050A4F846
:1013A00080510133062B01F1030104F1060402F11F
:1013B000030200F1030000F0488146FA03F5ED074F
:1013C000EFD58845CADC824500F38E814045C0F2E6
:1013D0005181904500F3BA818A4540F3C682BB45EE
:1013E00000F3CE82059DBD4240F3CA82BDF8105085
:1013F00024F8045C924506DDBDF8105024F8025C28
:101400008A4540F3A082E34500F39D82059D654532
:1014100040F39982BDF81050A4F8BC50924540F3B7
:10142000B282BDF81050A4F8BE508A4500F34D8139
:10143000F345B6DC059D7545B3DDBDF81050A4F845
:101440007E51AEE70125DD6281E6139B189A9B1A57
:101450001393B9E61B990B6A8869D1F81CC04F6ACF
:101460000493CB8A00930EEB04010B91049B039928
:1014700000EB030E0A44013A0EF1FF3E0CEB0703AA
:1014800072450B9FA8BF7246884203F1FF33B8BF75
:101490000846013FA4456146B8BF2146BB42A8BFEC
:1014A0003B46FFF7D5FD331911930A9B022D19789E
:1014B00000F08382032D3FF408AF002900F09F80E5
:1014C0000A2900F09C80BD4BBC4A98691E6AD3F87B
:1014D0001CB0119D5B6A128905925B4405EB4504C3
:1014E000039A0493630105320644069305F1080745
:1014F000A1F12003DBB26B2B96BFB149B14D51F87E
:101500002350069B119903929C18AF4B013D03EBAE
:101510004404A2F1050AA2F10409A2F10308A2F110
:10152000020C02F1FF3E15F8013FDA070CD55045D9
:101530000ADC564508DD594506DB049A9142BCBFDA
:10154000BDF8142024F80A2C9A070CD548450ADC6B
:101550004E4508DD8B4506DC049A8A42C4BFBDF8BF
:10156000142024F8082C5A070CD540450ADC4645BF
:1015700008DD8B4506DC049A8A42C4BFBDF81420FE
:1015800024F8062C1A070CD560450ADC664508DDF0
:101590008B4506DC049A8A42C4BFBDF8142024F8A7
:1015A000042CDA060CD570450ADC764508DD8B453F
:1015B00006DC049A8A42C4BFBDF8142024F8022C29
:1015C0009B060CD5039B984209DC9E4207DD8B45A8
:1015D00005DC049B8B42C4BFBDF81430238001316D
:1015E000B94204F1C0049ED10A9B039A13F8011F6B
:1015F0000A9321B10A2902F106027FF479AF199BFF
:101600000B9C197800293FF4F6AD0A936B4BDD6A09
:10161000D86822E690453FF7C4AE92457FF7C1AE49
:10162000BB4506DC059DBD4203DDBDF8105024F826
:10163000025CE3453FF7FCAE059D65457FF7F8AEDC
:10164000BDF81050A4F8BE50F2E6069B0133082BFB
:10165000069309F510790EF1030E07F103070CF15B
:10166000030C00F05681079B089A13F8016F07934B
:10167000099869E6904569DC8A4540F39480BB454A
:1016800000F32281059DBD4240F31E81BDF810503C
:1016900024F8045C924505DDBDF8105024F8025C86
:1016A0008A4574DDE34572DC059D65456FDDBDF857
:1016B0001050A4F8BC50924540F35081BDF8105032
:1016C000A4F8BE508A457FF7B3AEF3453FF769AE45
:1016D000059D75457FF765AEBDF81050A4F87C51A7
:1016E00092453FF7AAAE5CE64045C3DB92456DDC10
:1016F0008A4540F3ED80BB450CDC059DBD4209DD0C
:10170000BDF8105024F8045CBDF8105025808A45BF
:1017100040F3E480E3450DDC059D65450ADDBDF839
:101720001050A4F8BC50BDF81050A4F8C0508A4521
:101730007FF72EAEF3453FF734AE059D75457FF735
:1017400030AEBDF81050A4F87C5126E68A457FF7EC
:1017500028AEBB4506DC059DBD4203DDBDF810503B
:1017600024F8045CE34506DC059D654503DDBDF812
:101770001050A4F8BC50F3453FF713AE059D7545D6
:101780007FF70FAEBDF81050A4F87C5109E69245E2
:1017900005DDE34596DC059D654593DD8EE78A45CD
:1017A0007FF7FFAD91E79245F9DDBB453FF778AF95
:1017B000059DBD427FF774AF6EE700BFD4190120CD
:1017C00078300200C83F0200041A01208A456BDD10
:1017D000BB4569DC059DBD4266DDBDF8105024F8AF
:1017E000045C424567DA059DBD4202DDBDF810503C
:1017F00025808A454CDDE3454ADC059D654547DD8E
:10180000BDF81050A4F8BC50424548DA059D654526
:1018100003DDBDF81050A4F8C0508A4550DDF345F3
:101820004EDC059D75454BDDBDF81050A4F87C518C
:101830004245FFF6AFADBDF81050A4F87E51ACE5BF
:10184000924553DDBB450BDC059DBD4208DDBDF86F
:10185000105024F8025CBDF81050258092454ADDF6
:10186000E3450DDC059D65450ADDBDF81050A4F883
:10187000BE50BDF81050A4F8C05092457FF788AD17
:10188000F3453FF78EAD059D75457FF78AADD2E7ED
:1018900042453BDBE345C0DC059D6545BDDDBDF84C
:1018A0001050A4F8BE50B4E742452BDBBB45A0DC8A
:1018B000059DBD429DDDBDF8105024F8025C95E702
:1018C0004245FFF665ADDBE792453FF76EAFE9E6CF
:1018D000BB4503DC059DBD423FF716AFE3453FF72F
:1018E00057AD059D65453FF71EAF51E5BB4502DC91
:1018F000059DBD42AFDCE3453FF74AAD059D65451B
:10190000B7DC45E5BB453FF774AF6CE7E34584DCE6
:101910007CE70A9B13F8011F0A93039B123303937E
:1019200000293FF46CAE0C9B0A2903F124030C93AD
:101930003FF465AEA1F12003DBB26B2B7FF6F0AC78
:10194000AD4B0026F0E492457FF729AFE3453FF722
:101950006CAD059D65457FF768AD62E58A453FF74B
:10196000B4AE92453FF764AD1BE592457FF717AFE4
:10197000BB453FF745AD059DBD427FF741AD3BE51A
:101980009245F5DC3FE58A453FF79FAE92457FF7EC
:1019900008AD4DE502EB42025200199605FB02F23A
:1019A00033460133199370E4189B13989B1A03EB89
:1019B000D37300EB6303039376E400293FF41FAE77
:1019C0000A293FF41CAE8D4B8C481A6A9C69D3F8E7
:1019D0001CB05B6A00891A900BEB0309039B04EBB4
:1019E00002085A1C0C921A460B33099313460A3309
:1019F000089313460933109313460833069313468E
:101A000007320F929A1D07925A1D0D921A1D0492C9
:101A1000DA1C02330593119B0E9201331593A1F149
:101A20002003DBB26B2BCA4600F26D81744A52F878
:101A300023502978039E119A159BDDF86890013692
:101A40000020129699E0CE0715D50C9EB442039E55
:101A500000F3B881A64280F223820C9FB8450ADDCC
:101A60005B4508DB534506DA03EB430607EB4616F6
:101A7000644F27F816908F0715D50E9EB442059E29
:101A800000F3B781B44240F30E820E9FB8450ADDE1
:101A90009B4508DC9A4506DD03EB430607EB46163B
:101AA000584F27F816904E0715D50D9EB442049E48
:101AB00000F32C81B44240F3EF810D9FB8450ADD5D
:101AC0009B4508DC9A4506DD03EB430607EB46160B
:101AD0004C4F27F816900F0715D50F9EB442079E5E
:101AE00000F32B81B44240F3E1810F9FB8450ADD3A
:101AF0009B4508DC9A4506DD03EB430607EB4616DB
:101B0000404F27F81690CE0615D5109EB442069E7B
:101B100000F32A81B44240F3CD81109FB8450ADD1D
:101B20009B4508DC9A4506DD03EB430607EB4616AA
:101B3000344F27F81690890615D509998C420899D3
:101B400000F329818C4240F39E81099EB0450ADD55
:101B50009B4508DC9A4506DD03EB430106EB41118A
:101B6000284E26F811900130082802F1020203F1F4
:101B7000020300F0938015F8011F93453FF763AF10
:101B8000924526DCCE0715D50C9EB442039E00F389
:101B90005C81A64280F27A810C9FB8450ADD9B45A4
:101BA00008DC9A4506DD03EB430607EB4616154FA6
:101BB00027F816908F077FF576AF0E9EB442059EEC
:101BC00000F33881B4423FF760AFB04500F338818D
:101BD0005BE7129F169002EB420607EB4616094F91
:101BE000179203EB430E07EB460677467F011497E7
:101BF000DDF80CE0002724E0C83F0200D4190120E2
:101C000078300200041A0120C64501DA26F8029C49
:101C10000EF1010C64451FDDC6450BDA9B4506DC61
:101C20009A4504DD149AA548724420F81290644540
:101C300040F3FC800137062F0EF1020E06F1040678
:101C400022D041FA07FC1CF0010FF3D0A645DBDAE5
:101C50000EF1010C6445EDDCE04540F3E180A64562
:101C6000A6F8009080F2DF809B45E3DC9A45E1DD39
:101C7000149A01379444914A062F22F81C900EF1D1
:101C8000020E06F10406DCD11698179A01300828D6
:101C900002F1020203F102037FF46DAF0A9B13F815
:101CA000011F0A93039B0C33039300293FF4A7AC55
:101CB0000C9B0C330C93099B0C330993089B0C333E
:101CC0000893109B0C331093069B0C3306930F9BC9
:101CD0000C330F93079B0C3307930D9B0C330D9321
:101CE000049B0C3304930E9B0C330E93059B0A2923
:101CF00003F10C0305933FF482ACA1F12003DBB2A6
:101D00006B2B7FF693AE6E4D002193E6B4423FF706
:101D1000E2AEB0457FF7DFAE9B4509DC9A4507DDB3
:101D2000049F03EB430607EB4616644F27F8169013
:101D30000D9EB4423FF7CFAEBFE6B4423FF7E3AEED
:101D4000B0457FF7E0AE9B4509DC9A4507DD079F6C
:101D500003EB430607EB4616584F27F816900F9EE5
:101D6000B4423FF7D0AEC0E6B4423FF7E4AEB04570
:101D70007FF7E1AE9B4509DC9A4507DD069F03EB43
:101D8000430607EB46164D4F27F81690109EB442B7
:101D90003FF7D1AEC1E68C423FF7E5AE88457FF70D
:101DA000E2AE9B4509DC9A4507DD089E03EB430143
:101DB00006EB4111414E26F8119009998C423FF7EC
:101DC000D2AEC2E6A642FFF656AE4645BFF653AEC9
:101DD0009B4509DC9A4507DD039F03EB430607EBB0
:101DE0004616364F27F816900C9EB4423FF743AE86
:101DF00033E6B4423FF757AEB0457FF754AE5B458C
:101E000009DB534507DA059F03EB430607EB46164C
:101E10002A4F27F816900E9EB4423FF744AE34E6A0
:101E2000A645FFF607AFC645FFF6F8AEE0453FF71B
:101E30001BAFFFE6B4423FF736AEB0457FF733AE97
:101E40009B45E8DC9A45E6DDDDE7A642FFF6B2AE4B
:101E50004645BFF6AFAE9B4509DC9A4507DD039FBB
:101E600003EB430607EB4616144F27F816900C9E1B
:101E7000B4423FF79FAE8FE6189B13989B1A03441A
:101E80000393FFF711BA88458BDC5EE64645E2DB3B
:101E900082E61993002284E5B0453FF73DAF0CE69A
:101EA000464595DBD9E5B045A9DCEEE5B0453FF701
:101EB0004AAF1AE6B0453FF75DAF2EE6041A01209F
:101EC000C83F020070B5D0F8D80A134B0244013164
:101ED00092F890215960811882B091F8DC1511F0C8
:101EE000020F0CBF2026562611F0010F4FF0000202
:101EF00014BF4E24202420211E2501A80192DA605F
:101F00008DF804601A611D608DF806408DF805108B
:101F1000FFF70EF902B070BDD41901202DE9F0438E
:101F200083B0054641F2A5408946904605F10B0372
:101F3000691C00905D220220FFF78AF805F10C066B
:101F40004FF6FF7701223346294610460097FFF7E8
:101F50007FF82B46294600975E220120FFF778F88C
:101F60005E2233462946104600971A4CFFF770F858
:101F70003346314600975E220120FFF769F8EE1CD8
:101F80004FF0010E002560214846C0220223C4F80C
:101F90002CE021626262236027816660A562E560B1
:101FA00025612575E582A561E561FFF7C1F840F27D
:101FB000214219230848236066602281FFF7B8F8A0
:101FC0002523404666602581236003B0BDE8F043C9
:101FD000FFF7AEB8D4190120103D0200F0B5654CF2
:101FE000057854F825400C41E40707D50239052946
:101FF00004D8DFE801F01422344352050020F0BD7C
:10200000082ACCBF092122EAE27290F90830D4BF35
:1020100051B20A460172981A18BF0120F0BD612A18
:10202000CCBF622122EAE2724378D4BFD1B20A4621
:102030004170981A18BF0120F0BD40F2E6339A4271
:10204000CCBF40F2E73122EAE272B0F90A30D4BFE5
:1020500011B20A464181981A18BF0120F0BD464BC3
:1020600002321340002B6EDBDBB2837023B1C378E6
:10207000032B04BF0023C3700120F0BD622A5FDC84
:1020800012F1620F5ADA6FF062010A4690F90930D4
:102090004172981A18BF0120F0BD384EC778541D00
:1020A00086FB041EE117C1EB6E0101EB8101611A91
:1020B000C9B2D21BC170A1D087780C46AFB9012D2F
:1020C00046D0374601E0E1B2C1708D18053587FB77
:1020D0000546EC17C4EB660404EB84040429A5EB65
:1020E0000404F0D09942EED0C6E7012D16D0374651
:1020F00001E0E1B2C1708D18053587FB0546EC178C
:10210000C4EB6604CE1E04EB8404012EA5EB04048C
:10211000EFD99942EDD0AFE7E1B2C170551805355E
:1021200086FB0547EC17C4EB670404EB8404032922
:10213000A5EB0404F0D08B42EED09DE751B2A5E7A9
:1021400063210A46A2E7013B63F0010301338BE7F9
:102150001A44551D86FB0521EA17C2EB610101EB0C
:10216000810101E0C270D4B2A342A5EB0102F9D013
:1021700082E700BFD43C020001000080676666660B
:10218000114B027853F822300B41DB0716D5023988
:10219000052916D8DFE801F006080B0D100390F9A9
:1021A0000800704740787047B0F90A00704780789F
:1021B000704790F909007047C07870476FF00100D0
:1021C00070474FF0FF30704720430200F0B50468BD
:1021D000BB4A48F6907303FB04F3D11843F2FC1595
:1021E0004E5D042E00F01F81D0F8D8104FF0FF3361
:1021F00000220229C0F88830C0F89C31C0F8A03114
:1022000080F8902100F0E8800329C0F8942100F0C4
:10221000C5800023C0F89831D0F8D8114FF0FF33B3
:102220000022022980F89022C0F89C32C0F8A03227
:1022300000F0BA800329C0F8942200F0A98000239E
:10224000C0F89832D0F8D8124FF0FF33002202299C
:1022500080F89023C0F89C33C0F8A03300F0B4801D
:102260000329C0F8942300F08D800023C0F8983330
:10227000D0F8D8134FF0FF330022022980F89024C1
:10228000C0F89C34C0F8A03400F096800329C0F850
:10229000942472D00023C0F89834D0F8D8144FF0AA
:1022A000FF330022022980F89025C0F89C35C0F841
:1022B000A03500F0A1800329C0F8942558D0002350
:1022C000C0F89835D0F8D8154FF0FF330022022916
:1022D00080F89026C0F89C36C0F8A03600F08480C4
:1022E0000329C0F894263ED00023C0F89836D0F8D1
:1022F000D8164FF0FF330022022980F89027C0F84B
:102300009C37C0F8A03700F086800329C0F89427D6
:1023100024D00023C0F89837D0F8D8174FF0FF33F7
:102320000022022980F89028C0F89C38C0F8A03814
:102330006AD00329C0F8942807D00023C0F8983841
:102340004FF0FF33C0F86C39F0BD90F80238002B25
:10235000F3D14FF0FF33C0F86C39F0BD90F802377D
:10236000002BD9D0D5E790F80236002BBFD0BBE7C1
:1023700090F80235002BA5D0A1E790F80234002B8D
:102380008BD087E790F80233002B3FF471AF6CE7F6
:1023900090F80232002B3FF455AF50E790F802312D
:1023A000002B3FF439AF34E790F8F631002B3FF4BF
:1023B00046AFC0F8942242E790F8F633002B3FF482
:1023C00069AFC0F8942465E790F8F632002B3FF42B
:1023D0004CAFC0F8942348E790F8F630002B3FF458
:1023E00018AFC0F8942114E790F8F635002B3FF4AD
:1023F0007BAFC0F8942677E790F8F634002B3FF4D3
:102400005EAFC0F894255AE790F8F637002B94D0C9
:10241000C0F8942891E790F8F636002B3FF479AF96
:10242000C0F8942775E74CF2781744F2A006CF590C
:1024300006FB0733D61806F57E5EDEED007A06F55C
:102440007D5393ED0D7AF8EEE77A67EE877AF5EE35
:10245000407AF1EE10FA24D043F6687543F65C73C7
:102460007159F358591A9F2943F6707EC8BFA3F1DA
:10247000A0014FF0000C06F80EC0C8BF715148F61D
:10248000907101FB04F444F2A00101FB07473A44B8
:1024900043F66C741159C91A9F29C4BFA033135154
:1024A000A2E64CF27C134FF0FF32CA5001F54852BD
:1024B0000324136823F0240313604C5594E600BFF3
:1024C000A81CFF1F2DE9F04F0168DFF88C8348F648
:1024D000907303FB01F308EB030243F2FC1483B097
:1024E000155D042D00F06781DFF86CB300F644360B
:1024F00000F5356E48F6907900224FF0FF3156F81E
:10250000043F1868009009FB00F408EB040505F58A
:1025100047503C3090F800C0BCF1040F00F0F88048
:10252000D3F8D800C3F88810022883F89021C3F8A4
:102530009C11C3F8A01100F0E3800328C3F8942194
:1025400000F0D880C3F89821D3F8D80183F89022FE
:102550000228C3F89C12C3F8A01200F0C38003281D
:10256000C3F8942200F0B880C3F89822D3F8D802B8
:1025700083F890230228C3F89C13C3F8A01300F03B
:10258000A3800328C3F8942300F09880C3F898230D
:10259000D3F8D80383F890240228C3F89C14C3F816
:1025A000A01400F083800328C3F8942479D0C3F8E2
:1025B0009824D3F8D80483F890250228C3F89C15F2
:1025C000C3F8A01566D00328C3F894255DD0C3F8DE
:1025D0009825D3F8D80583F890260228C3F89C16CE
:1025E000C3F8A0164AD00328C3F8942641D0C3F8F4
:1025F0009826D3F8D80683F890270228C3F89C17AA
:10260000C3F8A0172ED00328C3F8942725D0C3F809
:102610009827D3F8D80783F890280228C3F89C1885
:10262000C3F8A01812D00328C3F8942809D0C3F81F
:102630009828B645C3F86C197FF461AF03B0BDE8C4
:10264000F08F93F802080028F1D1F2E793F8F6072B
:102650000028ECD0C3F89428E9E793F80207002893
:10266000D5D1D6E793F8F6060028D0D0C3F8942742
:10267000CDE793F802060028B9D1BAE793F8F6053A
:102680000028B4D0C3F89426B1E793F802050028D7
:102690009DD19EE793F8F604002898D0C3F89425BE
:1026A00095E793F80204002881D182E793F8F603B6
:1026B00000283FF47CAFC3F8942478E793F8020332
:1026C00000287FF463AF63E793F8F60200283FF435
:1026D0005DAFC3F8942359E793F8020200287FF412
:1026E00043AF43E793F8F60100283FF43DAFC3F84A
:1026F000942239E793F8020100287FF423AF23E7FF
:1027000093F8F60000283FF41DAFC3F8942119E7B1
:1027100005F5414CDCF878A044F2A00C0CFB0A440F
:102720000BEB040C27460CF57E540194494C2744CE
:1027300007F554542746019C97ED067AD4ED007AAC
:10274000F8EEE77A67EE877AF5EE407AF1EE10FA66
:1027500024D00CF57D5005468446C46980F83020AD
:10276000806A201A9F2805F11C050CF1280C03DD56
:10277000A03CCCF800402C68009809FB00F744F21C
:10278000A00000FB0A70404400F57D502C30056825
:102790002D1B9F2DC4BFA0340460C1E605F5414444
:1027A00005F54855E1672C6824F024042C604FF0AF
:1027B00003040470B4E64CF2781644F2A00596596E
:1027C00005FB063308EB030505F57E57D7ED007AC8
:1027D00005F57D5393ED0D7AF8EEE77A67EE877A8B
:1027E000F5EE407AF1EE10FA25D043F6687443F620
:1027F0005C7343F67077EA582B59D31A9F2BC8BFE6
:10280000A2F1A0034FF0000E05F807E0C8BF2B515E
:1028100048F6907303FB01F144F2A00303FB061397
:10282000434443F66C741959891A9F297FF75CAEAB
:10283000A0321A5158E64CF27C134FF0FF31D150C0
:1028400002F5485103250B6823F024030B6015554E
:102850004AE600BF0427FF1FA81CFF1FF0B5148C19
:10286000D0F87459DFED2F6AC66AC0F8781907EE00
:10287000904AD0F8D84AC0ED106AF8EE677A00277F
:1028800005EB4101C0ED117AC0ED127AC763264411
:10289000B1F802E096F89051528CDFED234A07EE32
:1028A00010EA06EE102A04EB850292ED7D5AC0ED87
:1028B000146AB8EEC77AB8EEC55A27EE247AB8EE95
:1028C000466AC7EE055AC764184A83B01268019277
:1028D000019D002280ED156A25EEA67A80ED166A2C
:1028E00080ED117A498B96F8906107EE901A04EB0F
:1028F000860494ED7D6AC0F87C59F8EEE77AB8EE6C
:10290000C66A67EEA47AC0F8BC2987EE867AC0F85A
:10291000C02967EE266AC0ED156AFFF7D3FD03B044
:10292000F0BD00BF00FF7F470000004274CE0120D1
:102930002DE9F84FD0F8D87AC26207EB020A0446B4
:102940009AF8903107EB43034FF0000EB3F88493ED
:10295000C0F830909AF8903107EB43031546B3F86E
:102960004C84C0F83480012200F6F80B80F85D201A
:102970000E4684F85CE07146602258461BF0D4FE97
:10298000D4F800E067489AF8903148F6907202FB5C
:102990000EF2811843F6142C51F80CC0BCF1000F54
:1029A0002CDB01F547523032D2F8587D7A0771D4CA
:1029B0005D4A48F6907101FB0E0002FB0CFC00F52D
:1029C0007D5E0CF1050C41F27172CEF8003002FB15
:1029D00003C243F6487143F6447C43F64C7347F018
:1029E0000907475040F80C2040F803B0D4F8D87AD3
:1029F000D4F83090D4F8348007EB050A338CDFED3F
:102A00004B7A9FED4B6AC4ED107A07EE103AB8EEA0
:102A1000477A002284ED117AE26384ED127A9AF803
:102A20009031718C06EE909A07EB8303D3ED7D5ABB
:102A3000E264B8EEE65AF8EEE55A25EE065A07EEDD
:102A4000101AC5EE256A0022B8EE477A66EEA76A2C
:102A500084ED157AC4ED147A84ED167AC4ED116A0A
:102A60009AF8903107EE108A07EB8307D7ED7D6A5D
:102A7000C4F8BC29B8EEC77AF8EEE66A27EE066A13
:102A8000C4F8C02986EE267A67EE277AC4ED157A57
:102A9000BDE8F88F01F57D521268934288D144F267
:102AA000C872194443F2E47702FB0E3303F5B353C3
:102AB000CA5D00EB4303D207B3F85C3A28D4B7EE03
:102AC000007A48F6907303FB0EF303F5755203F595
:102AD000775333321333024404F6F701184412F8E3
:102AE000013F07EE903AF8EEE77A904267EE877A78
:102AF000FCEEE77A17EE903A01F8013FEFD1D4F8F7
:102B0000D87AD4F83090D4F8348007EB050A75E70A
:102B100007EE903ADFED076AF8EE677A86EEA77A5D
:102B2000CFE700BFA81CFF1F2828090000FF7F4730
:102B30000000004200FEFF4630B57F4C83B02468A1
:102B40000194019DC46905F03F0504F03F041F2D69
:102B50008CBF002501251F2C8CBF00240124A54219
:102B60001CBF012480F8644090F87049002C78D193
:102B70000468012C02F10A0575D0032B7BD09C421E
:102B80006FD0072B6DD1D0F8C0399D4200F0C280C4
:102B9000B2F90A40DFED697A4B8CDFED695ADFED5F
:102BA000694AC0F8C05907EE104AF8EEC76A06EE47
:102BB000103A86EEA77A00F6AC1300F6B411B8EE20
:102BC000466A27EE257A83ED036AC3ED015AC3ED09
:102BD000004AF0EE657AB0EE645AF0EE466A81ED96
:102BE000007A76EE665AF5EEC05AF1EE10FA00F170
:102BF000828012DD77EEE66A9FED534A77EEC74A90
:102C0000F4EEC46AF1EE10FA64EEA55AD8BFF0EE05
:102C1000446AC5EEA64A37EE247AF4EEC77AF1EE9E
:102C200010FA08DDB4EEC75AF1EE10FA54BFF0EE18
:102C3000457AF0EE477ADFED456AC3ED027A9FED03
:102C4000447A83ED036A67EEA67A67EE877AFDEE33
:102C5000E77A17EE903AA3421CBF012180F8431B8C
:102C6000538103B030BD33B1012BFAD0072B8AD08A
:102C7000042BF6D187E7D0F8BC399D4242D0B2F997
:102C80000A309FED2E6ADFED2E6A07EE103AB8EE9D
:102C9000C77A0B8CC0F8BC59C7EE067A002400F640
:102CA000A41100EE103A67EEA67A00F69C13B8EE77
:102CB000400AC3ED016A1C6083ED030AC1ED007A8E
:102CC000054618461446FEF71DF9DFED207A9FED04
:102CD000207AB4F90A2020EE270A20EE070AFDEE3A
:102CE000C07A17EE903A93421CBF012285F8432B1D
:102CF000638103B030BD76EEC56A9FED134A77EE6F
:102D0000454A7DE70B8C00EE103A00F69C13B8EEB6
:102D1000400AD5E74B8CB2F90A4006EE103A00F6AD
:102D2000AC13B8EE466AD3ED036A93ED027A93EDE5
:102D3000005AD3ED017A54E774CE012000C07944E3
:102D400000FF7F4700000000BD37863500007A4451
:102D5000000080372DE9F04FD0F8603990F85E9090
:102D600090F85FA02DED068B07EE903A85B0F8EE57
:102D7000E77A00244FF0FF3300F65C17C7ED007AC6
:102D80000646DFEDC88A9FEDC88A9FEDC89A9FED81
:102D9000C8AADFEDC89A029288460546C0F86C3989
:102DA000C0F8643901940094A3461EE003EB43028B
:102DB000210201EB820232440A2B02F1DC0200F014
:102DC000D080042B00F0A380062B00F0A580022BFE
:102DD00000F0D4800B2B00F0F680032B00F027824C
:102DE0000134082C05F580752FD0D5F8D830092B83
:102DF000DCD1B14A95F9513152F82420B5F952117C
:102E0000083207EE101A38F8122003FB02F307EE1F
:102E1000903AF8EEE77AB8EEC77A67EE8A7AF7EE7C
:102E2000006AE7EE297AF4EEE67AF1EE10FA78D449
:102E3000F2EE007A97ED007A013467EE277A082CDB
:102E4000C7ED007A05F58075CFD1D6F86439002B2F
:102E5000C0F23E813168994A48F6907303FB012322
:102E600043F2FC100D461C5C042C00F038821B5C05
:102E7000052B40F03C824FF0FF3448F6907303FB83
:102E800001214CF26C130020C8523168002CC0F2B2
:102E90009182D6F86439E51A85EAE570A0EBE57011
:102EA00040F22945A84240F314821B1B002BCCBFE3
:102EB000A3F22A4303F22A4307EE903A9FED807A69
:102EC000F8EEE77A67EE877AB2EE007AF4EEC77A28
:102ED000F1EE10FA40F14082BAEE007AF4EEC77AD1
:102EE000F1EE10FAD8BFF0EE477AB0EE676AC7EDA0
:102EF000007A0D4606F5186406F6841106F5196683
:102F000000200023206008601C4630606DE195F8C9
:102F1000923149EA030963E795F891314AEA030AD5
:102F20005EE7F5EEC07AF1EE10FA40F3C5819FED51
:102F3000657A654B67EE877ABDEEE77A17EE102A61
:102F400003EB8202B8EEC77AD2ED006A92ED016A15
:102F500077EEC77A36EE667AE7EE876AF0EE667A43
:102F600068E7234641463046FFF7E6FD524A95F9A9
:102F70005D3152F82420B5F95E1141E73368012B29
:102F800000F09D8124F00403032B00F09C81D5F810
:102F90009431002B3FF424AF5B450BD8D6F86C2955
:102FA000002AFFF61DAF06EB0222D2F8D820032A32
:102FB0007FF416AFC6F86C499B46B5F9FE30009316
:102FC000002301930CE796F87039002B7FF408AFCB
:102FD000394B53F82430083306F6681238F81330AA
:102FE000D2ED007A00EE103AB8EEC00A20EE280AC0
:102FF00070EE677AF0EEE77AF4EEC87AF1EE10FA46
:1030000007DD06F69C2106F6982381ED000A83ED84
:10301000000A06F684200392FDF702FFD6F8643911
:10302000039A002B82ED000ABFF6DAAED6F8D83A42
:1030300095F8E9201A4492F89021632A3FF6D0AE21
:1030400003EB8201D1F8F41100297FF7C9AE03EB3D
:103050004203B3F88423B3F84C3407EE902A07EE0A
:10306000103AF8EEE77AB8EEC77A67EE897A27EE7B
:10307000097AFDEEE77ABDEEC77A17EE902A17EED1
:10308000103A9B1AF8EEE76A07EE903AF8EEE77A04
:10309000E0EE276AFDEEE67A17EE903AC6F864395C
:1030A0009EE600BF80008037ABAA2A3D00000042A8
:1030B0005A7F25340534833AC8440200A81CFF1FF8
:1030C000CDCCCC3A00802A44283202006F12833AD9
:1030D000B9F1000F05D0D7ED007AF1EE677AC7EDB0
:1030E000007ABAF1000F01D000233B60D6F86C39AA
:1030F000D6F89809834200F0FD80002BC0F21381BE
:10310000009A1FED0E7A013207EE902A06EB032299
:10311000F8EEE77AD2F8D81067EE877A06F68812CA
:1031200006F68C140329C2ED007AC4ED007A00F093
:103130001B8106F5186106F68414834200F00F81A6
:10314000019A9E48092AA8BF092200EB820292ED4B
:10315000006A06F6941006F5196282ED006A80EDA9
:10316000006AC6F898399DED027AF8EEC76AF4EE67
:10317000C66AF1EE10FAC0F2868006F68C1393ED63
:10318000007AC1ED007A84ED007AF5EEC07AF1EEB6
:1031900010FA97ED006A356840F3028167EE076A1E
:1031A0009FED875ADFED875A874A67EEA77AB1EE1F
:1031B000047AF0EE474AE7EE854AA6EE857AB0EE4D
:1031C000C65A27EE057A64EE856AF7EE007AB0EE0D
:1031D000675AA6EEA55AE7EE257ABDEEC57AFDEE52
:1031E000E77A17EE104A17EE903A48F6907101FB15
:1031F00005F1551805F54850734A0068460711D582
:10320000800638D54CF2781644F2A000AD59002D56
:1032100018BF002001440A4402F57D5282ED0D6A78
:103220009463D36305B0BDEC068BBDE8F08F3368C3
:10323000012B6FD024F00403032B6ED0D5F8983106
:10324000002B3FF4CDAD5B457FF6CAADD6F86C29B7
:10325000002A06DB06EB0222D2F8D820032A7FF4EC
:10326000BFADC6F86C49B5F90A21009295F908215D
:1032700001929B46B4E54CF2781044F2A00628581F
:1032800006FB0011C7E7C6EE865A91ED005A94ED91
:10329000007A77EEC57A77EE474AA5EEA75AA5EEF3
:1032A000A47A76EE666A81ED005AF0EE457A84EDF6
:1032B000007AC2ED006A68E7DFED447ABAE534F0DF
:1032C00004037FF464AE234641463046FFF734FCE6
:1032D0005DE69FED3F6A0D4687ED006A0AE6185CE1
:1032E0004CF27C1405281C597FF4D0ADC5E597ED50
:1032F000006AFFE5002BBFF603AF06F5196206F67C
:10330000881392ED006AD3ED007A06F5186106F68F
:10331000841428E734F0040390D123464146304614
:10332000FFF70AFC8AE706F6941292ED006A9FED19
:10333000287A06F68C1106F6881006F5196280EDDB
:10334000007AF0EE477A81ED007A06F6841406F5ED
:10335000186182ED006A04E7F0EE477AC5E506F5EC
:10336000196292ED006AFCE606F51861D1ED006A7B
:103370009FED187AF5EEC06A27EE877AF1EE10FA23
:1033800084ED007A06F684143FF6D7AE94ED007A09
:10339000B5EEC07AF1EE10FA98BFC1ED007ACCE636
:1033A000B5EEC07AF1EE10FA3FF7F8AE0023064A08
:1033B0001C461AE70D4697ED006A9BE57C45020026
:1033C0000000754300000042A81CFF1F0000003DE4
:1033D00000000000D7A3703F83691B02C21892F857
:1033E000EB10042900D0704730B4D0F8D85A92F8C6
:1033F000E9402C4494F89011632913D805EB81041B
:10340000D4F8F441002C0DDDD2F8EC4054B129443D
:1034100091F8DC3503F0020303F0FF0133B982F8C1
:10342000EB1003E00344002283F8EB2030BC70472C
:10343000D0F8482B436810B45468A3420CD0D0F89D
:103440004C2B5468A34225D0D0F8502B54689C4292
:1034500011D05DF8044B70479042F0D0D46AA1427D
:10346000EDD192F87049042C01D0022CE7D101244F
:1034700082F87A40E3E79042EBD0D36A8B42E8D1FE
:1034800092F87039042B01D0022BE2D1012382F88B
:103490007A30DEE79042D7D0D46AA142D4D192F8F4
:1034A0007049042C01D0022CCED1012482F87A403C
:1034B000CAE700BFFE2843D0431E03F0FE03FE2BE5
:1034C00022D0D12B22DCA92B22DC872B22DC692BFA
:1034D00022DC512B22DC3D2B22DC2B2B22DC1F2B70
:1034E00022DC152B22DC0D2B22DC092B22DC052B08
:1034F00022DC032B22DC012BD4BF00230123C207D3
:103500004CBF581CD84370470F23F8E70E23F6E74B
:103510000D23F4E70C23F2E70B23F0E70A23EEE791
:103520000923ECE70823EAE70723E8E70623E6E7B1
:103530000523E4E70423E2E70323E0E70223DEE7D1
:103540006FF00F00704700BF2DE9F04392F871391A
:10355000013B85B016460C46032B15D8DFE803F077
:10356000A6029717554A564904F10E00FEF7D6FCFD
:10357000544A554904F11E00FEF7D0FC04F12E0018
:10358000524A5349FEF7CAFC05B0BDE8F08304F186
:103590000E00504A4A49504DFEF7C0FC41F2A54387
:1035A000009304F11F0104F129035D22022004F1BC
:1035B0001E0704F12A084FF6FF79F668FDF748FD6B
:1035C0000122394643461046CDF80090FDF740FDF4
:1035D0003B463946CDF800905E220120FDF738FDCC
:1035E0005E22394643461046CDF80090FDF730FD87
:1035F00043464146CDF800905E220120FDF728FDAC
:1036000001200027602104F12108C0220223E86282
:10361000324829626A622B60AF62EF602F612F75BA
:10362000EF82AF61EF612F81C5F80480FDF780FD67
:1036300040F2214231232A482A812B60C5F80480B8
:10364000FDF776FD274AA5F80890731C82FB03213D
:10365000DA17C2EBA10202EB8201A3EB4103303384
:1036600003A83721303229608DF80D308DF80C20F9
:10367000C5F804808DF80E70FDF75AFD04F12E0098
:10368000124A1349FEF74AFC05B0BDE8F08304F185
:103690000A00154A0A49FEF741FC04F12A000B4AC8
:1036A0000B49FEF73BFC05B0BDE8F0830F4A044927
:1036B00004F10E00FEF732FC0D4A5AE7403D0200CD
:1036C000203D0200483D0200303D0200343D020032
:1036D0003C3D0200503D0200D41901205C3D020037
:1036E000643D020067666666683D0200143D0200A4
:1036F000243D0200F0B43C4C40F6583303FB014338
:10370000D3F8483B93F8602022B993F8702900322F
:1037100018BF012240F6583303FB0143D3F84C5B3A
:1037200095F8603033B995F87039002B0CBF13460B
:1037300042F0010340F6583202FB0142D2F8502B0E
:1037400092F860502DB340F6583303FB014393F8D1
:103750006020E2B993F87039CBB905788C0105B3D4
:1037600004EBC114A30103F5425420493E34BE3397
:103770000C4442F663401944A1F1C00333F8022F10
:1037800002B118809942F9D1C031A142F4D1F0BC04
:10379000704792F87029002AD5D1002BD3D1F0BC04
:1037A000704704F13F07BF2F24EAE4743E46A8BFE8
:1037B000BF26311B01310D4B01EB410104EB4402EB
:1037C000890103EB82122846FE2F06D8A64204DBAD
:1037D0000023D052C0338B42FBD10235602D02F161
:1037E0000402F1D1F0BC704704AA0120041A0120A0
:1037F00001380B463A2800F25C82DFE810F05302F1
:103800004C0245023E0237023002290222021B020C
:10381000AE01A701A001990192018B0184017D01F4
:1038200076016F01680161015A0153014C014501A4
:103830003E0137013001290122011B0113010B0157
:103840000301FB00F300EB00E300DB00D300CB003F
:10385000C300BB00B300AB00A3009B0093008B0030
:1038600083007B0073006B0063005B0053004B0020
:1038700043003B00BC48BD49C0F8EC201A463B2041
:1038800018F04EBAB848BA49C0F8E8201A463A20AB
:1038900018F046BAB448B749C0F8E4201A463920AF
:1038A00018F03EBAB048B449C0F8E0201A463820B3
:1038B00018F036BAAC48B149C0F8DC201A463720B7
:1038C00018F02EBAA848AE49C0F8D8201A463620BB
:1038D00018F026BAA448AB49C0F8D4201A463520BF
:1038E00018F01EBAA048A849C0F8D0201A463420C3
:1038F00018F016BA9C48A549C0F8CC201A463320C7
:1039000018F00EBA9848A249C0F8C8201A463220CA
:1039100018F006BA94489F49C0F8C4201A463120CE
:1039200018F0FEB990489C49C0F8C0201A463020D3
:1039300018F0F6B98C489949C0F8BC201A462F20D7
:1039400018F0EEB988489649C0F8B8201A462E20DB
:1039500018F0E6B984489349C0F8B4201A462D20DF
:1039600018F0DEB980489049C0F8B0201A462C20E3
:1039700018F0D6B97C488D49C0F8AC201A462B20E7
:1039800018F0CEB978488A49C0F8A8201A462A20EB
:1039900018F0C6B974488749C0F8A4201A462920EF
:1039A00018F0BEB970488449C0F8A0201A462820F3
:1039B00018F0B6B96C488149C0F89C201A462720F7
:1039C00018F0AEB968487E49C0F898201A462620FB
:1039D00018F0A6B964487B49C0F894201A462520FF
:1039E00018F09EB960487849C0F890201A46242003
:1039F00018F096B95C487549C0F88C201A46232007
:103A000018F08EB958487249C0F888201A4622200A
:103A100018F086B954486F49C0F884201A4621200E
:103A200018F07EB950486C49C0F880201A46202012
:103A300018F076B94C486949C2671A461F2018F039
:103A40006FB94948664982671A461E2018F068B95E
:103A50004548644942671A461D2018F061B942483A
:103A6000614902671A461C2018F05AB93E485F495E
:103A7000C2661A461B2018F053B93B485C4982665F
:103A80001A461A2018F04CB937485A4942661A4665
:103A9000192018F045B93448574902661A461820CB
:103AA00018F03EB930485549C2651A46172018F03B
:103AB00037B92D48524982651A46162018F030B998
:103AC0002948504942651A46152018F029B9264858
:103AD0004D4902651A46142018F022B922484B4974
:103AE000C2641A46132018F01BB91F484849826463
:103AF0001A46122018F014B91B48464942641A4667
:103B0000112018F00DB91848434902641A461020D4
:103B100018F006B914484149C2631A460F2018F03C
:103B2000FFB811483E4982631A460E2018F0F8B8D3
:103B30000D483C4942631A460D2018F0F1B80A4876
:103B4000394902631A460C2018F0EAB8064837498A
:103B5000C2621A460B2018F0E3B803483449826267
:103B60001A460A2018F0DCB848CD0120FD080000F4
:103B7000E9080000D5080000C1080000AD080000F9
:103B80009908000085080000710800005D08000029
:103B90004908000035080000210800000D08000059
:103BA000F9070000E5070000D1070000BD0700008D
:103BB000A907000095070000810700006D070000BD
:103BC0005907000045070000310700001D070000ED
:103BD00009070000F5060000E1060000CD06000020
:103BE000B9060000A5060000910600007D06000051
:103BF0006906000055060000410600002D06000081
:103C00001906000005060000F1050000DD050000B2
:103C1000C9050000B5050000A10500008D050000E4
:103C20007905000065050000510500003D05000014
:103C3000290500001F48204942621A46092018F051
:103C40006FB81C481D4902621A46082018F068B86F
:103C500018481B49C2611A46072018F061B8154878
:103C6000184982611A46062018F05AB811481649B8
:103C700042611A46052018F053B80E4813490261F4
:103C80001A46042018F04CB80A481149C2601A4676
:103C9000032018F045B807480E4982601A460220F2
:103CA00018F03EB803480C4942601A46012018F04B
:103CB00037B8704748CD0120150500000105000008
:103CC000ED040000D9040000C5040000B1040000A8
:103CD0009D040000890400007504000008B5134627
:103CE00040680A461946FFF783FD08BD2DE9F041FB
:103CF0004568AA6884B042F21071D3789E0640F1FC
:103D00008C800139F9D1917000BFAB6880229A7024
:103D100000BF01232B7343685A7B012A00F01D81E9
:103D20009A6D596D8A42C0F0C9800023056E80F8F3
:103D30005C30AA6842F21071D3789B064DD50139E8
:103D4000FAD1917000BFAB6880229A7000BF012346
:103D50002B73036E5A7B012A00F0B5809A6D596D62
:103D60008A42C0F0A6800023D0F8884280F8B8309C
:103D7000002C2FD0A24EA34F4FF0000801250FE0DA
:103D80006168821A8A4209D3002B40F08B80A068B8
:103D9000257590428CBF002201226275E468CCB187
:103DA00023681B68B3427AD1A369217F93F8583006
:103DB0003868226903900B4103F001030398002A3D
:103DC000DED1002BEAD13B680293029B2361E468B9
:103DD000002CE5D104B0BDE8F081B02190F8BA30F4
:103DE0009170AA68D478A70642F2107104D4013900
:103DF000A7D0D478A706FAD5D1788906A9D5917825
:103E000041F030019170A96842F21074CA789606A8
:103E100025D4013CFAD18C7094E7B02190F85E3043
:103E20009170AA68D478A40642F2107105D40139C1
:103E30003FF469AFD478A406F9D5D1788C067FF524
:103E40006AAF917841F030019170A96842F2107424
:103E5000CA78920613D4013CFAD18C7054E75B0007
:103E600043F00103DBB20B71AA6842F21073D17800
:103E700089073FF56EAF013BF9D1937062E75B00B4
:103E800043F00103DBB20B71AA6842F21073D178E0
:103E90008F073FF540AF013BF9D1937034E72046DF
:103EA00098477BE7C4F8108084F8148084F8158064
:103EB00074E7511C1A449965137D55E7511C1A4447
:103EC0009965137D32E700228DF806209C689DF8E5
:103ED000062042F21072E1780F060AD4013AFAD1B4
:103EE000A27000BF9A688021917000BF01221A73EE
:103EF00039E7A27802F0E702A2709A681179C9B294
:103F00008DF80610917841F0080191709A680221AD
:103F1000D1709A6842F21071D478A60703D401399F
:103F2000FAD19170DDE7917801F0C701917099683D
:103F300042F21072CC78A50659D5013AFAD18A70AE
:103F400000BF996880248C7000BF012499681C739D
:103F5000022413460A79CC7006E700228DF8072068
:103F60009C689DF8072042F21072E1780E060AD490
:103F7000013AFAD1A27000BF9A688021917000BF07
:103F800001221A73D1E6A27802F0E702A2709A68C1
:103F90001179C9B28DF80710917841F0080191703C
:103FA0009A680221D1709A6842F21071D478A507FC
:103FB00003D40139FAD19170DDE7917801F0C7019E
:103FC0009170996842F21072CC78A40613D5013A28
:103FD000FAD18A7000BF996880248C7000BF0124D8
:103FE00099681C73022413460A79CC709EE602225B
:103FF0000B79CA70B8E602220B79CA7096E600BF48
:10400000A509000074CE0120F8B5457D05B1F8BDC5
:1040100004464068036829469B689847A06803687F
:1040200029469B68984723681A684FF00041E323AC
:10403000D1625363D36A002BFCDAA068936B0368E8
:1040400000219B68984723681A684FF000411523A8
:10405000D1625363D36A002BFCDAA068936B0368C8
:1040600000219B68984723681A684FF0004100239D
:10407000D1625363D36A002BFCDAA068936B0368A8
:1040800000219B68984723681A684FF000415F231E
:10409000D1625363D36A002BFCDAA068936B036888
:1040A00000219B68984723681A684FF000417523E8
:1040B000D1625363D36A002BFCDAA068936B036868
:1040C00000219B68984723681A684FF0004100233D
:1040D000D1625363D36A002BFCDAA068936B036848
:1040E00000219B68984723681A684FF000413F23DE
:1040F000D1625363D36A002BFCDAA068936B036828
:1041000026699B681E4F012198472146002551F8DA
:10411000183BDA681068C571066001268680106851
:10412000866016684FF44050F0831268F760D082C2
:10413000DE681A68306834328571B2F1804F0261EE
:104140008582326817D2012090603268D8680D4DA0
:10415000066800209061B071DA681668F060127924
:104160002A701D682A6B012042F040722A6359614F
:1041700018742075F8BD90680028E4D0E6E700BF09
:1041800000D0FFFF1B8000402DE9F04F5C4D5D49E2
:104190002B680C688DB000220593059B0A921B1BAF
:1041A0000F2BCDF82B2040F2DE812B680693069B67
:1041B0000B6001238DF828308DF829308DF82A30D6
:1041C000012380F8B0399DF8293013B1012380F81C
:1041D000B1399DF82A3013B1012380F8B239D0F8F3
:1041E000AC3900F6E40203EB830302EBC303029253
:1041F00093F86430012B00F05D81D0F8C0A9BAF1CA
:10420000FF3F044600F05D8100F6AC1900F65C1B30
:104210004FF000474FF0810856465BF8240C0368C6
:1042200000219B6898475BF8200C036800219B687D
:1042300098475BF8283C1A68D762C2F83480D36A82
:10424000002BFCDA5BF8200C936B036800219B6861
:1042500098475BF8283C1A68F6B2D7625663D36A6F
:10426000002BFCDA5BF8200C936B036800219B6841
:1042700098475BF8283C1A688223D7625363D36A55
:10428000002BFCDA5BF8200C936B036800219B6821
:1042900098475BF8283C1A68D7625663D36A002BAC
:1042A000FCDA5BF8200C936B036800219B6898474D
:1042B0005BF8283C1A688323D7625363D36A002BC8
:1042C000FCDA5BF8200C936B036800219B6898472D
:1042D0005BF8283C1A68D7625663D36A002BFCDA75
:1042E0005BF8240C936B036801219B689847D945C0
:1042F00000F0E3800BF1280BD4F8C0698DE700BF14
:1043000074CE0120F817FF1F0023B34684F8C53987
:10431000BBF1000F40F0CE80D4F8AC395A1C022A11
:1043200000F32781A118286891F8B0190790C4F804
:10433000AC29079A31B104EB8301D1F8B819521AAC
:10434000212A16D80233032B08BF0023E21828685D
:1043500092F8B0190790C4F8AC39079A002900F018
:10436000A98004EB8303D3F8B439D21A212A40F28E
:10437000A180DFF8308203944FF0210B4FF0000A48
:10438000844940F6583303FB0A131A4693F8821007
:1043900019B993F88330002B6CD02B6808930899D7
:1043A00092F882307C4F7D4AC1F3012E0BB152F856
:1043B0002E70784C40F6583C0CFB0A4C0BF10A036B
:1043C0009CF883C059465D2202200BF1FF360BF1A9
:1043D0000B09BCF1000F02D0714C54F82E7041F261
:1043E000A5440094FCF734FE01224FF6FF731046FB
:1043F000314600934B46FCF72BFE4FF6FF733146D8
:1044000000935E2233460120FCF722FE5E224FF627
:10441000FF733146104600934B46FCF719FE4FF6EA
:10442000FF73009349464B465E220120FCF710FEC5
:10443000012200236026C0243021C8F82C20C8F8AF
:104440002820C8F80C20C8F8102038460BF10502C7
:1044500088F81430A8F81630C8F81830C8F81C309E
:10446000A8F80830C8F82060C8F8244088E806009A
:10447000FCF75EFE0AF1010ABAF1030F0BF1400BE3
:104480007FF47EAF039C029AD4F8AC3903EB83032C
:1044900002EBC3005030FFF7B7FDD4F8AC392A68FF
:1044A0000992E11804EB8303099A002081F8B0090E
:1044B000C3F8B4290DB0BDE8F08F4FF0FF33C4F856
:1044C000C03994F8C539002B37D094F8C4B904F634
:1044D000AC1704F65C1A4FF000484FF0AF095E4687
:1044E0001AF8133CB34221D05AF8240C03689B6895
:1044F00036B3002198475AF8200C036800219B68C6
:1045000098475AF8283C1A68AE23C2F82C805363A7
:10451000D36A002BFCDA5AF8240C936B0368012150
:104520009B6898470AF8136C94F8C46957450AF1D8
:1045300028033FF4E9AE9A46D2E794F8C4B9E7E617
:10454000314698475AF8200C036831469B689847D3
:104550005AF8283C1A68C2F82C80C2F83490D36A02
:10456000002BFCDAD7E79DF82830002B3FF42BAE68
:1045700026E62B6894F8B0290793C4F8ACB9079BDA
:104580002AB1D4F8B4299B1A212B3FF6F2AE0123AD
:10459000DCE600BF04AA0120703D02004C0AFF1FA8
:1045A0003C0AFF1FD419012010B4036841681A782F
:1045B0000C78417A037A0C4202EA03021BD0837A18
:1045C00003F003030AB143F0040343F008039A1015
:1045D000013B82720D2B0BD8DFE803F021071B078C
:1045E0000A152121150A071B0721C368013BC36077
:1045F0005DF8044B7047837A03F00303002AE6D08A
:1046000043F00403E3E7C3685DF8044B023BC36077
:104610007047C3685DF8044B0233C3607047C368DA
:104620005DF8044B0133C360704700BF08B5034B0E
:10463000D3F8EC00FFF7B8FF08BD00BF40CC012065
:1046400008B5034BD3F8E800FFF7AEFF08BD00BF85
:1046500040CC012008B5034BD3F8E400FFF7A4FFDA
:1046600008BD00BF40CC012008B5034BD3F8E000E3
:10467000FFF79AFF08BD00BF40CC012008B5034BEF
:10468000D3F8DC00FFF790FF08BD00BF40CC01204D
:1046900008B5034BD3F8D800FFF786FF08BD00BF6D
:1046A00040CC012008B5034BD3F8D400FFF77CFFC2
:1046B00008BD00BF40CC012008B5034BD3F8D000A3
:1046C000FFF772FF08BD00BF40CC012008B5034BC7
:1046D000D3F8CC00FFF768FF08BD00BF40CC012035
:1046E00008B5034BD3F8C800FFF75EFF08BD00BF55
:1046F00040CC012008B5034BD3F8C400FFF754FFAA
:1047000008BD00BF40CC012008B5034BD3F8C00062
:10471000FFF74AFF08BD00BF40CC012008B5034B9E
:10472000D3F8BC00FFF740FF08BD00BF40CC01201C
:1047300008B5034BD3F8B800FFF736FF08BD00BF3C
:1047400040CC012008B5034BD3F8B400FFF72CFF91
:1047500008BD00BF40CC012008B5034BD3F8B00022
:10476000FFF722FF08BD00BF40CC012008B5034B76
:10477000D3F8AC00FFF718FF08BD00BF40CC012004
:1047800008B5034BD3F8A800FFF70EFF08BD00BF24
:1047900040CC012008B5034BD3F8A400FFF704FF79
:1047A00008BD00BF40CC012008B5034BD3F8A000E2
:1047B000FFF7FAFE08BD00BF40CC012008B5034B4F
:1047C000D3F89C00FFF7F0FE08BD00BF40CC0120ED
:1047D00008B5034BD3F89800FFF7E6FE08BD00BF0D
:1047E00040CC012008B5034BD3F89400FFF7DCFE62
:1047F00008BD00BF40CC012008B5034BD3F89000A2
:10480000FFF7D2FE08BD00BF40CC012008B5034B26
:10481000D3F88C00FFF7C8FE08BD00BF40CC0120D4
:1048200008B5034BD3F88800FFF7BEFE08BD00BFF4
:1048300040CC012008B5034BD3F88400FFF7B4FE49
:1048400008BD00BF40CC012008B5034BD3F8800061
:10485000FFF7AAFE08BD00BF40CC012008B5024BFF
:10486000D86FFFF7A1FE08BD40CC012008B5024B70
:10487000986FFFF799FE08BD40CC012008B5024BA8
:10488000586FFFF791FE08BD40CC012008B5024BE0
:10489000186FFFF789FE08BD40CC012008B5024B18
:1048A000D86EFFF781FE08BD40CC012008B5024B51
:1048B000986EFFF779FE08BD40CC012008B5024B89
:1048C000586EFFF771FE08BD40CC012008B5024BC1
:1048D000186EFFF769FE08BD40CC012008B5024BF9
:1048E000D86DFFF761FE08BD40CC012008B5024B32
:1048F000986DFFF759FE08BD40CC012008B5024B6A
:10490000586DFFF751FE08BD40CC012008B5024BA1
:10491000186DFFF749FE08BD40CC012008B5024BD9
:10492000D86CFFF741FE08BD40CC012008B5024B12
:10493000986CFFF739FE08BD40CC012008B5024B4A
:10494000586CFFF731FE08BD40CC012008B5024B82
:10495000186CFFF729FE08BD40CC012008B5024BBA
:10496000D86BFFF721FE08BD40CC012008B5024BF3
:10497000986BFFF719FE08BD40CC012008B5024B2B
:10498000586BFFF711FE08BD40CC012008B5024B63
:10499000186BFFF709FE08BD40CC012008B5024B9B
:1049A000D86AFFF701FE08BD40CC012008B5024BD4
:1049B000986AFFF7F9FD08BD40CC012008B5024B0D
:1049C000586AFFF7F1FD08BD40CC012008B5024B45
:1049D000186AFFF7E9FD08BD40CC012008B5024B7D
:1049E000D869FFF7E1FD08BD40CC012008B5024BB6
:1049F0009869FFF7D9FD08BD40CC012008B5024BEE
:104A00005869FFF7D1FD08BD40CC012008B5024B25
:104A10001869FFF7C9FD08BD40CC012008B5024B5D
:104A2000D868FFF7C1FD08BD40CC012008B5024B96
:104A30009868FFF7B9FD08BD40CC012008B5024BCE
:104A40005868FFF7B1FD08BD40CC012001380B4686
:104A50003A2800F25C82DFE810F053024C02450273
:104A60003E0237023002290222021B02AE01A701D8
:104A7000A001990192018B0184017D0176016F01F2
:104A8000680161015A0153014C0145013E013701A2
:104A90003001290122011B0113010B010301FB005D
:104AA000F300EB00E300DB00D300CB00C300BB004E
:104AB000B300AB00A3009B0093008B0083007B003E
:104AC00073006B0063005B0053004B0043003B002E
:104AD000BC4ABD49C2F8EC303B20042217F020B993
:104AE000B84ABA49C2F8E8303A20042217F018B997
:104AF000B44AB749C2F8E4303920042217F010B99B
:104B0000B04AB449C2F8E0303820042217F008B99E
:104B1000AC4AB149C2F8DC303720042217F000B9A2
:104B2000A84AAE49C2F8D8303620042217F0F8B8A7
:104B3000A44AAB49C2F8D4303520042217F0F0B8AB
:104B4000A04AA849C2F8D0303420042217F0E8B8AF
:104B50009C4AA549C2F8CC303320042217F0E0B8B3
:104B6000984AA249C2F8C8303220042217F0D8B8B7
:104B7000944A9F49C2F8C4303120042217F0D0B8BB
:104B8000904A9C49C2F8C0303020042217F0C8B8BF
:104B90008C4A9949C2F8BC302F20042217F0C0B8C3
:104BA000884A9649C2F8B8302E20042217F0B8B8C7
:104BB000844A9349C2F8B4302D20042217F0B0B8CB
:104BC000804A9049C2F8B0302C20042217F0A8B8CF
:104BD0007C4A8D49C2F8AC302B20042217F0A0B8D3
:104BE000784A8A49C2F8A8302A20042217F098B8D7
:104BF000744A8749C2F8A4302920042217F090B8DB
:104C0000704A8449C2F8A0302820042217F088B8DE
:104C10006C4A8149C2F89C302720042217F080B8E2
:104C2000684A7E49C2F898302620042217F078B8E6
:104C3000644A7B49C2F894302520042217F070B8EA
:104C4000604A7849C2F890302420042217F068B8EE
:104C50005C4A7549C2F88C302320042217F060B8F2
:104C6000584A7249C2F888302220042217F058B8F6
:104C7000544A6F49C2F884302120042217F050B8FA
:104C8000504A6C49C2F880302020042217F048B8FE
:104C90004C4A6949D3671F20042217F041B8494A9A
:104CA000664993671E20042217F03AB8454A6449C2
:104CB00053671D20042217F033B8424A6149136735
:104CC0001C20042217F02CB83E4A5F49D3661B20F3
:104CD000042217F025B83B4A5C4993661A20042247
:104CE00017F01EB8374A5A4953661920042217F0A4
:104CF00017B8344A574913661820042217F010B821
:104D0000304A5549D3651720042217F009B82D4AB7
:104D1000524993651620042217F002B8294A5049D7
:104D200053651520042216F0FBBF264A4D49136532
:104D30001420042216F0F4BF224A4B49D3641320F6
:104D4000042216F0EDBF1F4A484993641220042242
:104D500016F0E6BF1B4A464953641120042216F0A0
:104D6000DFBF184A434913641020042216F0D8BF4D
:104D7000144A4149D3630F20042216F0D1BF114ACF
:104D80003E4993630E20042216F0CABF0D4A3C49E7
:104D900053630D20042216F0C3BF0A4A3949136336
:104DA0000C20042216F0BCBF064A3749D3620B2000
:104DB000042216F0B5BF034A344993620A20042244
:104DC00016F0AEBF40CC01202D4600004146000049
:104DD00055460000694600007D46000091460000EF
:104DE000A5460000B9460000CD460000E14600009F
:104DF000F5460000094700001D470000314700004C
:104E000045470000594700006D47000081470000FA
:104E100095470000A9470000BD470000D1470000AA
:104E2000E5470000F94700000D4800002148000058
:104E300035480000494800005D4800006D4800000A
:104E40007D4800008D4800009D480000AD480000EE
:104E5000BD480000CD480000DD480000ED480000DE
:104E6000FD4800000D4900001D4900002D490000CB
:104E70003D4900004D4900005D4900006D490000BA
:104E80007D4900008D4900009D490000AD490000AA
:104E90001F4A204953620920042216F041BF1C4AD0
:104EA0001D4913620820042216F03ABF184A1B4914
:104EB000D3610720042216F033BF154A18499361C5
:104EC0000620042216F02CBF114A16495361052012
:104ED000042216F025BF0E4A13491361042210461E
:104EE00016F01EBF0A4A1149D3600320042216F0AF
:104EF00017BF074A0E4993600220042216F010BF24
:104F0000034A0C4953600120042216F009BF704780
:104F100040CC0120BD490000CD490000DD49000022
:104F2000ED490000FD4900000D4A00001D4A000047
:104F30002D4A00003D4A00002DE9F041437D012B40
:104F40008CB05ED0036EC26D934207D300231C4623
:104F50004A1E9A420AD00CB0BDE8F0815A1C0344A4
:104F600002661C7F4A1E23469A42F4D1437D8DF887
:104F70000840012B00F05781036EC46DA342C0F0BE
:104F80008B8000258DF80950A34280F04A815E1C79
:104F9000034406661D7F33468DF80A50A34280F015
:104FA00039815C1C034404661B7F8DF80B30042997
:104FB0000DF1080E1FD00EEB020100250DF10B02C2
:104FC00002248027012609E00CF1010384440366D2
:104FD0009CF81C3002F8013F91420CD0437D012B1C
:104FE00060D0D0F860C0C36D9C45EDD3002302F8BB
:104FF000013F9142F2D14368704698470CB0BDE83A
:10500000F08100238DF8033004699DF8033042F2EB
:105010001073E27816060AD4013BFAD1A37000BFE0
:10502000036980229A7000BF012303758EE7A3787D
:1050300003F0E703A37003691A79D2B28DF8032055
:105040009A7842F008029A7003690222DA700369C2
:1050500042F21072DC78A50703D4013AFAD19A70B3
:10506000DDE79A7802F0C7029A70026942F2107383
:10507000D478A40640F1D080013BF9D1937000BFF1
:1050800002698024947000BF01240269047502241F
:105090001579D4701C465BE75E1C034406661D7FD1
:1050A00033466FE78DF80750D0F810809DF8073031
:1050B00042F2107398F803C01CF0800F0AD1013B34
:1050C000F8D188F8023000BF03699F7000BF002349
:1050D00006758CE798F8023003F0E70388F8023091
:1050E000036993F804C05FFA8CFC8DF807C093F84D
:1050F00002C04CF0080C83F802C00369DC7003693D
:1051000042F2107C93F8038018F0020F05D1BCF135
:10511000010CF7D183F802C0D5E793F802C00CF078
:10512000C70C83F802C0D0F8108042F2107C98F8C7
:1051300003309B0611D5BCF1010CF8D188F802C0F0
:1051400000BF03699F7000BFD0F8108006756346EA
:1051500098F804C088F803403CE798F8043088F8D1
:10516000034037E7AB7803F0E703AB7003691C79C2
:10517000E4B28DF806409C7844F008049C70036902
:105180000224DC70036942F21074DD78AE0759D452
:10519000013CFAD19C7000BF036980249C7000BF61
:1051A0000123447D03750023012C8DF8093040F064
:1051B000D88000238DF8053005699DF8053042F24E
:1051C0001073EC78270671D4013BFAD1AB7000BFA5
:1051D000036980249C7000BF0123447D0375002374
:1051E000012C8DF80A3040F0BF8000238DF8043088
:1051F00005699DF8043042F21073EC7827063BD421
:10520000013BFAD1AB7000BF036980249C7000BFE2
:10521000012303750023C8E6137902251C46D570C7
:1052200096E60025B8E600238DF8063005699DF85E
:10523000063042F21073EC78270693D4013BFAD182
:10524000AB70A8E79C7804F0C7049C70046942F234
:105250001073E578AD0676D5013BFAD1A37000BF97
:1052600004698025A57000BF012504690575022524
:105270002679E570447D97E7AB7803F0E703AB70E0
:1052800003691C79E4B28DF804409C7844F008046A
:105290009C7003690224DC70036942F21074DD78AB
:1052A000AE071DD4013CFAD19C70ACE7AB7803F09B
:1052B000E703AB7003691C79E4B28DF805409C7874
:1052C00044F008049C7003690224DC70036942F214
:1052D0001074DD78AE071CD4013CFAD19C7076E7DF
:1052E0009C7804F0C7049C70046942F21073E5785E
:1052F000AD0632D5013BFAD1A37000BF0469802509
:10530000A57000BF01250469057502252679E570A1
:105310004BE69C7804F0C7049C70046942F2107359
:10532000E578AD0614D5013BFAD1A37000BF04693E
:105330008025A57000BF0125046905750225267921
:10534000E570447D4CE702252379E570447D2BE729
:1053500002252379E570447D42E702252379E57033
:1053600023E6036EC46D0FE6036EC46D16E600BF40
:1053700008B5044B1B681BB101461846FFF7DCFD5E
:1053800008BD00BF3CCC01204FF47A72704B02FB89
:1053900001F19942F0B400F2AF806E4B994200F2F5
:1053A000AF806D4B994200F2AD806C4B994200F298
:1053B000AE806B4B994200F2AE806A4B994200F28C
:1053C000B080694B994200F2AE80684B994200F27E
:1053D0008A804AF6A833994288BF4FF4807200F25F
:1053E0008380634B4FF400464FF48072994280F003
:1053F0008B8053005F4CB4FBF3F5A94280F08980A9
:105400001344B4FBF3F5A94280F087801344B4FB46
:10541000F3F5A94280F083801344B4FBF3F5A9426D
:1054200080F083801344B4FBF3F5A9427FD2134488
:10543000B4FBF3F5A9427CD21344B4FBF3F5A942C3
:1054400079D21344B4FBF3F5A94276D21344B4FBEA
:10545000F3F4A14273D21344464CB4FBF3F5A942D2
:105460006FD21344B4FBF3F5A9426CD21344B4FBDE
:10547000F3F5A9423ED21344B4FBF3F5A94264D23A
:105480001344B4FBF3F5A94229D21344B4FBF3F45B
:10549000A14228BF102423D2F024374D3549374A82
:1054A0004FF47A7707FB03F3B1FBF3F303602B6848
:1054B00023F008032B60296821F47F2323F47F6302
:1054C00043F46023334323432B6013681B07FCD54D
:1054D000294A136843F008031360F0BC70470F2497
:1054E000013C2401D9E7802253081E02214BB3FB63
:1054F000F2F37BE70D24F3E71E4B0026012275E74C
:105500000222F1E70422EFE713460024C5E7082250
:10551000EAE70224E4E71022E6E70324E0E70424B4
:10552000DEE72022E0E74022DEE70524D8E7062474
:10553000D6E70724D4E70824D2E70924D0E70A24D1
:10554000CEE70B24CCE70C24CAE70E24C8E700BF43
:105550004FA9AB00A7D4550053EA2A0029751500BE
:1055600094BA0A00495D0500A4AE0200515701003B
:1055700095BA0A000095BA0A2C100B4024100B4073
:105580002DE9F0410746884616F0E8FD194C1A4E01
:10559000054604E016F0E2FD401BB04226D8236821
:1055A000DB07F7D4154A164BC2F800801F6016F0CF
:1055B000D5FD144C104D064604E016F0CFFD801BBF
:1055C000A84213D82268104B0E491340002BF4D088
:1055D0000E4B0A681A600A601B680B481840A0F15D
:1055E0000100B0FA80F04009BDE8F0810020BDE87C
:1055F000F08100BF24100B4040420F0008100B4008
:105600000C100B4030100B4001000F0018CC012093
:105610002DE9F04F85B03F4F01900291039216F0B3
:105620009DFDDFF82CA13C4EBB468146DAF8008098
:105630003A4D16F093FD044604E016F08FFD001B72
:10564000A84225D83368D907F7D4354A354BC2F874
:105650000080536016F082FD304C054604E016F0E1
:105660007DFD401BA04213D83A682F4B1340002BFE
:10567000F5D02E4CDBF800302360CBF800302268E8
:10568000294B1340012B03D1294A1268D2050FD4AC
:1056900016F064FD214BC9EB00009842C6D9019871
:1056A0004FF49572292105B0BDE8F04F15F00CBFFD
:1056B000204D21492B701A48029E204A0023236066
:1056C000039B0B6006601E4B1E4E16601E481F4A51
:1056D00088631A6016F042FD104E074604E016F08B
:1056E0003DFDC01BB0420BD82B78002BF7D12268B0
:1056F000154B1340022B03D1012005B0BDE8F08FFC
:1057000001984FF49A72232105B0BDE8F04F15F0CF
:10571000DBBE00BF30100B4024100B4040420F0096
:1057200008100B4000001A0D01000F0018CC0120DA
:1057300010100B4028CC012000100B4004100B402F
:105740000C100B404000010002007F1111003A06CE
:105750001CCC01202DE9F04F93B0804616F0FEFCE2
:10576000A44CA54E054605E016F0F8FC401BB042DF
:1057700000F2DC80236813F00103F5D19F49A04AB1
:105780000B60136016F0EAFC9E4C9B4D064605E04C
:1057900016F0E4FC801BA84200F2C88022689A4BF5
:1057A000984F1340002BF3D0DFF884A23B68CAF86F
:1057B00000303B60DAF80020934B1340012B40F09F
:1057C000B5808C4EBB464FF00A0916F0C7FC8A4DD7
:1057D000044604E016F0C2FC001BA84225D833683A
:1057E000DB07F7D48549894B834C4FF4D5720A60A7
:1057F000834A136016F0B2FC054604E016F0AEFCD6
:10580000401BA04211D83A687F4B1340002BF5D0C3
:10581000DBF80030CAF80030CBF80030DAF80020AE
:10582000794B1340012B00F0DD81B9F10109CCD196
:1058300098F80D20764B002A08BF4FF440130193CF
:1058400016F08CFC6F4F6B4CDFF8B0B10090B9468E
:1058500016F084FC684E054604E016F07FFC401B01
:10586000B04258D8236813F00103F6D1CBF80030CA
:10587000634B684A1A6016F071FC5F4D064604E0FF
:1058800016F06CFC801BA84245D83A685E4B13406A
:10589000002BF5D0D9F80030CAF80030C9F8003034
:1058A000DAF80020584B1340012B34D116F056FC87
:1058B000514E054604E016F051FC401BB0422AD878
:1058C0002368D807F7D4019ACBF800204C4A524BF2
:1058D000136016F043FC484D064604E016F03EFC0B
:1058E000801BA84217D83A68474B1340002BF5D0CD
:1058F000D9F80030CAF80030C9F80030DAF80030C2
:10590000414D1D40012D06D116F028FC009A3A4B5E
:10591000801A984215D940464FF4C472432115F0BD
:10592000D3FD8346584613B0BDE8F08F404640F2A1
:105930007512202115F0C8FD8346584613B0BDE806
:10594000F08F364B1A68002A82DA354A19681160DE
:105950001B68284C284E590044BF324B1D7016F06E
:10596000FDFB054605E016F0F9FB401BB04200F2D6
:105970004381236813F00103F5D12048204A2A49C6
:105980000360116016F0EAFB1E4D1B4C064605E055
:1059900016F0E4FB801BA04200F22E812A681A4B0D
:1059A00018491340002BF3D00B68CAF800300B6085
:1059B000DAF80020144B1340012B40F01D8116F043
:1059C000CDFB0C4C0C4E054605E016F0C7FB401B0A
:1059D000B04200F22181236813F00103F5D107489A
:1059E000074A12490360116016F0B8FB054C024DDE
:1059F000064625E024100B4040420F0008100B40E3
:105A00000C100B4030100B4001000F0000001A0872
:105A10000000304000001A370000022910100B402F
:105A200024CC012020CC01200000090200001A0330
:105A300018CC012016F092FB801BA84200F2EC80EB
:105A400022689E4B9E491340002BF3D00B68CAF886
:105A500000300B60DAF80020984B1340012B40F027
:105A6000DB80984BDFF87C921F68974C974E3F0C79
:105A70003F04C9F8007016F071FB054605E016F00A
:105A80006DFB401BB04200F2CF802368DA07F6D4EA
:105A90008F49904B904A0F601A6016F05FFB884D5B
:105AA0008A4C064605E016F059FB801BA04200F226
:105AB000BB802A68814B824F1340002BF3D03B6898
:105AC000CAF800303B60DAF800207C4B1340012B11
:105AD00040F0AA807B4BDFF830B21C687F4EDBF8C9
:105AE00000509A68316888F82C404FEA142E200C38
:105AF00088F82BE088F828504FEA146E88F82A00BE
:105B00002C0A280C2D0E88F8201088F8242088F8FC
:105B100029E088F827404FEA122E140C88F8260056
:105B2000120E080A88F82550090C002588F8224032
:105B300088F81F0088F81E1088F823E088F82120D4
:105B400088F82D50D9F8001065480093654CFFF790
:105B500017FD002870D0009B1A68634BDBF800101B
:105B60001B68306888F81D50160A150C88F81C2030
:105B700088F81B60120E0E0A88F81A500D0C4FEAB6
:105B8000132E88F8181088F81430090E88F8192098
:105B900088F81760020C1E0C88F816501B0E050AB8
:105BA00088F8100088F8151088F813E088F812605B
:105BB00088F8113088F80F5088F80E2021684B487B
:105BC000FFF7DEFC00283FD021684948FFF7D8FCEA
:105BD000002841D140464FF4D172402115F074FCA9
:105BE0008346AAE6374A1268B2F5D57F0CD188F809
:105BF0000D30404B019323E640464FF4C8722121FB
:105C000015F062FC834698E6404640F27B1225215F
:105C100015F05AFC834690E6404640F2931222214A
:105C200015F052FC834688E640464FF4CC7226219C
:105C300015F04AFC834680E6404640F29B1227213D
:105C400015F042FC834678E640464FF4CF7224219B
:105C500015F03AFC834670E602212748FFF790FCD6
:105C600083460028B6D0254A25481168164C21F0F5
:105C700006011160116841F0020111604FF010122D
:105C8000026016F06BFA8DE80101D9F800800F4E22
:105C900016F064FA054604E016F060FA401BB042C4
:105CA0004FD82368DB07F7D4094A164BC2F80080A7
:105CB000536016F053FA054D06462CE001000F0024
:105CC00030100B4010100B4024100B4040420F00CE
:105CD00008100B400C100B40000009091C100B4071
:105CE0000000090A1CCC012018100B4000001B0703
:105CF00000001A370000304000001A0628100B4040
:105D000044100B4000001A0D14100B4016F026FA38
:105D1000801BA84215D83A68474B1340002BF5D09A
:105D2000464B464A1B68CAF800301360DAF8003068
:105D3000414A43491A40012A03D1424B1B68D80506
:105D400036D416F00BFA009A3F4B801A98429CD931
:105D5000DDF804804FF495722921404615F0B4FB1C
:105D600000284ED146F2A811DFF818A1DFF81891EB
:105D7000364F374E374D384C0022CAF80020404687
:105D8000C9F800203A6032602A602260FFF7FCFA0E
:105D900040F243424FF488600121CAF80020C9F85C
:105DA0000020386032602A60226088F80C10C4E558
:105DB0002A4C2B4E22702B4DDDF804802A480022FD
:105DC00002AB0A6033602949294A6FF07F462E6092
:105DD000284D0D60284D29490560116016F0BEF967
:105DE000194D064604E016F0B9F9801BA8421CD8EC
:105DF0002378002BF7D1DAF800101F4A0A40022A54
:105E000013D19DF815209307ACD502AA1C49404632
:105E1000FFF7FEFB0028A5D09DF8182002F00F0226
:105E2000012A9FD14CF250319EE74FF49A72232100
:105E3000404615F049FB93E701000F0030100B407E
:105E400018CC012010100B4040420F0008D0044035
:105E50000CD0044010D0044014D0044028CC0120C1
:105E600000100B4008100B4038100B4004100B4082
:105E70000C100B404000010002007F1111003A0697
:105E8000F1FFFF8000D0044004D0044030B40F4C38
:105E9000029D04FB00F0063041F2717404FB010125
:105EA0000B4C002AB4BF02F1FF001046144001EB76
:105EB0002021002C196002DB2C6030BC7047013CB3
:105EC00064F0FF0401342C6030BC704728280900BE
:105ED000FF000080F8B5214CD0F880722478D0F80B
:105EE00084620137002C07F01F0714BF4FF0010E2A
:105EF0004FF0030EB7422DD00C46D0F88012184E4A
:105F000001EB8101890015460122425401448B6056
:105F1000069B4D60CB6081F810E0C0F8807216F0EF
:105F20001DF90746D4F88020D4F884309A420CD06A
:105F3000D4F88420D4F8843054F82220013303F0BC
:105F40001F039542C4F8843006D016F007F9C01B31
:105F5000B042E7D90020F8BD0120F8BD3ACC0120BD
:105F60009F860100F8B5214CD0F880722478D0F8D3
:105F700084620137002C07F01F0714BF4FF0010E99
:105F80004FF0030EB7422DD00C46D0F88012184EB9
:105F900001EB8101890015460022425401448B60C7
:105FA000069B4D60CB6081F810E0C0F8807216F05F
:105FB000D5F80746D4F88020D4F884309A420CD023
:105FC000D4F88420D4F8843054F82220013303F02C
:105FD0001F039542C4F8843006D016F0BFF8C01BEA
:105FE000B042E7D90020F8BD0120F8BD3ACC01202D
:105FF0009F8601002DE9F04FB54E3568A5B015F02C
:106000000105DDF8BC80DDF8C0B0059207460C46FE
:106010009A4600F0D781AF4D296811F0010600F0D3
:10602000BC81AD4DAD48AE4E4FF40062002118F07A
:106030007BFB4FF400620021284618F075FB06FB3D
:106040000AFA4FF400720021A6484FF0040918F034
:106050006BFB0AF10102CDF80090A04B21463846B7
:10606000FFF780FF002800F0D680059B434409938A
:10607000197C002940F0D38040F24462284618F091
:1060800053FB6422FF2105F5C87018F04DFB06FB99
:1060900008F307932E9B914ADFF858927C330893BC
:1060A00002EB830341F271725E68002E3346B8BF83
:1060B00006F1FF031B1203F1020890452E9A0AF124
:1060C000050A88BF03F1010841F2717303FB02A3C3
:1060D00003934A464FF0000A09E0D1F8F431002B4F
:1060E0000BDD0AF1010ABAF1630F00F0808112F8AA
:1060F000013F632B05EB8301EFD9002164220BA83C
:1061000018F012FB7849012019F8013F632B05EBC9
:10611000830207D8D2F8F421002A03DD24AA13440D
:1061200003F8640C4945EFD10DF12B02002303E085
:106130000133642B00F05B8112F8011F0029F7D1B5
:10614000D5F840260693511C08BF911CAA4441F281
:10615000717245F823108AF89031C5F8401602FB99
:1061600003F2079B053313440493B8F1000F00F0CA
:10617000D38008EB03025D4E029299465C4BD7F840
:1061800080221878D7F884120132002802F01F020A
:106190000CBF4FF0030C4FF0010C8A423BD0039B25
:1061A000D7F880029E46049B00EB800007EB80013D
:1061B000C3EB0E084FF0000E07F820E0494B8B6050
:1061C0000120C84481F80DE081F80EE081F80FE06D
:1061D00081F810C00873C1F80480C7F8802215F058
:1061E000BDFF8246D4F88020D4F884309A420CD087
:1061F000D4F88420D4F8843054F82220013303F0FA
:106200001F039045C4F8843018D015F0A7FFCAEBDF
:106210000000B042E6D9002025B0BDE8F08F06FBB3
:1062200008F307935A1CCDF800902B4621463846B8
:10623000FFF798FE00287FF42DAFECE72C4BD7F842
:1062400080221878D7F884120132002802F01F0249
:106250000CBF4FF003084FF001088A42DBD0D7F89B
:106260008002204B00EB800007EB80014FF0000E16
:106270004FF0010C07F820C081F81080C1F804909D
:106280008B6081F80CC081F80DE081F80EE081F898
:106290000FE0C7F8802215F061FF8046D4F8802017
:1062A000D4F884309A420CD0D4F88420D4F88430C6
:1062B00054F82220013303F01F034A45C4F8843008
:1062C0001AD015F04BFFC8EB0000B042E6D9A2E7A8
:1062D000CC0F0120B00F0120B0FF0020B00701203B
:1062E00028280900D00F0120A30101209F8601006A
:1062F0003ACC01203F010120DBF80020584612680B
:106300009047029B09F101094B457FF437AF3A4BA7
:10631000089A03EB82035E68374A2E99374B02EBEB
:10632000410E069A05EB42017046BEF884E3A1F8DF
:1063300084E30699B0F84CA42F48079A05EB41096D
:106340002E99A9F84CA400EB410C00EB010E069924
:10635000BCF814859EF8DCC505EB010E05EB810544
:106360000421009101322146A9F8148538468EF89F
:10637000DCC5C5F8F461FFF7ADFD00283FF44BAF75
:10638000099E059B327C01252A44327421463846F9
:1063900000950022FFF79EFD3EE7284615F07EFCA3
:1063A00000283FF43EAE314640F24462134818F0F4
:1063B000BBF96422FF21124818F0B6F9284615F0FF
:1063C00073FC2EE6304615F069FC00283FF423AE3E
:1063D000294640F24462084818F0A6F96422FF21D9
:1063E000084818F0A1F9304615F05EFC13E64FF0AE
:1063F000FF33054A0693B4E6B0070120B0FF002042
:1064000040010120400901208FE8FFFF2DE9F04FF6
:10641000DBB0649C659D0595669D0A95029003918D
:106420002046002115464FF400720994689EDDF85D
:10643000A491DDF8A8811C4618F076F94FF40062AB
:106440000021A54818F070F94FF480620021A3489C
:1064500018F06AF927A8CC22002118F065F9012369
:106460005893002C00F0F68004F28F173B4604F599
:10647000F97006E0D1F8F421002A08DD984200F016
:10648000E98013F8012F632A04EB8201F2D90DF1A0
:10649000380A00215046642218F046F904F2F3113C
:1064A000012017F8013F632B04EB830205D8D2F8D3
:1064B000F421002AC8BF0AF80300B942F1D10DF156
:1064C0003702002303E00133642B00F0C38012F88D
:1064D000011F0029F7D141F27177DAB207FB03F708
:1064E00008920793C6EB0903002B06937BDD7C4BD8
:1064F000059A0399029803FB05F303F105090B9331
:1065000041F2717303FB0293002E324603F1010343
:10651000B8BF06F1FF0203EB22231A4604930123BE
:1065200000936D4BFFF71EFD00285CD06D4D35408C
:10653000002DC0F23E8109EB07034FF0000A0D93D6
:1065400001330C94D1462C465746069E9B46554631
:106550002AE038460137604B33F914105AAB2B440C
:1065600081EAE17213F8CCCCA2EBE172C2F3C71E50
:10657000F44538BF03F8CCEC599B013B002B04F1E8
:106580000104599333DDD8F800E0544B9145B8BF6E
:10659000914623F81010013EDEF800304046CA460E
:1065A0000FFA89F9984796B1B4F5807F2CD0FF2F68
:1065B000CFDD012300935A46484B03990298FFF719
:1065C00089FC80B10BF1010B01270020C3E70123F7
:1065D0005A4600930399414B02980C9CD346FFF70F
:1065E00079FC00283BD100205BB0BDE8F08F01357D
:1065F000C02D579517D0589B59935AAB2B444FF049
:10660000000E03F8CCECBEE7049B0399029801331B
:106610000122049300921A462F4BFFF7A3FC002897
:10662000E1D00024C3E70DF19D0E0DF19B0C0DF29E
:106630005D1A1EF8015C1EF8023BAB42B8BF2B4648
:10664000F2450CF8013FF4D1589B60255B0058934C
:106650005795D1E7FF2307930893234F42E7C02DB7
:1066600000F0AF805F2D40F3BE80602D48D007EE74
:10667000905ADFED1E6A9FED1E7AF8EEE77A3246F9
:1066800067EEA67A27A914E0BF28A8BFBF20BF2BBA
:10669000A8BFBF235AAD28442B4410F8CC0C13F8E4
:1066A000CC3C8342B8BF03460136602E26D001F8A9
:1066B000013B37EE277A1346FDEEC76A501C16EEF3
:1066C000902AD51A012DDFDCBF2BA8BFBF235AA803
:1066D000034413F8CC3CE7E7D01101206018FF1FFA
:1066E00028280900FF0000808F591700ABAA2A3C18
:1066F0000000000000007A446F1203388DF8FB3070
:10670000099E304627A960223430012515F0E6F9AC
:1067100033460D9A009503990298FFF7DBFB00289A
:106720003FF461AFDDED067A5FED0E6A059F0A9AD0
:1067300054F82730B8EEE77A5FED117A67EE277AE2
:10674000002067EEA67A44F8270004EB8706FCEEEB
:10675000E77A079FCDED047A224444F8273004EB12
:10676000870104EB47039DF8207082F890714FF089
:10677000FF37BDF81020C6F8F471069EC1F8F46129
:10678000A3F88403D2B1A3F84C24079A0399029882
:10679000A3F814B5224416460B9A00270425234675
:1067A000013286F8DC7564955BB0BDE8F04FFFF709
:1067B00091BB013D65F0FF050135BCE6A3F84C54E3
:1067C000E3E70DF19D010DF19B000DF25D1511F850
:1067D000012C11F8023B9342B8BF13468D4200F8DA
:1067E000013FF4D18CE73146C02227A817F09CFF67
:1067F00086E700BF2DE9F04F83B001EB8101434BE9
:10680000434A01920DF10809804649000B4459F8AA
:10681000040D404FC8F8843008F58E56C8F888003B
:10682000183608F1880A08F18C052C4657F8D43C34
:1068300044F8043B05F2C455BB465946224651F87C
:10684000040B42F8040BB8341046B42215F046F994
:10685000AC420BF5807BF0D1A64207F65837E4D165
:10686000B6EB0A0650D00022114608F1870010F856
:10687000013F01F00F0401311A448E4203FA04F380
:1068800082EA0302F3D1224B1344019341F2D8135D
:10689000D9F8000048F80300D8F878401E4AD4F828
:1068A00080321278D4F884021C49D8F8845001331D
:1068B000002A41F29B6E03F01F0342F2F3164FF0E1
:1068C00000020CBF03270127834201F80E2081F844
:1068D000432B8A5512D0D4F8800200EB8000800050
:1068E0002118012626540A204D60C1F808A04A73D9
:1068F0008A73CA730F740873C4F88032022388F84D
:10690000083003B0BDE8F08F014BBEE779878A03FA
:10691000FF16FE12DCAA01203ACC012004AA0120B5
:10692000F8B54D4B1B682BB193F88010C27811B9A4
:10693000162A3BD0F8BD93F8811011B9162A39D028
:10694000F8BD013A0179162AF4D801A050F822F0D6
:10695000EF690000E1690000356900003569000059
:1069600035690000356900003569000035690000AF
:10697000356900003569000035690000356900009F
:10698000356900003569000035690000356900008F
:10699000356900003569000035690000356900007F
:1069A00035690000B5690000CF69000093F88110D7
:1069B0000029C6D1294941F29A6441F29960012225
:1069C0000A550A5483F8802083F88120F8BD2348B3
:1069D00041F2996100240122445483F88120F8BDDA
:1069E0001A7A002AA6D11846FFF704FFF8BD1A7AD2
:1069F000002A9FD19E6F1A4CD6F8800294F800E0CE
:106A0000184DD6F884420130BEF1000F4FF00A074E
:106A100000F01F0017FB015114BF4FF0010E4FF0A3
:106A2000030EA042C3F8841003F1880C11D0D6F8ED
:106A3000805205EB8505AD00741972556160C4F88C
:106A400008C027736273A273E27384F810E0C6F87B
:106A5000800201221A72F8BD601CFF1F04AA0120E7
:106A60003ACC012079878A0370B40668B26883B093
:106A700042F21074D3789B060DD5013CFAD1947084
:106A800000BFB36880229A7000BF012333730020D7
:106A900003B070BC7047B02403799470B268D578A5
:106AA000AD0642F2107404D4013CE8D0D578AD06AE
:106AB000FAD5D478A506EAD5947844F030049470D9
:106AC000B46842F21075E278920603D4013DFAD11F
:106AD000A570D5E75B00DBB22371B26842F2107398
:106AE000D478A40703D4013BFAD19370C8E70568B2
:106AF000AC6842F21073E27816060AD4013BFAD170
:106B0000A37000BFAB6880229A7000BF01232B7373
:106B1000BDE70223E370AA68937843F010039370F3
:106B2000AB680A0A1A71AA6842F21073D478A407F3
:106B300003D4013BFAD19370E3E7D3780224DBB2AC
:106B4000D47013F0100240F01A81DE0700F1C78004
:106B5000AB68DC700568AC68E278120642F210732C
:106B600004D4013BCCD0E2781206FAD50223E370BC
:106B7000AA68937843F010039370AB68C9B2197197
:106B8000AA68D1788E0742F2107304D4013BD2D0A8
:106B9000D1788E07FAD5D3780221DBB2D17013F009
:106BA000100240F0F580DC0700F1A880AB68D970D6
:106BB0000468A268937803F0C7039370A16842F257
:106BC0001072CB789B060AD5013AFAD18A7000BFC1
:106BD000A36880229A7000BF0123237357E70368DC
:106BE0009A6842F21071D478A60603D50139FAD119
:106BF00091702CE0B024017994709A6842F210747C
:106C0000D578AD0603D4013CFAD194701FE0D47856
:106C1000A4067FF53CAF947844F0300494709C68EF
:106C200042F21075E278960603D4013DFAD1A570C0
:106C30000DE04A0042F00102D2B22271996842F29C
:106C40001072CC78A4070AD4013AFAD18A7000BF36
:106C50009A688021917000BF01221A7317E70268B9
:106C600000238DF8053094689DF8053042F21073CA
:106C7000E17809060AD4013BFAD1A37000BF9368FA
:106C80008021997000BF0123137300E7A37803F0FC
:106C9000E703A37091680B790224DBB28DF805300D
:106CA000CC70936842F21071DC78A60714D51C7979
:106CB00099788DF8064041F0080199709368022197
:106CC000D970936842F21074D9788D071DD4013CB5
:106CD000FAD100219970D1E70139E5D1F9E7AB6824
:106CE0000121D97000BFAB682C739A7000BFAB68EC
:106CF00080229A70AB680222DA70C8E6AB68012085
:106D0000D87000BFAB682973EFE7997801F0C7012D
:106D10009970936842F21071DC78A4060ED501399F
:106D2000FAD1997000BF93688021997000BF01214A
:106D30009368117302221979DA70A8E602211A7990
:106D4000D97000688DF807208268937803F0C70334
:106D50009370816842F21072CB789E060AD5013A90
:106D6000FAD18A7000BF836880229A7000BF012325
:106D700003738CE6BDF8060003B070BC7047AB68C7
:106D80001022DA7000BF0321AB6829730022ACE740
:106D9000AB681022DA7000BF0321AB6829730022B0
:106DA000A3E700BFF0B40768BC6842F21075E3784F
:106DB0009B060CD5013DFAD1A57000BFBB688022AF
:106DC0009A7000BF01233B730020F0BC7047B025D0
:106DD0000379A570BC68E678B60642F2107504D453
:106DE000013DE9D0E678B606FAD5E578AD06EBD5F3
:106DF000A57845F03005A570BD6842F21076EC78B4
:106E0000A40603D4013EFAD1AE70D6E75B00DBB234
:106E10002B71BC6842F21073E578AD0703D4013BD7
:106E2000FAD1A370C9E70668B56842F21073EC782E
:106E300027060AD4013BFAD1AB7000BFB3688022A9
:106E40009A7000BF01233373BEE70223EB70B4686E
:106E5000A37843F01003A370B3680C0A1C71B468E4
:106E600042F21073E578AD0703D4013BFAD1A37069
:106E7000E3E7E3780225DBB2E57013F0100440F09D
:106E8000D480DB0700F1A680B368DD700668B568C2
:106E9000EC78270642F2107304D4013BCCD0EC7896
:106EA0002706FAD50223EB70B468A37843F01003E9
:106EB000A370B368C9B21971B16842F21073CC788B
:106EC000A40703D4013BFAD18B70B6E7CB78022438
:106ED000DBB2CC7013F0100140F0A780DF0700F1A7
:106EE0008980B368DC700568AC6842F21073E178A1
:106EF0000E060AD4013BFAD1A37000BFAB68802212
:106F00009A7000BF01232B735EE70223E370A96828
:106F10008B7843F010038B70AB68110A1971A96864
:106F200042F21073CC78A40703D4013BFAD18B70E2
:106F3000E3E7CB780224DBB2CC7013F0100140F011
:106F40008280DF0762D4AB68DC700568AC68E178EA
:106F50000E0642F2107304D4013BCDD0E1780E0648
:106F6000FAD50223E370A9688B7843F010038B7085
:106F7000AB68D2B21A71AA6842F21073D17889074D
:106F800003D4013BFAD19370B7E7D3780221DBB287
:106F9000D17013F0100256D1DF0762D4AB68D970FC
:106FA00001688A68937803F0C70393708A6842F295
:106FB0001070D3789E060AD50138FAD1907000BFC0
:106FC0008B6880229A7000BF01230B73FDE60120BD
:106FD000F0BC7047B3680122DA7000BFB368357344
:106FE0009C7000BFB36880229A70B3680222DA7086
:106FF0000020EAE6B3680122DA7000BFB368347398
:10700000997000BFB36880229A70EEE7AB680122E6
:10701000DA7000BFAB682C73997000BFAB68802238
:107020009A70AB680222DA70CEE6B3681022DA708A
:1070300000BFB3680321002231739A7000BFB368A8
:1070400080229A70D1E7AB681022DA7000BFAB687B
:107050000321002229739A7000BFAB6880229A70C6
:10706000DFE7AB680120D87000BFAB68F2E700BF74
:10707000F0B40023002744F2900644F2940544F251
:10708000980400F58142876003604360C360036138
:1070900043610376C3610362436201274FF0FF330C
:1070A0004FF07E518762835143510351D161F0BC4F
:1070B000704700BF2DE9F843037B052B01D0BDE8E5
:1070C000F88348F6887244F2A00382587D4C03FB93
:1070D00002F3C11844F6FC5244F6F8558A584A5156
:1070E000466894F80080D6F88012D6F8844202EB05
:1070F000420203EB82030131B8F1000F00EB0302FF
:1071000001F01F0144F69C530CBF03250125A14249
:10711000D75818D0D6F8803203EB83039B0044F68F
:10712000985E012452F80EE0F45433440022042403
:107130005F60C3F808E01D741C735A739A73DA73A6
:10714000C6F88012466800F50E44A834D4F8C03062
:1071500048F67472C02B0546875800F099805F2B63
:1071600040F3AA80602B31D007EE903ADFED566AEB
:10717000B8EEE77A0021DFED557A27EE267A084649
:10718000A6460FE0BF2AA8BFBF22BF2BA8BFBF23C0
:10719000A25CE35C9342B8BF13460131602913D06F
:1071A0000EF8013B77EE877A0346FDEEE76A421C54
:1071B00016EE900AC3EB000CBCF1010FE2DCBF2B12
:1071C000A8BFBF23E35CE8E784F85F3048F6787334
:1071D000DFED3F7AEA58DFED3F6AA2F5007207EE75
:1071E000102AB8EE477A05EB870067EE277AEA5057
:1071F00067EEA67A05EB4701FCEEE77AC0F80C22B1
:1072000017EE903A4FF0000948F67E72A1F8643408
:10721000A1F89C932F44AB5AA1F82C35602287F833
:10722000F495214605F6843014F058FCD6F88032E7
:10723000D6F884220133C84503F01F030CBF03278F
:107240000127934218D0D6F88012D5F854ED01EBFF
:10725000810189007218012405F535607454C2F863
:1072600004E0147382F80D9082F80E9082F80F906B
:1072700017749060C6F88032D5F81C38013304BF0B
:107280004FF47A53C5F81C3803232B73BDE8F883F9
:1072900000F50E4100F50F4EA7310EF1070E234603
:1072A00018785A788242B8BF024601F8012F8E45FD
:1072B00003F10203F4D189E7C0220021204617F030
:1072C00033FA83E73ACC0120ABAA2A3C0000000045
:1072D0006F12033800007A44F8B590F87069002303
:1072E00001228E4280F8642080F8713980F8633082
:1072F00080F85C3080F8803000F0A9804A1E012AB6
:107300000D46044616D94FF0FF32C0F88C20C0F865
:107310009020C0F89420C0F89820C0F89C2080F8F5
:107320007E3080F87F30C0F8A03019463422A43077
:1073300017F0FAF90EB1002D4CD12046FBF7C2F838
:1073400004F5186004F6841100224FF0FF3704F6AC
:107350008813C4F8987904F68C1602600A6004F564
:10736000196004F694111A600023326002600A600A
:10737000C4F8647984F89031C4F89431C4F8983131
:1073800084F89032C4F89432C4F8983284F8903378
:10739000C4F89433C4F8983384F89034C4F894341F
:1073A000C4F8983484F89035C4F89435C4F8983506
:1073B00084F89036C4F89436C4F8983684F8903738
:1073C000C4F89437C4F8983784F89038C4F89438DF
:1073D000C4F89838A3691B02E21892F8EB1004294C
:1073E00036D094F860307BB3012D2DD02C4A2D4B34
:1073F00010792D49226818700B682C4E48F6907051
:1074000000FB026023F0004306F5F1320B6000F54B
:1074100047504FF0FF33C2F8B4303030FFF74AFE28
:10742000D4F8487BD4F84C0BD4F8501B002301222D
:1074300084F8603087F87C3080F87C3081F87C30CC
:1074400086F8C43986F8C52984F87059F8BDF8BDA6
:10745000D4F8D80A92F8E910014491F89011632900
:1074600014D800EB8106D6F8F461002E0EDDD2F8B8
:10747000EC605EB1014491F8DC3503F0020303F0E7
:10748000FF01002BADD182F8EB10AAE723440022C4
:1074900083F8EB2094F86030002BD5D0A4E700BF30
:1074A0002CCC01201A80004080F00240A81CFF1F55
:1074B0002DE9F04700F5EC356B6E013B002B6B6658
:1074C00001DDBDE8F087EE6DC84F48F6907404FB0F
:1074D00006F403194BF2207244F2A0019A58B7F94E
:1074E00000E001FB02F21119014447F2945C4BF2F7
:1074F000147851F80CC001F554510CEB4C0CD1ED43
:10750000027A04EB8C042244024447F23054FDEE2C
:10751000E77A125917EE901A22F811E04BF2167C16
:1075200033F808A033F80C104BF210798EEAEE72A3
:10753000A2EBEE7253F809409245D646B8BF964684
:107540009142B8BF1146013443F8094023F808E0DE
:1075500023F80C1003F537414BF2406409680B44E3
:10756000C2F3C71213F804E0964538BF1A5548F61F
:10757000907202FB06F200EB020804464BF2087020
:1075800058F80030013B002B48F8003040F39C8154
:1075900048F6907303FB06F3E1184BF22072F7EE06
:1075A000006A8A5844F2A00101FB0233234403F528
:1075B000545292ED027A37EE267A43F2045082ED6D
:1075C000027A1A5807EE902AF8EEE77A43F2285228
:1075D00077EEA67A9958FDEEE77A17EE902A07EE35
:1075E000901A1A5003F55453F8EEE77A93ED077AA0
:1075F00067EE877AF5EEC07AF1EE10FAC0F20E82ED
:107600007B4B9A42B4BF00220122002A40F0FC8149
:1076100048F6907303FB06F2A0184BF2207144F277
:10762000A003415803FB0123234443F2285003F5F0
:107630005452185892ED077A07EE900AF8EEE77A5E
:1076400003F5545367EE877A0833F5EEC07AF1EE0E
:1076500010FA93ED007AC0F2E781DFED667AB4EEBE
:10766000E77AF1EE10FACCBF01230023002B40F0A3
:10767000468148F6907303FB064642F2A073F35826
:10768000D3F88010D3F88420914208D0D3F8842016
:10769000D3F88420013202F01F02C3F884203B8813
:1076A00095F8602083F40043591241F08006C3F33B
:1076B00086081AB1E96D002900F0A080216A886867
:1076C0004F6887421AD9E769D1F800E047F00047D0
:1076D00000F1010CC1F808C04EF82070216AE7697A
:1076E00088684B68834209D9D1F800E047F0C007A9
:1076F00000F1010CC1F808C04EF82070002A40F0DB
:107700009E80E16A88684F6887421AD9A76AD1F8D3
:1077100000E047F0004700F1010CC1F808C04EF846
:107720002070E16AA76A88684B68834209D9D1F85A
:1077300000E047F0C00700F1010CC1F808C04EF8A6
:107740002070002A40F09E80A36B9A6859688A4294
:1077500014D2616B186841F00041551C9D6040F8DF
:107760002210A36B616B9A685868824206D218682F
:1077700041F0C001551C9D6040F82210E26B236E61
:10778000D168D4F85CE00868022500266666C571F9
:107790000F68C0F800E004248480BC600C68AB4033
:1077A000C3F38F00E08309685B42E360C882D0685E
:1077B0001368016834338D71B3F1804F0B618E8291
:1077C000036801D3996811B9042199600368D068EE
:1077D000094900249C6103790B7011680B6B01202F
:1077E00043F040730B631074BDE8F08738CC012080
:1077F00000E02E0000C07F441B800040216A8868A2
:107800004F6887421BD9E769D1F800E047F000478D
:1078100047EA080700F1010CC1F808C04EF82070D3
:10782000216AE76988684B68834208D9D1F800E08B
:10783000374300F1010CC1F808C04EF82070E96D23
:1078400001297FF45EAFE26A91685068884219D9D5
:10785000A06A176840F0004040EA080001F1010EFC
:10786000C2F808E047F82100E26AA06A9168576808
:107870008F4207D91768304301F1010EC2F808E0C2
:1078800047F82100EA6D022A7FF45EAFA26B91688F
:1078900050688142BFF472AF606B156840F00040E1
:1078A00048EA0003481C906045F82130A36B616BE7
:1078B0009A6858688242BFF461AF18683143551C1A
:1078C0009D6040F8221059E7013108F53749C02979
:1078D000C9F8001000F0B18048F6907303FB06432E
:1078E0004BF204714BF208725958995003F5374224
:1078F0004BF240611268134400225A5448E644F2A5
:10790000A00348F6907203FB01F302FB06F29818FD
:10791000204447F2945147F2905E415840F80E10CF
:1079200004EB020E42F29C70DFF840C15EF800E00A
:107930009CF80080DEF88002DEF884C201EB410191
:1079400002EB810213440130B8F1000F234447F2E7
:10795000345200F01F000CBF4FF003084FF0010835
:10796000604553F802901BD0DEF8801247F2305C7D
:1079700001EB8101890053F80CC00EEB01020123D9
:107980000EF8013000230421C2F80490C2F808C0A8
:1079900082F81080117353739373D373CEF88002FF
:1079A00048F6907E0EFB06FE04EB0E014BF22073B0
:1079B00044F2A002CB5802FB03F202EB0E03E018E4
:1079C00047F2945C47F2345150F80C3003F101084F
:1079D00003EB43030EEB830308F00708134423442F
:1079E00008EB48090EEB890E724453F8019040F8F9
:1079F0000C8000F5545322444FF0000A09F10400B2
:107A0000C3F808A0505034E648F6907000FB0640DA
:107A100000F51E501830FFF74DFBF9E521DA002A7A
:107A2000CCBF00220122F0E518DAB5EEC07AF1EE03
:107A300010FA4CBF0123002318E602F5364040300F
:107A40002044F9F7ADFA4BF20472602158F8023085
:107A50005B0048F80230C9F800103DE7DFED027A1C
:107A6000FDE50023CDE500BF000000003ACC012079
:107A700030B4D0F82458002D15DBD0F8584D6307EA
:107A800013D4214BC0F8501D03FB05F3053341F21D
:107A9000717544F0090405FB0131C0F8584DC0F878
:107AA0005C2DC0F8541D30BC7047D0F8503D8B425F
:107AB000E7D1C11800EB430391F8F415B3F82C3566
:107AC000C90718D4B7EE007A511E00F6833200F6CB
:107AD000E33012F8013F07EE903AF8EEE77A82427F
:107AE00067EE877AFCEEE77A17EE903A01F8013FED
:107AF000EFD130BC704707EE903ADFED046AF8EE44
:107B0000677A86EEA77ADFE72828090000FEFF469D
:107B100070B4D0F82458002D15DBD0F8584D630709
:107B200013D4174BC0F8501D03FB05F3053341F286
:107B3000717544F0110405FB0131C0F8584DC0F8CF
:107B4000602DC0F8541D70BC7047D0F8503D8B427A
:107B5000E7D1FF2380F8823B00F5356300F53860FC
:107B60001D685C689968DE68D660103383421560D2
:107B70005460916002F11002F2D11B681360E2E7D9
:107B800028280900012970B5044634D000F16C059D
:107B9000242128461646FEF767FF4FF6FB72024087
:107BA0002421284604F5EC34FFF7FCF8002384F880
:107BB0006030032E09D8DFE806F0091017022846C6
:107BC00040F273122A21FFF7EDF870BD28464FF4FA
:107BD000B8722A21FFF7E6F870BD284640F271120C
:107BE0002A21FFF7DFF870BD28464FF4B9722A2129
:107BF000FFF7D8F870BD00F16C060D463046242121
:107C0000FEF732FF04F5EC3440F0040292B2304645
:107C10002421FFF7C7F884F8605070BD30B4144CCD
:107C200048F690734FF0FF3203FB004343F2FC151C
:107C30000A604A608A605A5D042A14D048F690733C
:107C400003FB004043F2FC13C35C052B09D14CF24B
:107C500068124CF26C1382580A60C25A4A600022C1
:107C6000C25230BC70474CF27C129B588B60E5E7E7
:107C7000A81CFF1F2DE9F04FDFF82CA32DED048B7E
:107C800040F6583404FB01A48946D4F8543B5B7891
:107C900003F0010383F001010170B5B0D4F8D02ADC
:107CA00003904FEA891B002A78D0B94DDFF8F4829F
:107CB0002B681D931D9A2B681C931C9B29681B9194
:107CC0001B9928681A901A982E681996199F2E6881
:107CD0001896189E5208400850325030D2B2643183
:107CE000C0B26436C1F38401C0F58070C6F3840667
:107CF000C2F58072C3F3C503C7F3C507D20841EAD2
:107D00004313C10846EA471040EAC12143EAC223AF
:107D1000C3F307228BB242EA03239BB200935F2294
:107D20000BF13F0359460020F9F792F92B6817939E
:107D3000179BD4F8D00AC3F30803FF2B0BF1020101
:107D40004FF0000341F2FD424FF001064FF0600595
:107D50004FF0C00488BF0022C8F80410C8F80C30E7
:107D60000221C8F81030C8F82C60C8F82050C8F8B4
:107D70002440A8F8082088F81430A8F81630C8F86D
:107D80001830C8F81C30C8F82810C8F80010F9F7E7
:107D9000CFF935B0BDEC048BBDE8F08F41F22C6219
:107DA000DAF8D45A5AF80220002A00F0FF8042F292
:107DB00084135AF80350002D08BF154641F29C6108
:107DC00042F2F414022041F2A54300935F224AF8E4
:107DD00001000BF13F035946CAF8440B4AF804006E
:107DE0000020F9F735F96B49284616F033FF854234
:107DF00000F0A780664E6849284616F02BFF3368CE
:107E00001E931E9BC3F30803B3F5807F00F2A3808B
:107E1000A84240F0A08061492B4601F1630400258F
:107E200001274FF0200E07E00A2A17D0022FD8BFF3
:107E300081F800E0A14213D01A7801F8012F18460A
:107E400001336AB100782E28EED118782E28EBD1B4
:107E500058782E2808BF0D460A2AE7D10137E9E7EE
:107E600045B133682193219BC3F3C113032B1CBF7E
:107E70002022EA544A49DFF82C810A786020012345
:107E8000C0250624C8F820000020C8F82450C8F8EF
:107E90002840C8F82C30C8F80C30C8F8103088F8E2
:107EA0001400A8F81600C8F81800C8F81C00A8F8B4
:107EB0000800C2BB04246FF003050BF120073D440A
:107EC0003C4441F2A542E31C691C009205205A2261
:107ED000F9F7BEF80434002604222346294610464A
:107EE0000096F9F7B5F82B46294600965B22042048
:107EF000F9F7AEF85B222946234610460096F9F7BB
:107F0000A7F8234621465B2200960420F9F7A0F843
:107F10003023234888E88800F9F70AF935B0BDEC2A
:107F2000048BBDE8F08F0A2A08BF013311F8012F36
:107F3000002AF8D1C3EBC3035C0065106D426410E6
:107F4000BBE7134E33681E931E9BC3F30803B3F5C0
:107F5000807F7FF660AF114A2B4602F16304002553
:107F600002E094423FF47CAF197802F8011F1846F2
:107F7000013300293FF474AF01782E29F1D119782B
:107F80002E29EED159782E2908BF1546E9E700BF02
:107F900074CE01209C3D0200AC3D0200FB17FF1F88
:107FA000FC17FF1FD419012004AA012042F28412F9
:107FB0005AF80220002A41F07382002D7FF4FEAEB1
:107FC000D4F8D80A002800F01B83D4F8B46A1EB392
:107FD0000BF13F03594628465F22F8F7E9FE8D4B27
:107FE000D4F8B40A1D750BF120024FF6FF7E60270E
:107FF000C02602245A6030210122DD829D61DD61AC
:10800000A3F808E01F625E629C621960DA62DA60BF
:108010001A61F9F78DF8BCE694F87D20002A00F08B
:10802000C080B9F1010F41F3DD80002B41F2A5457D
:108030000CBF2B460023009359460BF10803304632
:108040005F22F9F705F8039FDFF8C8813B78002B22
:108050000CBF2B46002300930BF109010BF13F03EA
:1080600030465F22F8F7F4FF3B78039783F0010373
:1080700001276021C022C8F828605B42C8F80C6064
:10808000C8F8106088F81460A8F81660C8F818607E
:10809000C8F81C606048C8F820100BEB0706C8F849
:1080A0002420A8F80830C8F80460C8F82C70C8F874
:1080B0000070F9F73DF83723584888E84800F9F789
:1080C00037F8039B56481B78C8F80070002B14BF84
:1080D0002B4600230BF12F05A8F80830C8F80450F0
:1080E000F9F726F8D4F8543BC8F804501B79052B4F
:1080F00096BF4C4A4C4852F8230040F6583606FBCF
:1081000009A63723C8F80030F9F712F8D6F8543B1F
:10811000464A1B784648002B18BF15460BF1380419
:108120000123C8F80030C8F80440F9F701F8D6F880
:10813000543B5878FBF7BEF93E4B0028B8BF40428D
:1081400083FB0032C317C3EBA20303EB8302A0EB54
:108150004202092802F1300203F13003CCBF2CA8FF
:108160000DF1B1008DF8B1208DF8B0300022492317
:108170008DF8B22088E81800F8F7DAFF40F6583397
:1081800003FB09A35A22D3F8543B2B481B78C8F8A9
:108190000020012B08BF2546C8F80450F8F7C8FF97
:1081A000F7E5264C6378002B50D0254B62681B689E
:1081B0001F931F9B9B1AB3F5FA7F47D9B9F1020FA2
:1081C0007FF4E7AD1F4A002102F1C0050023D15022
:1081D000C033B3F5104FFAD10432AA421948F5D191
:1081E000E168194BA3FB01429209A3FB0243DB099F
:1081F00003EB4303A2EB831302EB4202A1EB421217
:1082000003EB430302EB43134FF6FF7220F81320F6
:10821000BFE500BFD4190120B83D0200C43D0200F3
:10822000CC3D0200E8440200783D020019FCFFFF4B
:10823000D83D020067666666E43D0200B40F012087
:1082400074CE0120041A0120ABAAAAAA40F6583322
:1082500003FB09A3049393F87049042C00F0C68330
:10826000012C01F05381022C00F0E285032C01F077
:108270000E80BD4CDFF814831E460FCC24AD0FC515
:1082800094E80F00103485E80F000FCC2CAD089552
:108290000FC594E80F0085E80F00D6F8D82000231A
:1082A00001244FF6FF756020C0210B2AC8F82C402E
:1082B000A8F80850C8F82000C8F82410C8F82830DA
:1082C000C8F80030C8F80430C8F80C30C8F81030CE
:1082D00088F81430A8F81630C8F81830C8F81C30E0
:1082E00000F0CE87D6F8D8310B2B01F0C780D6F836
:1082F000D8320B2B01F0BE80D6F8D8330B2B01F00F
:10830000B580D6F8D8340B2B01F0AC80D6F8D83530
:108310000B2B00F0B88740F6583303FB09A3D3F8C2
:10832000D8260B2A00F0AB87D3F8D8370B2B14BF15
:108330004FF0FF330723079321A94846FFF76EFC50
:1083400040F6583303FB09F30AEB030200260C93B3
:108350009FED869ADFED868A9FED868A05924FEA29
:10836000490306920D961393CDF850B00496CDF8BC
:1083700054900499139A24AB53F82140089B53F866
:108380002130D71801EBA10313F0010F039B04EB7D
:1083900044044FEAC4044FEA47171B7800F02A81CF
:1083A000002B40F0198140F2B269059AD2F8D850FA
:1083B000A5F10902032A0E9200F2DF8249F6327219
:1083C00041F66479002B18BF9146002207980146B8
:1083D000013000F0C3820498814200F0BF824AF667
:1083E000522942F64201002B18BF89460C2D0D9BE5
:1083F00008BF01230D93002A0CBF4B4600230093B6
:1084000004F1170207F11F0339466E00204611964A
:10841000F8F71EFE0C9A731902EB8303049A1202FA
:10842000134453441092039A117893F8DF2093F881
:10843000DE300F93504B53F8253009934F4B53F8D0
:1084400025300A934E4B002953F82530129308BF6C
:108450004FF00009022A00F07E82032A00F08F828A
:10846000042A00F0E1844748474B012A08BF184618
:108470000B906B1E0B2B00F2AB80DFE803F09389AF
:108480008969A9529393A9A90693069B049A9B69AB
:10849000934200F0C08004F1020B4FF6FF73BA1C48
:1084A0001298A8F80830C8F80420C8F800B0F8F707
:1084B0003FFE079AA8F80890511C134600F0F6807A
:1084C000049A934200F0F280049B01331A4604930D
:1084D000059B082A03F5807305937FF44AAF039B3D
:1084E000DDF850B01B78DDF85490ABB10BF12002F1
:1084F000BF2A40F2C6870BF140070BF10106172493
:1085000042F663452246204600953B4631461834E4
:10851000F8F7D6FD5F2CF5D149460398FBF7EAF84A
:1085200037E40F9B049A012B0BBF069B059B93F826
:108530005F3093F891311E46069B9B6993426CD045
:1085400004F1020B4FF6FF73002E08BF4B46A6E75F
:108550000F9B049A012B0BBF069B059B93F85E3083
:1085600093F892311E46E7E7BC2F02000534833AA8
:1085700000802A440000C84220430200D43C02008C
:10858000BC450200103D0200983D0200D4190120B4
:10859000069B049AD3F86C399B1AB3FA83F35B09F0
:1085A0001E46C9E7059A92F890311BB9D2F89C3162
:1085B000013303D0239B002BBFF667AF069B049AC1
:1085C0009B69934200F09E8704F1020B4B4666E7DD
:1085D00000231E46049AAFE7059BD3F8D850A5F1B7
:1085E00009030122032B0E93134640F2B18140F29E
:1085F000F929EBE6002BEFD1012340F2B129D4E6B3
:1086000041F2A543009359460BF13F035F22F8F76F
:108610001FFDFFF7BEBB01231E46069B93F8622099
:108620004B429BB23AB1204A12682092209AC2F380
:108630000802FF2A84D8069A5269013A062A3FF6B0
:108640007FAFDFE802F02D2A2A1D1004040007F195
:108650001E0200931146134604F1110004F11502A5
:10866000F8F7F6FC6CE707F11E020093114613467B
:10867000E01C04F11302F8F7EBFC04F1020B61E7D4
:1086800007F11E0204F1020B0093114613465846EF
:1086900004F10C02F8F7DCFC54E707F11402E4E7FC
:1086A00007F10A02E1E700BF74CE0120099B5A07D7
:1086B00055D5059B039993F8E920C64B09780132FB
:1086C00083FB0230D317C3EBA00303EB8300A2EBC1
:1086D0004002303230338DF8792000228DF8783026
:1086E0008DF87A2019B142F66343A8F8083007F1F3
:1086F0000C09B948C8F800B0C8F80490F8F718FD9C
:108700000A9B5B0740F15481039B1B78002B42F6C8
:10871000634208BF0022069B0599D3F8D83A91F826
:10872000E910A8F808205A1892F89021632A09D86D
:1087300003EB8203D3F8F431002B03DD059BD3F860
:10874000EC3023B92A238DF878308DF8793004F194
:1087500008031EA888E80802F8F7EAFC099B1E0730
:1087600050D5119B0C9A9D492B4402EB8303109A20
:108770001344534493F8DC2051F82220100740F1B1
:108780002181B3F9E6200E9B012B01F2178007EE41
:10879000902AF8EEE77AB7EE007A67EE897AF4EE7F
:1087A000C77AF1EE10FA00F1C4873022134638215F
:1087B00000201E908DF879300A9B8DF878101907EB
:1087C0008DF87A2040F1FB80069B1B68012B049BEF
:1087D00000F0F18023F00403032B00F0F080039BF2
:1087E0001B78002B42F6634308BF002307F10C02FD
:1087F0001EA8A8F80830C8F800B0C8F80420F8F798
:1088000097FC099B9A0636D5119B0C9A73492B4409
:1088100002EB8303109A1344534493F8DC2051F87D
:10882000222012F0200200F0AD8093F9E510002321
:1088300099421E9340F0468620228DF878203023FE
:108840008DF87A300A9B8DF879209B0640F1A18043
:10885000039B1B78002B42F6634308BF002307F1FC
:1088600016021EA8A8F80830C8F800B0C8F80420FE
:10887000F8F75EFC099BDE061CD5039B1B78002BDA
:1088800000F08A800A9B4CF2F65213F0100F42F669
:10889000634318BF1346A8F808300F9A504B02EBF9
:1088A00042001844621C07F1160388E80C00F8F730
:1088B0003FFC099B58061AD5072D00F0AF870A9B8D
:1088C00013F0400F039B00F09F871B78002B4CF2A6
:1088D000174318BF0423A8F8083007F1160304F162
:1088E00010020B9888E80C00F8F722FC099B190687
:1088F0007FF5EAAD119B0C9A38492B4402EB8303B8
:10890000109A1344534434A893F8DC2051F82220E1
:10891000120643BF93F9E4303033DBB22E2300223A
:10892000ADF8782000F8583D039B197849F6FC72A1
:1089300043F2994310341637002908BF1346C8F88C
:108940000040C8F80470A8F80830F8F7F1FBBBE560
:1089500045F614793AE5234B0B938AE50D990029E6
:108960003FF444AD0C2D7FF446AD4AF6522942F651
:108970004201002B18BF89463DE5002226E51A4B2F
:108980000B9376E52D211E9232238DF8781020224C
:1089900056E74FF6FF7362E70A9B4EF2FF4213F071
:1089A000100F48F2396318BF1346A8F8083074E76F
:1089B0004FF6FF72AFE633F004037FF410AF4FF6CB
:1089C000FF7313E70E9B012B40F2158430231946E9
:1089D0002E22EDE667666666FC3D0200204302003B
:1089E000FC2F0200A83D0200903D0200DB6A002B34
:1089F000C0F20687034493F8903100EB8300D0ED7A
:108A00007D7AFAEEED7AFDEEE77ACDED057A41F268
:108A1000A54300935F220BF10803594600200BF198
:108A200009040BF13F0507940995F8F711FB21465E
:108A30002B465F220020F8F7BBF940F6583303FBC2
:108A400009A3DFF8DC83DA6A0123C8F82C3000239D
:108A50006020C0219A42C8F82000C8F82410C8F845
:108A60002830C8F80030C8F80430C8F80C30C8F80E
:108A7000103088F81430A8F81630C8F81830C8F844
:108A80001C30A8F808301BDBDF492C93531C81FBFA
:108A90000321DA17C2EBA10202EB8201A3EB41032F
:108AA000303330327A240BF101012CA88DF8B2302A
:108AB0008DF8B1208DF8B040C8F80410F8F738FBF5
:108AC00040F6583303FB09A3D3F874C9BCF1000F77
:108AD00000F0CD809CF83220002A00F0C880D3F846
:108AE0007829CA4EC84BCA49CA4D0CEB420CBCF897
:108AF000024086FB0426B60981FB042183FB0402A5
:108B000083FB067080089208490900EB8000A6EB01
:108B1000400683FB017083FB027380089B0885FB82
:108B2000047500EB800003EB8303A1EB4001A2EB93
:108B300043032CA802EB82022D0B0746A4EB420450
:108B400005F13002302A03F1300308904FF00000A5
:108B5000C7F8030006F130068DF8B4304FF02E0050
:108B600008BF202301F130018DF8B02004F130045A
:108B700008BF8DF8B030022238238DF8B1608DF82F
:108B8000B2000BF1010608988DF8B3108DF8B540CE
:108B9000C8F80C2088E84800F8F7CAFA40F65833BD
:108BA00003FB09A3994CD3F87809D3F874299849A1
:108BB000954BC8F8046002EB4002558B84FB0524FA
:108BC000A40981FB052183FB050283FB0470800857
:108BD000490900EB8000A4EB4007920883FB0140A9
:108BE000800883FB02438B4C9B0800EB8000A1EBC9
:108BF000400003EB830384FB0514A2EB4303240B27
:108C000002EB8202A5EB42023034089D8DF8B040A1
:108C100030330021302CC5F8031000F130008DF8FE
:108C2000B43002F1300208BF2023C8F80C108DF8D0
:108C3000B3004FF02E018DF8B52008BF8DF8B0308D
:108C400002225F2330370898C8F80C20C8F800309B
:108C50008DF8B1708DF8B210F8F76AFA40F6583313
:108C600003FB09A30022D3F874C9C8F80C2040F60E
:108C7000583707FB09A7DFF8AC81674D07F6F70700
:108C80000BF1240E002617F8012F02EB420202EB33
:108C9000C2021212C2EB0E010EEB0203994217DC64
:108CA0000133581A01EB410100EB400006EB41147F
:108CB000800108EB44045242002382EAE271A1EBF6
:108CC000E271013235F81110E152C0338342F4D120
:108CD0000136602ED7D1BCF1000F79D09CF832302C
:108CE000002B75D09CF80030002B71D00599CDF881
:108CF000289001EBD17340F658325B10012902FB3A
:108D000009A605930B46B8BF012306930BF10C0788
:108D10004FF00008CDF820B06246B14620E04FF693
:108D2000FF7607F1020B39465B4622462046009645
:108D3000F8F78EF9AC422246B8BF2A46AC425B46F1
:108D400020460096A8BF28465946F8F781F9D9F879
:108D50007429137808F10108434507F1040733DD4E
:108D600002EB480CBCF80220BCF81A3002EB4204BB
:108D700003EB4305C2EB4414C3EB4515059A059B71
:108D800014441D44069A069B94FBF2F495FBF3F5FC
:108D90005E2CD9F87839D4BF24EAE4745F245E2DC0
:108DA000D4BF25EAE5755F254345B8D11B4BD9F8FB
:108DB0007C291B682C932C9B9B1AC3F30803FF2B65
:108DC000ADD840F22146ACE7DDF820B0DDF82890C0
:108DD00040F6583303FB09A39A6B002A07DB4FF6D2
:108DE000FF700090099B07991046F8F731F9039C32
:108DF000049A59462046FAF7A7FB49462046FAF757
:108E000079FCFEF7C6BF00BF67666666D34D621089
:108E10001F85EB51AD8BDB680045020074CE01204D
:108E2000D4190120041A0120BA4B0B93FFF721BB80
:108E30001946DB6A002BC0F20F82C2180B6B92F846
:108E4000902100EB8200D0ED7D7AFAEEED7A03EB13
:108E50004302FDEEE77AC3EB421117EE903A03EBC3
:108E6000D37252101144012B1046059140F3FB813F
:108E70000846049990FBF3F0496B059001EB410023
:108E8000C1EB401117EE904A8D1841F2A5430BF14A
:108E900009060BF13F0700935F220BF108035946C7
:108EA0000020B04695FBF4F4079609940A97F8F76A
:108EB000CFF83146059E2546304648F231646A1E99
:108EC0003B460130F7F774FF41463B46009432467B
:108ED0000020F8F7BDF8009440F6583404FB09A4CC
:108EE00041463B46DFF8448228465F22F8F7B0F857
:108EF0000123E26AC8F82C3000236020C0219A4286
:108F0000C8F82000C8F82410C8F82830C8F8003085
:108F1000C8F80430C8F80C30C8F8103088F814309D
:108F2000A8F81630C8F81830C8F81C30A8F808306F
:108F300080F266810BF1010306932CAB089340F697
:108F4000583303FB09A3744A196B93F85D005F6BF8
:108F5000724D734B734C002818BF0F46F81782FBF5
:108F60000712C0EB223283FB021685FB071584FB38
:108F70000714D117C0EBA51EC1EBA60683FB07158E
:108F8000C0EB641CC0EBA50506EB860683FB0E1048
:108F90004FEAEE71C1EBA001A2EB460483FB0C0289
:108FA00083FB05034FEAEC70C0EBA20201EB8101E9
:108FB000E817AEEB4101C0EBA303303103EB8303B1
:108FC0003034E4B205EB8500A5EB43038DF8B11016
:108FD00002EB820208998DF8B0403033302CACEBB4
:108FE00042024FF00006A7EB4000C1F8036000F119
:108FF00030008DF8B43002F1300208BF20238DF824
:10900000B5008DF8B32008BF8DF8B03002225F2381
:1090100008980699C8F80C202E25C8F80030C8F822
:1090200004108DF8B250F8F783F840F6583303FB7C
:1090300009F3002203F6F706C8F80C2053440BF19D
:10904000240C0BF13C08CDF820B0DFF8E4E0DDF8AB
:1090500024B03548CDF82490DDF8149006931446DA
:10906000564416F8015F05EB450505EBC5052D12C5
:109070004C45C5EB0C020CEB05035BDDA34531DD74
:109080009A4217DC01339B1A02EB420203EB4303C3
:1090900004EB42129B010EEB42026D42002185EA75
:1090A000E577A7EBE577013530F817705752C031F7
:1090B0008B42F4D10134602CD3D1DDF82490DDF85B
:1090C00020B040F6583303FB09A39A6B002AFFF641
:1090D0008EAE4FF6FF7000900A9B07991046F7F787
:1090E000B7FF84E6A34500F0B0809A42E2DC01338A
:1090F0009B1A02EB420203EB430304EB42110EEB1B
:1091000041019A0148F673650023CD52C033934262
:10911000FBD1CFE7943D0200AD8BDB68D34D6210ED
:10912000676666661F85EB5100450200D419012071
:10913000041A0120D6D1069991F85D10002900F09B
:109140007A83069991F87179002FCED1D6490968B2
:1091500024912499C1F30801FF298CBF002101212A
:109160009A42059116DC01339B1A02EB420203EB93
:10917000430304EB42129B010EEB42016D4285EA70
:10918000E572A2EBE572013530F81220CA53C03700
:10919000BB42F4D1079B059A03EB4203984589DB58
:1091A00003EB4302C3EB080352019B0803EB4303A9
:1091B00002F5C07101EBC3112144A3180EEB430368
:1091C0000EEB41024FF6FF714FF00005A3F840127D
:1091D0001D80A3F8C050A3F8801103F540739A4294
:1091E000F2D167E730460BF13F0359465F22F7F7AC
:1091F000DFFDFEF7CEBD302319463322FFF7D8BA84
:10920000AA492C93013281FB0231D317C3EBA1038E
:1092100003EB8301A2EB410230322CA908913033D9
:1092200008468DF8B2207A210BF1010206928DF8E2
:10923000B010C8F804208DF8B130F7F779FFE26A72
:1092400004985946F8F73EFE79E6069991F85D10C4
:1092500000293FF476AF48E70B6B03EB4302C3EB07
:1092600042130593002040F6583101FB09A1012467
:109270004B6B03EB4302C3EB42131D1805E60623B9
:109280000793FFF759B805230793FFF755B800294F
:1092900041F2A54318BF0023DFF81C8200935F2230
:1092A0000BF13F0359460020F7F7D2FE0123C8F81F
:1092B0002C300023C8F82830C8F80030C8F8043033
:1092C000C8F80C30C8F8103088F81430A8F81630F8
:1092D000C8F81830C8F81C301E46049BCDF818900A
:1092E0004FF6FF706021C0220BF1010AA8F80800B8
:1092F000C8F82010C8F824205546994627E003995D
:109300008DF8843091F800E08DF88520D64508BFAF
:1093100057461E2388E828008DF886A0A8F8087014
:10932000F7F706FF624B6348C8F80450012C08BFEA
:1093300018463023C8F80030F7F7FAFE032E0599D7
:1093400068D00136072E05F1090500F08880D9F8AC
:109350000430F41E1C44554B04F1010C83FB0C3209
:109360004FEAEC73C3EBA20303EB83022CA9ACEB33
:1093700042023033622C49F2B5674FF0000A0846CA
:109380004FF02E0E059302F13002DAD8039B8DF8D0
:10939000B22093F800C09DF814308DF8B3E0D445A6
:1093A0000CBFD446BC464C44032E14BF202184215C
:1093B00001228DF8B13088E82400A8F808C08DF8A3
:1093C000B0108DF8B4A0F7F7B3FE94F8DC4A374A32
:1093D0003949059182FB04239B0803EB8302A4EB2C
:1093E000420221A848F6736C3033303242F6634EA5
:1093F000002C84D1039B31481B78C8F804502422E8
:10940000002B08BFE646C8F80020A8F808E0F7F7E8
:109410008FFE96E7D9F81000244A431C82FB0324F0
:10942000DA17C2EBA40202EB8204A3EB440350451B
:1094300002F1300203F130034FF6FF774FF053048F
:1094400024A8FFF67EAF8DF892A08DF890208DF8BD
:1094500091300F8181E83000F7F76AFE71E7DDF89F
:109460001890C4E404230793FEF766BF0323079311
:10947000FEF762BF02230793FEF75EBF0794FEF775
:109480005BBF0F4B02EB420203EB821242F66341D9
:10949000002322F813100233602BFAD1FFF72BB808
:1094A0001546FEF78BBC00BF74CE0120676666666A
:1094B000803D0200883D0200D4190120F43D0200E5
:1094C000041A012040F32281DD4BCA1783FB0103FC
:1094D000C2EBA30303EB8303A1EB43033033DBB203
:1094E00001F109004FF02B0E12288DF878E040F2C0
:1094F0000A81D34880FB0101C2EBA1023032D2B213
:10950000FFF79EB900231E46FFF787B841F2A54238
:109510000BF108050BF109062B46009259465F2214
:1095200000200BF13F0705960697F7F791FD3146AE
:109530003B465F220020F7F73BFC049EDFF82083C8
:10954000326AC8F82C4000236020C0219A42C8F833
:109550002000C8F82410C8F82830C8F80030C8F82F
:109560000430C8F80C30C8F8103088F81430A8F867
:109570001630C8F81830C8F81C30A8F8083020DBBE
:10958000AF492C93531C81FB0321DA17C2EBA102D4
:1095900002EB8201A3EB410330320BF101013033C6
:1095A0002CA87A248DF8B120C8F804108DF8B230B8
:1095B0008DF8B040F7F7BCFD326A59463046F8F7EF
:1095C00081FC40F6583303FB09A393F8602022B3D3
:1095D000D3ED097A9FED9B7AF8EEE77A40F2B2601C
:1095E00067EE877A4FF6FF7177EEA77A2B46FDEE8E
:1095F000E77A322217EE904A14F0010F18BF0146A5
:10960000009120205946F7F723FD20220BF101039A
:109610008D4888E80C00F7F78BFD40F6583303FBC4
:1096200009A35B6A002B28DD07EE903ADFED876A1D
:10963000834B874AF8EEE77AB6EE007AA7EEA67A71
:109640002CA8FDEEC77A17EE901A83FB0134CB17D6
:10965000C3EBA40303EB8304A1EB440100910F21AE
:1096600015F0C6F802215F220BF101032CA8C8F8FF
:109670000C1088E80C00F7F75BFD40F6583707FB45
:1096800009A7DFF8E0C1734D07F6F7070BF1240EC9
:10969000002617F8012F02EB420202EBC20212125F
:1096A000C2EB0E010EEB0203994217DC0133581A8C
:1096B00001EB410100EB400006EB411480010CEB93
:1096C00044045242002382EAE271A1EBE2710132CA
:1096D00035F81110E152C0339842F4D10136602EB2
:1096E000D7D140F6583303FB09A39A6B002AFFF643
:1096F0007EAB4FF6FF700090069B05991046F7F77A
:10970000A7FCFFF774BB2022FFF79AB8A3F19933A7
:1097100001F10900494283FB0123CA17C2EBA303ED
:1097200003EB8303A1EB43033033DBB24FF02D0E89
:10973000DAE6F5EEC07AF1EE10FA7FF75CAD67EE8F
:10974000A87A454B3E4ABDEEE77AB6EE006A17EEC0
:10975000101A03EB8101D1ED006AD1ED015AB8EE88
:10976000C77A77EEC77A35EEE67AE7EE876AF0EEEB
:10977000467AE6EE887AFDEEE77A17EE903A82FBBB
:109780000360D917C1EBA00082FB002E334EC21735
:10979000C2EBAE0202EB820C86FB036E00EB800292
:1097A000A3EB4202A0EB4C00C1EB6E113030303223
:1097B0003031C3B2D2B2C9B2FEF7FABF204BD117D3
:1097C00083FB0260C1EBA00C83FB0C30234E4FEAFD
:1097D000EC73C3EBA00086FB026E0CEB8C0300EB7A
:1097E0008000A2EB4302ACEB4000C1EB6E1100F134
:1097F000300330323031DBB2D2B2C9B2FEF7D8BF5B
:1098000001230593FFF703B9197848F2396242F64C
:109810006343002908BF1346FFF75DB8039B19781F
:1098200049F6FC7243F29943002908BF1346A8F891
:109830000830FFF752B8A3457FF457AC81E400BF6E
:10984000676666666F120338E83D02000BD7A339DE
:10985000EC3D020000450200283202001F85EB515A
:10986000D4190120041A01202DE9F04F8DB0804653
:1098700008916C480992002199466B4CFEF7FAF961
:1098800001216848FEF7F6F902216648FEF7F2F971
:10989000236813F0010500F0A380DFF8A8B1634F3F
:1098A000634C644D002648F6907A0AFB06F2BB181A
:1098B00003F547533C33197804294BD00AFB067350
:1098C00003F547533C331B78052B00F085800AFBDA
:1098D000067303F547533C331A78032A02D01A78EB
:1098E000002AF9D1013604F50F4405F50F45032E82
:1098F00004F1900405F1900548F69073D5D103FB6F
:1099000008F3FC1843F614221698CDF818B0A258A4
:10991000494905900998029004F548530898019028
:1099200004F575570DF12F05CDF810900833009709
:10993000A1F5A6600395FCF769FD40B104F57D52E1
:1099400043F648739DF82F1011600422E2500DB0C9
:10995000BDE8F08F19780429B0D155F8041CDFF860
:10996000E8E044F2A00000FB01223048104400F57A
:109970007E5CDCED007A724492ED007AF8EEE77AD4
:1099800067EE877AF5EE407AF1EE10FA3FD000F5F7
:109990007D5300201A469E4683F83000D8699B6AA2
:1099A000C31A9F2B02F11C020EF1280E03DDA03812
:1099B000CEF80000106844F2A0020AFB06F302FB96
:1099C00001333B4403F57D532C331A68121A9F2A46
:1099D000C4BFA030186071E72046FDF76BFB76E747
:1099E000204612F05BF9DFF85CB008B90F4F57E77B
:1099F000124A134B0D4FCBF80C502046CBF80020E9
:109A0000CBF80830CBF8047012F04EF948E74FF06D
:109A1000FF322A602269032122F024022261197098
:109A20004CE700BFD0190120E417FF1FA81CFF1F3F
:109A3000984EFF1F24DEFF1F7C39FF1FB82F020046
:109A400089410000E817FF1F1C5CFF1F0FB410B511
:109A500082B004AB054C53F8042B019340212046FF
:109A600016F0B6FD2146024810F012FA641CFF1FE2
:109A7000A81CFF1FF8B5164BD0F880521E78D0F8FE
:109A80008442144B0135002E05F01F0514BF012739
:109A90000327A54203FB01F116D0D0F8804204EB66
:109AA0008404A4000319002601314FF0040E06556A
:109AB0009A6059605E739E73DE731F7483F80CE0C6
:109AC000C0F880520846F8BD0348FFF7BFFF00BF4B
:109AD0003ACC0120282809009C3D02002DE9F04FD6
:109AE00041F204332DED048BC458ADF5717D8346EE
:109AF00064B1237C022B00F08D85032B00F0CC8118
:109B0000012B00F02C85DF48FFF7A0FF41F2083061
:109B10005BF80020531C052B00F341824FF42271A7
:109B20004BF8003001FB03B1D1F82443D1F82813DE
:109B3000A14200F0BD844FF4227202FB03F30BEB51
:109B4000030041F20434D0F82813D0F8282301EBA5
:109B5000810103EB81035B440132A43302F01F0255
:109B6000C0F828234BF804300BF598541034237AAE
:109B7000012B40F0C081D4F88400E36FD3F880104B
:109B8000D3F88420914200F0B981D3F88410D3F83F
:109B9000842053F82110013202F01F028842C3F8DA
:109BA0008420EBD1B84BB94E1D68B94A0E9541F2ED
:109BB000983000235BF800A00E98506006F51862FC
:109BC00006F68410136006F68812036006F68C1001
:109BD0001360B049036006F5196206F6941013602D
:109BE0008A454FF0FF320360C6F8982901F0D0840F
:109BF0004FF0000992464F4606EB09054FF0080862
:109C00003422002105F5D27085F8907185F89171A4
:109C100085F89271C5F8A0A1C5F89471C5F898713E
:109C200014F082FD0220622301224FF4FA7185F8BC
:109C3000F4004FF0030E042085F800E1C5F89CA164
:109C400085F8DC70C5F8E07085F8DF7085F8E470A1
:109C500085F8E570C5F8EC7085F8EB7085F8F07064
:109C600085F8F170C5F8F87085F8F67085F8F7702A
:109C700085F8FC7085F8FD70C5F8047185F80271EF
:109C800085F8037185F80871C5F8D82085F8DE20BD
:109C900085F8E82085F8EA2085F8DD3085F8E93098
:109CA00085F8F53085F80131A5F8E610A5F8F21031
:109CB000A5F8FE104FF0050E85F8097185F80C0126
:109CC000062085F818E185F824014FF0070E0820DA
:109CD00085F830E1A5F80A1185F80D31A5F81611BF
:109CE00085F8193185F81A21A5F8221185F8253152
:109CF000A5F82E1185F8313185F83221C5F810719B
:109D000085F80E7185F80F7185F8147185F8157155
:109D1000C5F81C7185F81B7185F8207185F82171D3
:109D2000C5F8287185F8267185F8277185F82C719A
:109D300085F82D71C5F8347185F8337185F838715F
:109D400085F839714FF0090EA5F83A1185F83C01F4
:109D50004FF41C7085F848E1A5F85201A5F85E01A2
:109D60004FF00B0E0C204FF00A0C85F860E185F8DF
:109D70003D3185F83E21A5F8461185F8493185F831
:109D80004A2185F8553185F8562185F8613185F8E5
:109D90006221A5F86A11C5F8407185F83F7185F810
:109DA000447185F84571C5F84C7185F84B7185F89B
:109DB000507185F85171C5F8587185F8577185F85B
:109DC0005C7185F85D71C5F8647185F8637185F81B
:109DD000687185F8697185F854C14FF00D0E85F8EA
:109DE0006C01B8F101084FF00E0085F86D3185F86F
:109DF0006E21A5F8761185F8793185F87A21A5F8D4
:109E0000821185F8853185F88621A5F88E11C5F86F
:109E1000707185F86F7185F8747185F87571C5F882
:109E20007C7185F87B7185F8807185F88171C5F842
:109E3000887185F8877185F88C7185F88D7185F842
:109E400078E185F8840105F580757FF4D9AE09F6CF
:109E5000583942F2082399457FF4CEAE41F29B6017
:109E600042F2F31141F22A7306F8008006F80180ED
:109E7000F25486F8438B86F87A2086F8D22B00239A
:109E800023723BE0003E020074CE012004AA0120B0
:109E9000B40F0120FF16FE122378AF4A002B40F0CA
:109EA0009D83AE49AE4EAF4D09781360A0686268DD
:109EB00001233370E368286001B95202AA4DAB4E0A
:109EC000AB48AC492A601B0443F40073AA4DAB4A6B
:109ED000336005600A6041F2043302225BF803300C
:109EE0002274002B3FF412AE0BF598541034237AF1
:109EF000012B3FF440AE022B00F018830BF5EC323F
:109F0000936D5C1C42D0013B40F0CB829C49DBF856
:109F1000440D0C78DBF8481D0130002C00F01F00C8
:109F20004FF0FF340CBF4FF0030E4FF0010E88428C
:109F3000946519D0DBF8444D04EB8404A4000BF6BF
:109F4000C42739190BF5EB35012658353E550B71F1
:109F50004B718B71CB710E734B738B73CB7381F819
:109F600010E08D60CBF8440D0BF58F531433D3F80C
:109F70008000D3F88410884208D0D3F88410D3F836
:109F80008410013101F01F01C3F88410D36D013337
:109F900011D00DF5717DBDEC048BBDE8F08FDBF8C1
:109FA0002433DBF82813002299424BF8002000F0FC
:109FB00079831346BFE543F2F0450BF51E545BF879
:109FC0000530D80704F1180400F1E284990717D589
:109FD000D4F8540DA3680DE0D3F88410D3F884208E
:109FE00053F82110013202F01F028842C3F8842086
:109FF00000F0B483D3F88010D3F884209142EBD1E1
:10A00000D4F81C38591C4CD0013BC4F81C3843B15F
:10A0100004F50463D3ED007AF5EE407AF1EE10FA20
:10A020003FD06668564BD4F818581878D6F8803266
:10A03000EC950133D6F8842203F01F0504F5046380
:10A0400000284FF000014FF0FF300CBF032701271D
:10A05000C4F81C08954219604FF0010004F1180182
:10A060004FF004038DF8BC738DF8AC03ED91EE93C3
:10A0700017D00DF56B7ED6F88072BEE80F0007EBA7
:10A080008707BF0006EB070C9EF800E0F051CCF804
:10A090000410CCF80820CCF80C308CF810E0C6F88E
:10A0A0008052237BDBB2022B00F09585052B1FD05D
:10A0B000012B00F080850BF53F561C36D6F80023A7
:10A0C000D6F804339A420FD0D6F804330293D6F868
:10A0D00004332269013303F01F03C6F8043312F07E
:10A0E0002003099300F03C87237B042B02F05C8063
:10A0F00000244FF4005242F298735BF80300816829
:10A100008B684D68AB4215D246680F6846F0004632
:10A1100034435E1C8E6047F82340D211B542446838
:10A1200042F080024FEA830004D9384402332243CC
:10A130008B6042604CF280460BF537445BF806308A
:10A14000DA0704F1280400F1B0849B072ED5D4F877
:10A15000540DA36824E000BF18CC012020CC0120BE
:10A1600028CC012000100B4008100B4004100B40BD
:10A1700038100B400C100B4002007F1137003A12D0
:10A180003ACC0120D3F88410D3F8842053F821105E
:10A19000013202F01F028842C3F8842000F0AC8331
:10A1A000D3F88010D3F884209142EBD1D4F81C3836
:10A1B000591C49D0013BC4F81C3843B104F5046371
:10A1C000D3ED007AF5EE407AF1EE10FA3CD06668F5
:10A1D000B54B0422A3921878D6F88032D6F88422A0
:10A1E0000133002803F01F05D4F81838A1934FF06D
:10A1F00001000CBF032301238DF880028DF89032FB
:10A2000004F1180004F504630021A29095424FF078
:10A21000FF30C4F81C08196016D0A0AFD6F880E251
:10A220000FCF0EEB8E0E4FEA8E0E06EB0E0C46F89D
:10A230000E00CCF80410CCF80820CCF80C303B7899
:10A240008CF81030C6F88052237BDBB2022B00F072
:10A250006C84052B1FD0012B00F09D840BF53F472C
:10A260006C37D7F80023D7F804339A420FD0D7F8C9
:10A2700004330293D7F804332269013303F01F0338
:10A28000C7F8043312F02003099300F0F384237B12
:10A29000042B02F04D8300244FF400524BF228733C
:10A2A0005BF8030081688B684D68AB4215D2466845
:10A2B0000F6846F0004634435E1C8E6047F823402A
:10A2C000D211B542446842F080024FEA830004D9BB
:10A2D0003844023322438B6042600BF5AA352B6968
:10A2E000DA0700F1A0839B0700F1AA820BF5A334E3
:10A2F0000BF5A333B8340293D4F81C38591C4BD057
:10A30000013BC4F81C384BB1029B03F6F803D3EDB4
:10A31000007AF5EE407AF1EE10FA3DD06668624BB5
:10A32000029F187804225892D6F88032D6F88422F8
:10A330000133002803F01F054FF00100D4F818384E
:10A3400056938DF854010CBF032301233846D030B7
:10A350008DF8643107F6F8030021579095424FF0CD
:10A36000FF30C4F81C08196016D055AFD6F880E24B
:10A370000FCF0EEB8E0E4FEA8E0E06EB0E0C46F84C
:10A380000E00CCF80410CCF80820CCF80C303B7848
:10A390008CF81030C6F88052237BDBB2022B00F021
:10A3A0004084052B1ED0012B00F0E5830BF5A7366A
:10A3B000FC36D6F80023D6F804339A420ED0D6F8ED
:10A3C00004A3D6F804332269013303F01F03C6F84F
:10A3D000043312F020030A9300F06C87237B042BD4
:10A3E00001F0238300244FF40052029BD3F8B800FD
:10A3F00081688B684D68AB4215D246680F6846F09D
:10A40000004634435E1C8E6047F82340D211B542AB
:10A41000446842F080024FEA830004D93844023392
:10A4200022438B604260DBF83C10DBF85C60CA685A
:10A43000DBF86030106802240025CBF86450C4714A
:10A440001768066004268680BE601668A340C3F3C2
:10A450008F00F08312685B42F360D082C8680B689B
:10A46000026834339471B3F1804F136195820368AD
:10A4700001D39A6812B904229A600368C8680B4A2B
:10A4800000249C61037913700A68136B012043F068
:10A490004073136308740DF5717DBDEC048BBDE84A
:10A4A000F08F936572E500BF3ACC01201B8000401D
:10A4B000931C41F204310022062B4BF8012040F09E
:10A4C000F680DBF82433DBF828434BF800209C426D
:10A4D0007FF46FAD4BF80120012341F208304FF4B7
:10A4E00022724BF8003002FB03B2D2F82413D2F8E8
:10A4F00028238A427FF41FAB41F20431013300224A
:10A50000052B4BF8012040F3F680DBF82433DBF811
:10A5100028434BF800209C427FF44BAD4BF80120C0
:10A52000012341F208324BF80230FFE0D4F88400F6
:10A53000E36F0DE0D3F88410D3F8842053F8211092
:10A54000013202F01F028842C3F884203FF497AC26
:10A55000D3F88010D3F884209142EBD1CEE4A54B00
:10A56000A54DD3F80080A54F11F0F8FD064605E093
:10A5700011F0F4FD801BB84200F2EA802B68DB0783
:10A58000F6D49F499F4BA04AC1F800801A6011F091
:10A59000E5FD9E4D994E074605E011F0DFFDC01B1D
:10A5A000B04200F2D5802A68994B98491340002B9D
:10A5B000F3D0984A0B6813600B601168944B0B4002
:10A5C000012B40F0C580944B1B68DD0540F1C08035
:10A5D000032323742378002B3FF463AC8F49904B03
:10A5E00090480978A56801261E70002313606268F0
:10A5F000E368056001B95202814D8B4E8B48814959
:10A600002A601B0443F40073894D8A4A3360056055
:10A610000A6060E4824B1B78002B40F0FA8141F223
:10A62000083241F254005BF802102278237401EBE7
:10A6300001110BEBC10641F25805335875597E4F95
:10A640000133A2F1010203F01F03B2FA82F25209B0
:10A65000AB423A7008D03258656802EB41020BEB0E
:10A660008202C2F8D45F33509BF8782041F204355F
:10A6700041F20C3100230A204BF805308BF878307A
:10A680004BF80100002A3FF441AA41F20C315BF87B
:10A690000120002A05F06780013A012020744BF860
:10A6A00001201EE441F2043101234BF8012041F264
:10A6B00008304FF422724BF8003002FB03B2D2F89C
:10A6C0002413D2F8282391427FF435AA41F20431B1
:10A6D00001330022062B4BF801207FF4FEAEDBF89D
:10A6E0002433DBF828434BF800209C427FF461AC14
:10A6F0004BF80120012341F208304FF422724BF84D
:10A70000003002FB03B2D2F82413D2F828238A4285
:10A710007FF411AA41F2043101330022062B4BF8D9
:10A7200001207FF4FEAE4BF8002013464FF4227256
:10A7300002FB03B2D2F82413D2F8282391427FF40B
:10A74000FAA941F2043300224BF80320FFF7CCBBF7
:10A7500041F204335BF80330FFF7C3BB43F2F0432D
:10A760005BF803301A0739D5D4F8503DD4F85C1D96
:10A77000E21804EB430392F8F425B3F82C3507EE06
:10A78000903AD60742BFF8EE677ADFED2C6A86EE84
:10A79000A77A0BF54C520BF54D5001F1FF3102F148
:10A7A0001B0200F13B0058BFB7EE007A12F8013FE0
:10A7B00007EE903AF8EEE77A824267EE877AFCEE8F
:10A7C000E77A17EE903A01F8013FEFD143F2F042F9
:10A7D0005BF8023023F008034BF80230D80601F191
:10A7E000B68023F0020343F2F04243F004034BF837
:10A7F000023005E41CCC012024100B4040420F0025
:10A8000008100B400C100B4000001A0D30100B40CC
:10A8100001000F0018CC012010100B4020CC0120AB
:10A8200028CC012000100B4004100B4038100B40C6
:10A8300002007F1127003A193ACC012000FEFF46A2
:10A840000BF5A33303F1B8040293D4F8540DA368B5
:10A85000D3F88010D3F8842091423FF44DADD3F863
:10A860008410D3F8842053F82110013202F01F0223
:10A870008842C3F88420EBD12B691F0733D5D4F865
:10A88000503DD4F85C1DE21804EB430392F8F42524
:10A89000B3F82C3507EE903AD60742BFF8EE677A48
:10A8A0005FED1A6A86EEA77A0BF5A93000F13B023C
:10A8B00001F1FF3100F19B0058BFB7EE007A12F8AA
:10A8C000013F07EE903AF8EEE77A904267EE877A1A
:10A8D000FCEEE77A17EE903A01F8013FEFD12B69D1
:10A8E00023F008032B61D80601F16B8023F00203EB
:10A8F00043F004032B61FFE44CF280435BF8033028
:10A900001F0739D5D4F8503DD4F85C1DE21804EB8C
:10A91000430392F8F425B3F82C3507EE903AD607A6
:10A9200042BFF8EE677A5FED3B6A86EEA77A0BF5D9
:10A9300042420BF5434001F1FF3102F1AB0200F15D
:10A940000B0058BFB7EE007A12F8013F07EE903ABD
:10A95000F8EEE77A824267EE877AFCEEE77A17EE46
:10A96000903A01F8013FEFD14CF280425BF802309F
:10A9700023F008034BF80230D80601F1058023F0DC
:10A9800002034CF2804243F004034BF802300DE422
:10A99000B74AD4F804E01678DEF88022D4F8540DD3
:10A9A000DEF88412E790002E02F101020CBF0320B2
:10A9B000012002F01F0C04F535628DF8A803E8921F
:10A9C000002001228C458DF89803E99217D0E6AE5D
:10A9D000DEF880720FCE07EB8707BF000EEB07088B
:10A9E0004EF807003078C8F80410C8F80820C8F8F6
:10A9F0000C3088F81000CEF880C25BF8053023F0E8
:10AA0000010343F2F04243F002034BF80230FFF738
:10AA1000F7BA90F87830002280F87820002B3FF4C5
:10AA200063AA234631E60BF5A33202F1B8041646B9
:10AA30006768029201225392D7F880228C49013232
:10AA40000878D7F8841202F01F0E00228DF84021FA
:10AA5000D4F8542D5192002806F6084252920CBFA9
:10AA6000032201228E458DF8502118D00DF5A07CCF
:10AA7000D7F88062BCE80F0006EB8606B60007EB4D
:10AA80000608B851C8F80410C8F80820C8F80C30F7
:10AA90009CF8003088F81030C7F880E22B6923F06A
:10AAA000010343F002032B6126E4D4F804E070496B
:10AAB00001229E92DEF880220878DEF884120132AC
:10AAC00002F01F0C00228DF86C22D4F8542D9C92B9
:10AAD000002804F535629D920CBF032201228C45AB
:10AAE0008DF87C2217D09BADDEF880720FCD07EB7E
:10AAF0008707BF000EEB07084EF80700C8F80410E0
:10AB0000C8F80820C8F80C302B7888F81030CEF838
:10AB100080C25BF8063023F001034CF2804243F020
:10AB200002034BF80230FFF741BBD4F81808A368C2
:10AB3000D3F88010D3F8842091423FF4ACABD3F823
:10AB40008410D3F8842053F82110013202F01F0240
:10AB50008842C3F88420EBD1D4F82038C4F82438D4
:10AB60004FF0FF320323C4F8202823734FF4005220
:10AB70000024FFF793BB029BD4F82018606803F110
:10AB8000D002FEF777FF0223C4F8180823734FF4AE
:10AB90000052002429E404F11802D4F82018606857
:10ABA000FEF768FF0223C4F8180823734FF400521D
:10ABB0000024FFF773BB04F11802D4F82018606872
:10ABC000FEF758FF0223C4F8180823734FF400520D
:10ABD0000024FFF790BAD4F81808A368D3F88010BF
:10ABE000D3F8842091423FF483AAD3F88410D3F899
:10ABF000842053F82110013202F01F028842C3F86A
:10AC00008420EBD1D4F82038C4F824384FF0FF3238
:10AC10000323C4F8202823734FF400520024FFF7C5
:10AC20006ABAD4F81808A368D3F88010D3F884203F
:10AC300091423FF4D7ABD3F88410D3F8842053F873
:10AC40002110013202F01F028842C3F88420EBD1A8
:10AC5000D4F82038C4F824384FF0FF320323C4F866
:10AC6000202823734FF400520024FFF7BEBB00BF1F
:10AC70003ACC0120029A530004931344DB000BEBFF
:10AC8000030211463B4406924BF67072D3F80890CB
:10AC900051F80280049B029A134407EBC303C84592
:10ACA0005B69AABF4E464646C146002B06DB4B45B4
:10ACB00082F2FD83B342B8BF33469846069AD4F871
:10ACC00024084BF66C73C6EB080652F803A087AA5B
:10ACD000514682AB00924246FBF7D8F8D4F82428BC
:10ACE0009C4B8299059103FB02F3063341F271728A
:10ACF00002FB0A33CB1A032E089302F32E83964BE2
:10AD00001B780793012200230A920393194648F601
:10AD1000887344F2A002E358059D079E8D95B3FA0F
:10AD200083F35B0901EB410102FB03F202EB8102B9
:10AD3000224444F69C5044F6A05115504FF00100B7
:10AD40005054D4F804C09DED878ADCF88012DCF8FA
:10AD50008402013101F01F01002E0E4644F6985185
:10AD6000354652588E920CBF032201228DF84022A4
:10AD70004FF000028DF8302286424FF004028F928D
:10AD80006ED0DCF880E28CAE0FCE0EEB8E0E4FEA6A
:10AD90008E0E0CEB0E0A4CF80E00C8EB0909CAF82F
:10ADA0000C303678CAF8041048F68873CAF80820C0
:10ADB0008AF81060B9F1030FCCF88052E3584CDDEB
:10ADC0000A9A079D44F2A001002B18BF002102EB54
:10ADD000420201EB8202224444F6A0514FF00100EE
:10ADE000059B505444F69C5104335350D4F804C08E
:10ADF0009793DCF8800244F6985100F1010951580C
:10AE0000DCF884229891002D09F01F090CBF032063
:10AE100001204FF00001042391458DF858129993B9
:10AE20008DF8680216D096AEDCF880E20FCE0EEBFD
:10AE30008E0E4FEA8E0E0CEB0E0A36784CF80E0092
:10AE4000CAF80410CAF80820CAF80C308AF8106052
:10AE5000CCF8809248F68873E358B3FA83F35B0921
:10AE600044F2A00202FB034000F66850FCF700F930
:10AE700048F68873E358002B42F015810299049B31
:10AE8000069D4BF66C720B44A85807EBC3034BF6B8
:10AE9000707244F60861AE5893F80CE09A686050FE
:10AEA000231848F69861039D93F8F435655044F6ED
:10AEB0000C61B8EEC88A44F6206C44F801809642D2
:10AEC00004F59C4181ED048A04F80CE044F6186115
:10AED000B646A8BF9646B242B8BF324644F61C6694
:10AEE00044F801E044F61461A251089A6250DA076E
:10AEF00042F1E38204EB4003DFED186AB3F82C352E
:10AF000007EE903AF8EE677A04F50E4386EEA77ADC
:10AF100083ED297A029A049B134407EBC3071D466D
:10AF200004F59C433869586244F6286201230021E5
:10AF3000A15009931A4644F2A00303FB02430022E6
:10AF4000C3F88C2D236923F0020343F0010323612E
:10AF5000FFF79DB9282809003ACC012000FEFF46E2
:10AF6000029A530004931344DB000BEB03021146D7
:10AF70003344059242F6E072D3F808808F58049B60
:10AF8000029A134406EBC30347455B69B6BFC2464A
:10AF9000BA46B846002B06DB534582F2858243450C
:10AFA000B8BF43461F46059AD4F8240842F6DC731E
:10AFB000C8EB070852F80390D2AB494600933A46D3
:10AFC000CDABFAF763FFD4F82428B74BCD9906919F
:10AFD00003FB02F3063341F2717202FB0933CB1A11
:10AFE000B8F1030F089302F35B81B04B1B78079312
:10AFF000012200230A9203930D46184648F68873EF
:10B0000044F2A001E258D895B2FA82F35B0900EB52
:10B01000400001FB03F101EB8001214444F69C5EFA
:10B0200044F6A05041F80E504FF001050D54079D15
:10B03000D4F80480DDEDD27AD8F88002D8F884E222
:10B04000002D44F6985500F101004959D9910CBFE3
:10B050000321012100F01F008DF86C134FF0000157
:10B060008DF85C1370454FF00401DA91054602F04B
:10B070003A820DF5577CD8F880E2BCE80F000EEB61
:10B080008E0E4FEA8E0E08EB0E09C7EB0A0A9CF8EB
:10B0900000C048F80E00BAF1030FC9F80C30C9F827
:10B0A0000410C9F8082089F810C048F68873C8F859
:10B0B000805242F31082E3584FF000028DF884234F
:10B0C00044F2A002002B18BF002213460A9A02EB9A
:10B0D000420203EB8202224444F6A0514FF00100E9
:10B0E000069B505444F69C510433535044F69851F7
:10B0F000D4F804805058D8F88022E3900798D8F804
:10B100008412E2930132002802F01F094FF0040379
:10B110000CBF032201228945E4938DF8942319D0B2
:10B120000DF5617CD8F880E2BCE80F000EEB8E0EC6
:10B130004FEA8E0E08EB0E0A9CF800C048F80E008D
:10B14000CAF80410CAF80820CAF80C308AF810C0EF
:10B15000C8F8809248F68873F8EEE77AE258B2FAB7
:10B1600082F35B0944F2A00101FB034303F557603E
:10B1700000214FF00008C3F8681DC3F86C1D44F6A9
:10B18000FC5CC0F8008003F59C4844F6F850C3F816
:10B19000741DC3F8781DC3F87C1D83F8801DC3F8A7
:10B1A000841DC3F8881DC3F88C1D4FF0FF3E01219C
:10B1B0004FF07E5AC3F8901D43F80CE043F800E0CE
:10B1C000C8F800E0C8F804A0002A42F01C810298E8
:10B1D000049A059D024442F6DC7106EBC20242F677
:10B1E000E070695855F800C0906892F80C80039D93
:10B1F00004EB010E44F6086284459EF8F495A150D4
:10B200006246A8BF02466045B8BF604648F6986EE1
:10B2100044F60C6C44F80E5044F80C7004F59C4E47
:10B2200044F6186CCEED047A44F6146744F6206EAA
:10B2300044F80C2019F0010F089AE251C3F87C0D74
:10B2400004F80E8002F0538104EB4101DFED186A2F
:10B25000B1F82C3507EE903AF8EE677A04F50E4314
:10B2600086EEA77A83ED297A029A049B134406EBB3
:10B27000C3061D4604F59C433069586244F62862B3
:10B2800001230021A15009931A4644F2A00303FBB5
:10B2900002430022C3F88C2D236923F0020343F0FC
:10B2A00001032361FEF720BF282809003ACC0120C2
:10B2B00000FEFF464FEA4A0304935344DB000BEBC6
:10B2C0000302334402F5A7329D68049BD2F8007153
:10B2D0000792534406EBC303AF425B69B6BFA9466E
:10B2E000B9463D46002B06DB4B4582F2E380AB427C
:10B2F000B8BF2B461F46079BD4F82408D3F8FC8020
:10B300003CAA414637AB00923A46FAF7BFFDD4F863
:10B3100024289C4B3799059103FB02F3063341F235
:10B3200071727D1B02FB0833CB1A032D089301F3C6
:10B330005E87954B1B780693012200230B920393A3
:10B34000194648F6887344F2A002E358059D9DED26
:10B350003C8A4295B3FA83F35B0901EB410102FB9E
:10B3600003F202EB8102224444F69C5044F6A051C1
:10B3700015504FF001005054D4F804C00698DCF882
:10B380008012DCF884E2002844F6985001F10101B3
:10B390001258439201F01F010CBF032201220991B0
:10B3A0008DF81421099A4FF000008DF804017245C0
:10B3B0004FF0040044906FD0DCF880E241AD0FCD37
:10B3C0000EEB8E0E4FEA8E0E0CEB0E084CF80E00B4
:10B3D000C7EB0909C8F80C302D78C8F8082048F6E2
:10B3E0008873C8F8041088F81050099ACCF88022A5
:10B3F000B9F1030FE3584CDD0B9A44F2A001002B86
:10B4000018BF002102EB420201EB8203234444F601
:10B41000A0514FF00100059A585444F69C51043253
:10B420005A5044F69851D4F804C05958DCF8803288
:10B430000698DCF884524D910133002803F01F096F
:10B440004FF000030CBF032001208DF82C31A945DB
:10B450004FF004034C924E938DF83C0116D04BAD47
:10B46000DCF880E20FCD0EEB8E0E4FEA8E0E0CEB69
:10B470000E082D784CF80E00C8F80410C8F8082003
:10B48000C8F80C3088F81050CCF8809248F68873D1
:10B49000E358B3FA83F35B0944F2A00202FB0340D2
:10B4A00000F66850FBF7E4FD48F68873E358002B7C
:10B4B00041F04C86079A039DD2F8FC30D2F8000187
:10B4C000049AE11802EB0A0E91F8F4C506EBCE0ED1
:10B4D00044F6086248F69861A350DEF808209EF80A
:10B4E0000CE0655044F60C61B8EEC88A675044F62B
:10B4F0002067904204F59C4181ED048A04F807E03E
:10B5000044F618610746A8BF17468242B8BF0246F4
:10B5100044F61C60675044F6146122501CF0010F81
:10B52000089A625001F0E98704EB4303DFED176AE4
:10B53000B3F82C3507EE903AF8EE677A04F50E432F
:10B5400086EEA77A83ED297A049B534406EBC30663
:10B5500004F59C433069586244F6286201230021B7
:10B56000A1500A931A4644F2A00303FB02430022AF
:10B57000C3F88C2D236923F0020343F001032361F8
:10B58000FEF72CBF282809003ACC012000FEFF4618
:10B590000BF513530BF59C5728331C37029306F118
:10B5A000D8083D46C14655F8043B48F8D43C07F25C
:10B5B000C45729464B4651F8040B43F8040BB835E1
:10B5C0001846B42210F08AFABD4209F58079F0D10C
:10B5D0004FF0010308F8613C0023C8F8E438C8F8CC
:10B5E000E838029BAB4208F65838DAD142F2E8421A
:10B5F00004F188035BF80270029AB2EB030913D0DE
:10B600000BF59C5500221735104615F8013F00F048
:10B610000F0101301A44814503FA01F382EA030263
:10B62000F3D1DFF8A8A49244574500F037814FF0DA
:10B6300000094F464FF0FF3A06EB09054FF00808A6
:10B640003422002105F5D27085F8907185F891714A
:10B6500085F89271C5F8A0A1C5F89471C5F89871E4
:10B6600013F062F80220622301214FF4FA7285F888
:10B67000F4004FF0030E042085F800E1C5F89CA10A
:10B6800085F8DC70C5F8E07085F8DF7085F8E47047
:10B6900085F8E570C5F8EC7085F8EB7085F8F0700A
:10B6A00085F8F170C5F8F87085F8F67085F8F770D0
:10B6B00085F8FC7085F8FD70C5F8047185F8027195
:10B6C00085F8037185F80871C5F8D81085F8DE1083
:10B6D00085F8E81085F8EA1085F8DD3085F8E9305E
:10B6E00085F8F53085F80131A5F8E620A5F8F220B7
:10B6F000A5F8FE204FF0050E85F8097185F80C01BC
:10B70000062085F818E185F824014FF0070E08207F
:10B7100085F830E1A5F80A2185F80D31A5F8162144
:10B7200085F8193185F81A11A5F8222185F82531F7
:10B73000A5F82E2185F8313185F83211C5F8107140
:10B7400085F80E7185F80F7185F8147185F81571FB
:10B75000C5F81C7185F81B7185F8207185F8217179
:10B76000C5F8287185F8267185F8277185F82C7140
:10B7700085F82D71C5F8347185F8337185F8387105
:10B7800085F839714FF0090EA5F83A2185F83C018A
:10B790004FF41C7085F848E1A5F85201A5F85E0148
:10B7A0004FF00B0E0C204FF00A0C85F860E185F885
:10B7B0003D3185F83E11A5F8462185F8493185F8D7
:10B7C0004A1185F8553185F8561185F8613185F8AB
:10B7D0006211A5F86A21C5F8407185F83F7185F8B6
:10B7E000447185F84571C5F84C7185F84B7185F841
:10B7F000507185F85171C5F8587185F8577185F801
:10B800005C7185F85D71C5F8647185F8637185F8C0
:10B81000687185F8697185F854C14FF00D0E85F88F
:10B820006C01B8F101084FF00E0085F86D3185F814
:10B830006E11A5F8762185F8793185F87A11A5F889
:10B84000822185F8853185F88611A5F88E21C5F805
:10B85000707185F86F7185F8747185F87571C5F828
:10B860007C7185F87B7185F8807185F88171C5F8E8
:10B87000887185F8877185F88C7185F88D7185F8E8
:10B8800078E185F8840105F580757FF4D9AE09F675
:10B89000583942F2082399457FF4CEAEDFF830A242
:10B8A000874D884B4FF00008A146DAF80440622C1F
:10B8B00003F2568748F6907202FB083707F54757A0
:10B8C0003C373A78022A29D03A78012A26D0D5F88E
:10B8D0000C28944222D0D5F8342B02932244117CB8
:10B8E000002900F08B804FF40072002105F63830FB
:10B8F00012F01AFF4FF0FF3100220120029BC5F821
:10B900000848C5F8381DC5F83C1DC5F80C18C5F821
:10B91000402DC5F8442DC5F8482D387008F10108B0
:10B9200005F50F45B8F1030F05F190050AF6583AF1
:10B93000BBD142F2102141F22A7201234C467354CA
:10B9400086F87A3086F8D23BB354FEF798BAD4F82A
:10B95000602D04F5356304F538611E685D689868EC
:10B96000DF68D76010338B4216605560906002F13B
:10B970001002F2D11B68136043F2F0435BF803300E
:10B9800023F01003FEF72DBFD4F8602D04F53563C6
:10B9900004F538611E685D689868DF68D760103309
:10B9A0008B4216605560906002F11002F2D11B6864
:10B9B00013604CF280435BF8033023F01003FEF772
:10B9C000DEBF0299D4F8602D01F6084301F6384134
:10B9D0001F685E689868D3F80CE0C2F80CE010337A
:10B9E0008B4217605660906002F11002F0D11B6824
:10B9F00013602B6923F01003FEF778BF40F2446216
:10BA0000284612F091FE6422FF2105F5C87012F05D
:10BA10008BFE2D4BC5F80C4803FB04F201320321C9
:10BA2000C5F80028029B397078E72369DA072FD51B
:10BA300048F6887144F2A0026758A068B7FA87F107
:10BA4000490902FB01F2A61844F6F8559C467559BF
:10BA50006E0006EB050E02EB8E02224444F69C5E5D
:10BA600052F80EE00DE0D0F88430D0F8842050F881
:10BA70002330013202F01F029E45C0F8842002F0FC
:10BA8000ED82D0F88030D0F884209342EBD1634629
:10BA90009F0738D548F6887244F2A001A558A068DF
:10BAA00001FB05F1661844F6F852B6587700BA194A
:10BAB00001EB8201214444F69C5251F802E01BE064
:10BAC000B04EFF1FA81CFF1F28280900FF16FE12FA
:10BAD00004AA012031082C3F00C07F44D0F8841014
:10BAE000D0F8842050F82110013202F01F028E4558
:10BAF000C0F8842002F0ED82D0F88010D0F88420C5
:10BB00009142EBD123695E077EF56CAC48F68871F3
:10BB100044F2A00267585FED116A02FB074202F689
:10BB2000845191ED007AD2F8901D07EE901AF8EE4C
:10BB3000E77A27EE877AB5EEC07AF1EE10FA67EE73
:10BB4000266A42F3128513F0200A02F0DA8402F525
:10BB50005762D2ED007A1FED207A76EEA77A0125A2
:10BB6000C2ED007AB4EEE77AF1EE10FA4CBF012292
:10BB70000022002A02F0B284AA0207EE102A44F240
:10BB8000A006B8EEC77A06FB07F604EB060E77EEC2
:10BB9000C77A0EF5576244F6FC5CC2ED007A5EF897
:10BBA0000C100492294401F007024EF80C205119A0
:10BBB00001F00701084602EB4201DEF8742D039004
:10BBC00006EB810100EB40084FEA850C06EB880686
:10BBD000624444F69C582144CEF8742D51F8081064
:10BBE00026448C4456F808108C4548D0BCF1000F10
:10BBF00045DB46F808C0E34AD4F804801278D8F848
:10BC00008012D8F88402CDF840C0002A01F1010961
:10BC100044F698510CBF0322012209F01F097658FF
:10BC20008DF84C200421002281458DF83C2011968E
:10BC3000129102F05B840FAED8F880C20FCE0CEBED
:10BC40008C0C4FEA8C0C08EB0C0A48F80C0044F6FC
:10BC5000F850CAF8041036780399CAF80820CAF8D0
:10BC60000C308AF81060C8F880924EF800102369F2
:10BC700043F002032361DEF8742D03F0200A44F23E
:10BC8000A00101FB07F104EB010E0EF5576090EDEA
:10BC9000005AFDEEC57A48F68C7C17EE908A1202A7
:10BCA00044F6FC5602EB08005EF80660CEF86C0D18
:10BCB00044F80C00DEF8900D07EE100A0EF6845ED4
:10BCC000DEED007AB8EEC77A700000EB060C27EEC6
:10BCD000277A01EB8C0101F59B41B5EEC07A183152
:10BCE000F1EE10FA214408EB050EC3F2AC8540F2E8
:10BCF000FF3CE64542F39281711901F0070144F2DD
:10BD0000A00501EB410E05FB07F101EB8E0101F5EA
:10BD10009B41183121444FF0000E07EE908AB8EE97
:10BD2000E76A35EE466A44F2A005304405FB07F5A4
:10BD300005EB8000204444F6985C0E6850F80C1027
:10BD400036F90E0031F9181005EE900A06EE901A39
:10BD5000F8EEE55AF8EEE66A611975EEE65A01F575
:10BD60009C40E5EE866A90ED018AB5EEC07AF1EE70
:10BD700010FA26EE888AC4F23581D1F8781DDFEDFD
:10BD8000826A511A07EE901AF8EEE77A77EE857A12
:10BD9000F4EEE67AF1EE10FA42F131819FED7A6A23
:10BDA000DFED7A5A36EE676AF7EE006AE6EE656A0C
:10BDB00028EE268AB5EEC07AF1EE10FA82F21F81E3
:10BDC00044F2A00101FB0747D7F8781D511A07EE8E
:10BDD000901AB8EEE77A77EE057A9FED6B7AF4EE7B
:10BDE000C77AF1EE10FA09D577EE677ADFED676A68
:10BDF000B7EE007AA7EEE67A28EE078ABAF1000FCE
:10BE000001F0338448F6887244F2A003A6589FEDEF
:10BE1000607AB6FA86F6760903FB064303F6845287
:10BE2000D2ED006AD3F8902D07EE902AF8EEE77A6B
:10BE300003F5576367EEA67AF5EEC07AF1EE10FAD5
:10BE400027EE877AD3ED007A43F3128377EE277AD1
:10BE5000DFED506AC3ED007A0125F4EEE76AF1EEFA
:10BE600010FA4CBF01230023002B01F02D84AB02FC
:10BE700006EE903A44F2A007F8EEE66A07FB06F7F2
:10BE800004EB070E77EEE67A44F6FC520EF55760A7
:10BE9000C0ED007A5EF802302B4403F007014EF843
:10BEA000021001EB050A01EB41080AF0070ADEF86F
:10BEB000741D07EB8808AA000AEB4A0307EB83030B
:10BEC00044F69C5C5718A044CEF8747D58F80C10CA
:10BED00023440A4453F80C108A4203F0F484002AE5
:10BEE000C3F2F18443F80C20D4F804802549D8F833
:10BEF00080920F78D8F88412159209F1010944F65E
:10BF0000985C002F09F01F07039753F80C30169325
:10BF1000039B0CBF032701278DF8607004220027C4
:10BF20008B428DF85070179203F0238014AA1746A5
:10BF3000D8F880C20FCF0CEB8C0C4FEA8C0C08EBBE
:10BF40000C0948F80C0044F6F850C9F80C303F785A
:10BF5000039BC9F8082089F81070C9F80410C8F8C4
:10BF600080324EF800A048F688722369A25843F048
:10BF700002032361B2FA82F8DEF8747D4FEA5818A2
:10BF80000AE000BF3ACC012000002043CDCCCC3BDE
:10BF900031082C3F00C07F4444F2A00303FB06F3AA
:10BFA00004EB030C0CF5576292ED005AFDEEC57AD6
:10BFB000390217EE90EA48F68C7744F6FC5001EB14
:10BFC0000E025CF80000CCF86C2DE251DCF8902DEC
:10BFD00007EE102A0CF68457D7ED007AB8EEC77A30
:10BFE000420002EB000C27EE277A03EB8C0303F5EB
:10BFF0009B43B5EEC07A1833F1EE10FA23440EEBF2
:10C000000507C2F2718740F2FF3C674542F3A08307
:10C01000431903F0070344F2A00503EB430705FBB4
:10C0200006F303EB870303F59B43183323440027F0
:10C0300007EE90EAB8EEE76A35EE466A44F2A005EC
:10C04000024405FB06F505EB8202224444F6985CA7
:10C05000186852F80C30C25F33F91E3005EE902A92
:10C0600006EE903AF8EEE55AF8EEE66A631975EED8
:10C07000E65A03F59C42E5EE866AD2ED018AB5EEFA
:10C08000C07AF1EE10FA66EEA88AC1F20A83D3F8FC
:10C09000783D5FED436ACB1A07EE903AF8EEE77A07
:10C0A00077EE857AF4EEE67AF1EE10FA11D51FED0F
:10C0B0004A6A5FED4A5A36EE676AF7EE006AE6EEC4
:10C0C000656A68EEA68AB5EEC07AF1EE10FAC3F2A0
:10C0D000FD8344F2A00303FB0646D6F87C2D521ADA
:10C0E00007EE902AB8EEE77A77EE457A1FED5A7A96
:10C0F000F4EEC77AF1EE10FA09D577EE677A5FEDC4
:10C100005D6AB7EE007AA7EEE67A68EE878A029B50
:10C1100003F6EC0595ED007AB5EEC07AF1EE10FA73
:10C1200042F236871A4603F50F63D3ED007A02F622
:10C13000F40377EEC77A93ED009A17EE100A27EE14
:10C14000899A11F0F5FE44F2A00303FB084404F6BB
:10C150008453D4F8902D93ED006A5FED736A07EE77
:10C16000902AB8EEE77A064667EE067A0F4667EE43
:10C17000A67A69EE288AF0EEE77A17EE900A11F0B7
:10C18000D7FE02460B463046394611F071FD11F0DC
:10C1900023FFF7EE007A37EEC99A2860E9EE088AA5
:10C1A000B0EE688A01F071BA2369DA072FD548F634
:10C1B000887144F2A0026558A168B5FA85F676093F
:10C1C00002FB06F2A71844F6F8503858470007EB70
:10C1D000000E02EB8E02224444F69C5E52F80EC022
:10C1E0009E460DE0D1F88430D1F8842051F82330F8
:10C1F000013202F01F029C45C1F8842001F00A853B
:10C20000D1F88030D1F884209342EBD173469F0758
:10C210002AD548F6887244F2A001A558A06801FB0F
:10C2200005F1661844F6F852B6587700BA1901EBD2
:10C230008201214444F69C5251F802E00DE0D0F80E
:10C240008410D0F8842050F82110013202F01F022F
:10C250008E45C0F8842001F01785D0F88010D0F802
:10C2600084209142EBD123695E077DF541AF48F60A
:10C27000887144F2A00267585FEDBB6A02FB074277
:10C2800002F6845191ED007AD2F8901D07EE901AD3
:10C29000F8EEE77A27EE877AB5EEC07AF1EE10FA7B
:10C2A00067EE266A42F3338213F0200002F0FC812D
:10C2B00002F55762D2ED007A1FEDCA7A76EEA77AC0
:10C2C0000125C2ED007AB4EEE77AF1EE10FA4CBF28
:10C2D00001220022002A02F08A81AA0207EE102A17
:10C2E00044F2A008B8EEC77A08FB07F804EB080E82
:10C2F00077EEC77A0EF5576244F6FC5CC2ED007A21
:10C300005EF80C100492294401F007024EF80C204C
:10C31000511901F007010E4602EB4201DEF8742DBF
:10C32000029608EB81014FEA850C06EB460908EB03
:10C330008909214444F69C586244CEF8742D51F882
:10C340000810A1440CEB010A59F808108A454CD09A
:10C35000BAF1000F49DB49F808A0D4F804C0E54A57
:10C36000DCF880121278DCF88462CDF898A201F132
:10C37000010844F69851002A0CBF0322012259F803
:10C380000110039108F01F088DF8A4220022042157
:10C390008DF89422B045039AA792A89102F02F81BC
:10C3A000A5AB1E46DCF880920FCE09EB89094FEA57
:10C3B00089090CEB090A4CF8090044F6F850CAF850
:10C3C000041036780299CAF80820CAF80C308AF8A6
:10C3D0001060CCF880824EF80010236943F002030D
:10C3E0002361DEF8742D03F0200044F2A00101FB6C
:10C3F00007F104EB010C0CF55766D6ED006AFDEE73
:10C40000E67A48F68C7917EE908A120244F6FC5EC2
:10C4100002EB08065CF80EE0CCF86C6D44F809609D
:10C42000DCF8906D07EE106A0CF6845CDCED007AA7
:10C43000B8EEC77A4FEA4E0606EB0E0927EE277ACA
:10C4400001EB890101F59B41B5EEC07A1831F1EE9F
:10C4500010FA214408EB050CC3F21C8240F2FF39AC
:10C46000CC4542F3A7800EEB050101F0070144F231
:10C47000A00501EB410C05FB07F101EB8C0101F577
:10C480009B4118312144002507EE908AB8EEE76AF7
:10C4900036EEC66A44F2A00C76440CFB07FC0CEBAB
:10C4A0008606264444F69859D1F800E056F809105B
:10C4B0003EF9055031F9181005EE905A07EE901A22
:10C4C000F8EEE55AF8EEE77A04EB0C0175EEE75A60
:10C4D00001F59C45E5EE867A043595ED008AB5EECA
:10C4E000C07AF1EE10FA27EE888AC3F20A81D1F8F9
:10C4F000781D9FED816A511A07EE901AF8EEE77ADF
:10C5000077EEA67AF4EEC67AF1EE10FA42F14380A5
:10C510009FED796ADFED795A36EE676AF7EE007AB9
:10C52000E6EE657A28EE278AB5EEC07AF1EE10FACB
:10C5300082F2318044F2A00101FB0747D7F8781D51
:10C54000511A07EE901AB8EEE77A77EE267A9FED49
:10C550006A7AF4EEC77AF1EE10FA09D577EE677AC7
:10C56000DFED666AB7EE007AA7EEE67A28EE078A74
:10C57000002801F0C78048F6887244F2A003A6584C
:10C580009FED5F7AB6FA86F6760903FB064303F65B
:10C590008452D2ED006AD3F8902D07EE902AF8EE7F
:10C5A000E77A03F5576367EEA67AF5EEC07AF1EE07
:10C5B00010FA27EE877AD3ED007A43F3438377EEC0
:10C5C000277ADFED506AC3ED007A0125F4EEE76AC1
:10C5D000F1EE10FA4CBF01230023002B00F0E88796
:10C5E000AB0206EE903A44F2A001F8EEE66A01FBD7
:10C5F00006F104EB010E77EEE67A44F6FC580EF5F0
:10C60000576CCCED007A5EF80830DEF8742D2B44C0
:10C6100003F0070303EB050A03EB43070AF0070ADD
:10C620004EF8083001EB87074FEA85080AEB4A000D
:10C63000E31901EB80004244414644F69C58CEF891
:10C64000742D204453F8083050F808701944B9424A
:10C6500002F090800029C2F28D8040F80810254B2E
:10C66000D4F804801B78D8F88072D8F88422AB9173
:10C67000002B07F1010944F6985309F01F070297B0
:10C68000C358AC93029B0CBF032701270020042151
:10C6900093428DF8B8728DF8A802AD9103F06481D1
:10C6A000AAAA1746D8F880C20FCF0CEB8C0C4FEA21
:10C6B0008C0C08EB0C0948F80C0044F6F850C9F84B
:10C6C0000C303F78029BC9F80820C9F8041089F89B
:10C6D0001070C8F880324EF800A048F688722369BE
:10C6E000A75843F002032361B7FA87F7DEF8742DE9
:10C6F0007F0909E03ACC012000002043CDCCCC3B9F
:10C7000031082C3F00C07F4444F2A00303FB06FC29
:10C7100004EB0C0303F5576191ED005AFDEEC57A69
:10C7200048F68C7017EE908A110244F6FC5E01EB1D
:10C73000080253F80EE0C3F86C2D2250D3F8902D68
:10C7400007EE102A03F68452D2ED007AB8EEC77ACB
:10C750004FEA4E0000EB0E0327EE277A0CEB830323
:10C7600003F59B43B5EEC07A1833F1EE10FA23447B
:10C7700008EB0502C3F2E38040F2FF3C624543F35D
:10C7800019810EEB050303F0070344F2A00203EB4B
:10C79000430502FB06F303EB850303F59B431833C4
:10C7A0002344002207EE908AB8EEE76A35EE466A27
:10C7B00044F2A005704405FB06F505EB800020441B
:10C7C00044F6985CD3F800E050F80C303EF90220B3
:10C7D00033F9183005EE902A06EE903AF8EEE55A55
:10C7E000F8EEE66A631975EEE65A03F59C42E5EE4B
:10C7F000866AD2ED018AB5EEC07AF1EE10FA66EEE5
:10C80000A88AC0F2C286D3F8783D5FED456ACB1A9C
:10C8100007EE903AF8EEE77A77EE857AF4EEE67A6C
:10C82000F1EE10FA11D51FED4C6A5FED4C5A36EE61
:10C83000676AF7EE006AE6EE656A68EEA68AB5EE0C
:10C84000C07AF1EE10FAC3F2638044F2A00303FB56
:10C850000646D6F87C2D521A07EE902AB8EEE77AF3
:10C8600077EE457A1FED5C7AF4EEC77AF1EE10FAB6
:10C8700009D577EE677A5FED5F6AB7EE007AA7EECB
:10C88000E67A68EE878A04F6340595ED007AB5EE0F
:10C89000C07AF1EE10FA43F2958004F63803D3ED36
:10C8A000007A04F63C0377EEC77A93ED009A17EE10
:10C8B000100A27EE899A11F03BFB44F2A00303FB18
:10C8C000074404F68453D4F8902D93ED006A5FED8D
:10C8D000746A07EE902AB8EEE77A804667EE067A29
:10C8E000894667EEA67A69EE288AF0EEE77A17EEB7
:10C8F000900A11F01DFB02460B464046494611F0D6
:10C90000B7F911F069FBF7EE007A37EEC99A2860A3
:10C91000E9EE088AB0EE688AFDEEC87A17EE902A32
:10C92000A2F50042C2F38D0202F07F04FDF7E3BBE3
:10C930002369DA072FD548F6887144F2A0026758B8
:10C94000A168B7FA87F0400902FB00F2A61844F686
:10C95000F85575596E0006EB050E02EB8E02224467
:10C9600044F69C5E52F80EC09E460DE0D1F884302D
:10C97000D1F8842051F82330013202F01F029C4587
:10C98000C1F8842000F01D86D1F88030D1F88420D1
:10C990009342EBD173469F072AD548F6887244F23A
:10C9A000A001A558A06801FB05F1661844F6F852ED
:10C9B000B6587700BA1901EB8201214444F69C5223
:10C9C00051F802E00DE0D0F88410D0F8842050F83F
:10C9D0002110013202F01F028E45C0F8842000F0C1
:10C9E0002D86D0F88010D0F884209142EBD12369B5
:10C9F0005E077DF550AC48F6887144F2A002675896
:10CA00005FEDC16A02FB074202F6845191ED007AA4
:10CA1000D2F8901D07EE901AF8EEE77A27EE877AA3
:10CA2000B5EEC07AF1EE10FA67EE266A41F326867B
:10CA300013F0200001F0EE8502F55762D2ED007A86
:10CA40001FEDD07A76EEA77A0125C2ED007AB4EE1A
:10CA5000E77AF1EE10FA4CBF01220022002A01F021
:10CA60002A85AA0207EE102A44F2A008B8EEC77A77
:10CA700008FB07F804EB080E77EEC77A0EF557624D
:10CA800044F6FC5CC2ED007A5EF80C100492294476
:10CA900001F007024EF80C20511901F007010E4673
:10CAA00002EB4201DEF8742D029608EB81014FEA99
:10CAB000850C06EB460908EB8909214444F69C588D
:10CAC0006244CEF8742D51F80810A1440CEB010A11
:10CAD00059F808108A454CD0BAF1000F49DB49F8E3
:10CAE00008A0D4F804C0E84ADCF880121278DCF818
:10CAF0008462CDF86CA101F1010844F69851002A36
:10CB00000CBF0322012259F80110039108F01F08FD
:10CB10008DF87821002204218DF86821B045039A10
:10CB20005C925D9101F0CF845AAB1E46DCF8809296
:10CB30000FCE09EB89094FEA89090CEB090A4CF879
:10CB4000090044F6F850CAF8041036780299CAF879
:10CB50000820CAF80C308AF81060CCF880824EF8B1
:10CB60000010236943F002032361DEF8742D03F003
:10CB7000200044F2A00101FB07F104EB010C0CF5CD
:10CB8000576696ED005AFDEEC57A48F68C7917EE99
:10CB9000908A120244F6FC5E02EB08065CF80EE096
:10CBA000CCF86C6D44F80960DCF8906D07EE106A03
:10CBB0000CF6845CDCED007AB8EEC77A4FEA4E06DC
:10CBC00006EB0E0927EE277A01EB890101F59B415F
:10CBD000B5EEC07A1831F1EE10FA214408EB050CDD
:10CBE000C2F2008640F2FF39CC4541F347840EEB98
:10CBF000050101F0070144F2A00501EB410C05FB22
:10CC000007F101EB8C0101F59B41183121444FF0F4
:10CC1000000C07EE908AB8EEE76A35EE466A44F2F9
:10CC2000A00505FB07F5764405EB8606264444F689
:10CC30009859D1F800E056F809103EF90C6031F926
:10CC4000181005EE906A06EE901AF8EEE55AF8EE26
:10CC5000E66A611975EEE65A01F59C45E5EE866ACD
:10CC6000043595ED008AB5EEC07AF1EE10FA26EEA5
:10CC7000888AC2F2A485D1F8781DDFED856A511A41
:10CC800007EE901AF8EEE77A77EE857AF4EEE67A18
:10CC9000F1EE10FA41F1DD839FED7D6ADFED7D5A03
:10CCA00036EE676AF7EE006AE6EE656A28EE268AD7
:10CCB000B5EEC07AF1EE10FA81F2CB8344F2A00116
:10CCC00001FB0747D7F8781D511A07EE901AB8EE06
:10CCD000E77A77EE057A9FED6E7AF4EEC77AF1EE99
:10CCE00010FA09D577EE677ADFED6A6AB7EE007A57
:10CCF000A7EEE67A28EE078A002800F0118448F6AD
:10CD0000887244F2A003A6589FED637AB6FA86F6BD
:10CD1000760903FB064303F68452D2ED006AD3F88A
:10CD2000902D07EE902AF8EEE77A03F5576367EE49
:10CD3000A67AF5EEC07AF1EE10FA27EE877AD3EDF7
:10CD4000007A42F3D28577EE277ADFED506AC3EDA1
:10CD5000007A0125F4EEE76AF1EE10FA4CBF0123E8
:10CD60000023002B00F00984AB0206EE903A44F257
:10CD7000A001F8EEE66A01FB06F104EB010E77EE86
:10CD8000E67A44F6FC580EF55767C7ED007A5EF870
:10CD90000830DEF8742D2B4403F0070303EB050A7B
:10CDA00003EB430C4EF8083001EB8C0C4FEA85087E
:10CDB0000AF0070A04EB0C030AEB4A0044F69C5CF9
:10CDC000424401EB8000CEF8742D53F80C3020441F
:10CDD0004146194450F80C30994201F07D860029F3
:10CDE000C1F27A8640F80C10274BD4F804801B78E7
:10CDF000D8F88092D8F884220392002B44F69853F6
:10CE000009F1010909F01F02C35861930292134608
:10CE1000039A60910CBF4FF0030C4FF0010C0020FF
:10CE2000042193428DF88CC18DF87C01629101F050
:10CE300048865FAFD8F880C20FCF0CEB8C0C4FEA5E
:10CE40008C0C08EB0C0948F80C0044F6F850C9F8B3
:10CE50000C303F78029BC9F80820C9F8041089F803
:10CE60001070C8F880324EF800A048F68872236926
:10CE7000A25843F002032361B2FA82F8DEF8742D5F
:10CE80004FEA58180CE000BF3ACC012000C07F44A4
:10CE900000002043CDCCCC3B31082C3F00FEFF46A8
:10CEA00044F2A00303FB06FC04EB0C0303F55761FB
:10CEB00091ED005AFDEEC57A48F68C7017EE90EAB7
:10CEC000110244F6FC5701EB0E02DF59C3F86C2D3A
:10CED0002250D3F8902D07EE102A03F68452D2ED9B
:10CEE000007AB8EEC77A7800C31927EE277A0CEBE0
:10CEF000830303F59B43B5EEC07A1833F1EE10FAC5
:10CF000023440EEB0502C1F2DA8740F2FF3C624592
:10CF100041F327847B1903F0070344F2A00203EBDB
:10CF2000430502FB06F303EB850303F59B4318332C
:10CF30002344002207EE90EAB8EEE76A35EE466A2F
:10CF400044F2A005384405FB06F505EB80002044BB
:10CF500044F6985C1F6850F80C30BA5E33F91E3006
:10CF600005EE902A06EE903AF8EEE55AF8EEE66AFB
:10CF7000631975EEE65A03F59C42E5EE866AD2ED3A
:10CF8000018AB5EEC07AF1EE10FA66EEA88AC0F218
:10CF9000E282D3F8783D5FED426ACB1A07EE903A11
:10CFA000F8EEE77A77EE857AF4EEE67AF1EE10FAAB
:10CFB00011D51FED496A5FED495A36EE676AF7EE03
:10CFC000006AE6EE656A68EEA68AB5EEC07AF1EE12
:10CFD00010FAC1F2E58344F2A00303FB0646D6F83B
:10CFE0007C2D521A07EE902AB8EEE77A77EE457A52
:10CFF0001FED597AF4EEC77AF1EE10FA09D577EE03
:10D00000677A5FED5C6AB7EE007AA7EEE67A68EEC3
:10D01000878A04F6340595ED007AB5EEC07AF1EE14
:10D0200010FA41F2AA8304F63803D3ED007A04F62D
:10D030003C0377EEC77A93ED009A17EE100A27EEBD
:10D04000899A10F075FF44F2A00303FB084404F62C
:10D050008453D4F8902D93ED006A5FED716A07EE6A
:10D06000902AB8EEE77A064667EE067A0F4667EE34
:10D07000A67A69EE288AF0EEE77A17EE900A10F0A9
:10D0800057FF02460B463046394610F0F1FD10F0CE
:10D09000A3FFF7EE007A37EEC99A2860E9EE088A16
:10D0A000B0EE688A4BE20299049B0698039D4BF60A
:10D0B0006C720B4407EBC30381581E7BC4F8681DD8
:10D0C0004BF6707244F6F85E82589868C4F86C8D1E
:10D0D0006318B8EEC88A44F80E5093F8F435089DEA
:10D0E000904204F5576E8EED008A8646A8BF96469C
:10D0F0008242B8BF0246DB07C4F8745D84F8806DD5
:10D10000C4F878EDC4F87C2D40F1FF8104EB4103B5
:10D110005FED9E6AB3F82C3507EE903AF8EE677A29
:10D1200004F59C4386EEA77A83ED017A029A049B6C
:10D13000134407EBC3071D4604F68453396919608D
:10D140000022C4F8882D099AFDF7F5BE079A0499C4
:10D15000D2F8FC30D2F800210398C4F8683D01EB06
:10D160000A05E11806EBC50591F8F4E5C4F86C7DF5
:10D1700044F6F857A9682D7BE0510298B8EEC88AAA
:10D1800000F62867914287ED008A0F46A8BF174630
:10D190008A42B8BF0A460898C4F8740D1EF0010F01
:10D1A00084F8805DC4F8787DC4F87C2D00F08D8112
:10D1B00004EB43035FEDC76AB3F82C3507EE903AF2
:10D1C000F8EE677A04F59C4386EEA77A83ED017A40
:10D1D000049B534406EBC306029B316903F63C6390
:10D1E00000221960C4F8882D0A9AFEF7BCB948F6E7
:10D1F000887344F2A002E358DFF800E5B3FA83F342
:10D200005B0902FB03420D4644F69C5044F6A051D4
:10D21000043D15504FF001005054D4F804C09EF85E
:10D220000010DCF88082069144F69850002908F13D
:10D23000010101F01F011258DCF884E2489208460F
:10D240004FF0040214BF01210321499270454FF0B1
:10D25000000247958DF828118DF81821099000F0EB
:10D26000D084DCF880E246AD0FCD0EEB8E0E4FEA97
:10D270008E0E0CEB0E084CF80E002D78C8F804103A
:10D280000120C8F80C300999C8F80820022388F852
:10D2900010500390CCF880120B930146FEF751B862
:10D2A00048F688730D46E258DFF85084B2FA82F3EC
:10D2B00044F2A0015B0901FB034144F69C5E44F685
:10D2C000A050A5F1040C4FF0010541F80EC00D541B
:10D2D00098F80000D4F804E007900546CDF874C330
:10D2E000DEF88002DEF8848244F6985C013051F862
:10D2F0000C10DE91002D00F01F010D4614BF01211E
:10D30000032100208DF8801345454FF004018DF86E
:10D310007003DF9100F0E181DEF880920DF55C781A
:10D32000B8E80F0009EB89094FEA89090EEB090CEF
:10D330004EF8090098F80080CCF80C300120022348
:10D34000CCF80410CCF808208CF810800390CEF8AC
:10D3500080520A93069DFDF751BE48F6887344F249
:10D36000A002E358DFF894E3B3FA83F35B090D46B8
:10D3700002FB034244F69C502E1F44F6A051165067
:10D380004FF0010050549EF80010D4F804C00791EB
:10D390000D46DCF88012DCF884E2929644F6985050
:10D3A000013101F01F0112589392002D4FF0040239
:10D3B0000D46949214BF01210321002275458DF87A
:10D3C00054128DF8442200F01584DCF880E291AE0E
:10D3D0000FCE0EEB8E0E4FEA8E0E0CEB0E0A4CF8B3
:10D3E0000E003678CAF80C3001200223CAF8041067
:10D3F000CAF808208AF8106003900A93CCF880528B
:10D400000146FDF784BC029D049A42F6DC712A4471
:10D41000059D6958039D255006EBC202059DD2F873
:10D4200008C0127B42F6E07004EB010E28589EF80B
:10D43000F4E5C4F86C7D84456746A8BF074660459F
:10D44000B8BF6046089DC4F8681D04F5576C1EF00F
:10D45000010FCCED007AC4F8787DC4F8745DC3F890
:10D460007C0D84F8802D56D004EB4103DFED9E6ADD
:10D47000B3F82C3507EE903AF8EE677A04F59C4342
:10D4800086EEA77A83ED017A029A049B134406EB99
:10D49000C3061D4604F68453316919600022C4F89E
:10D4A000882D099AFDF7F1BE5746FDF77CBDC846A9
:10D4B000FDF704BC4F46FDF71EBF04F50E434FF0C9
:10D4C0007E52C3F8A420FDF725BD04F59C434FF020
:10D4D0007E525A607CE6E258B2FA82F3F8EEE77ABE
:10D4E0005B09FDF73FBEF8EEE77AFDF73BBE04F5BA
:10D4F0000E43C3F8A4A0FDF7B7BE04F50E434FF0EA
:10D500007E52C3F8A420FEF71FB804F59C434FF0E9
:10D510007E525A600AE604F59C43C3F804A0B3E7C0
:10D5200048F6887144F2A002655802FB054292F861
:10D53000801D012901F0C883022901F0FB82FDEE64
:10D54000C87A17EE902AA2F50042C2F38D0202F0CB
:10D550007F04FCF7A3BED3F87C3DDFED646A5B1A61
:10D5600007EE903AF8EEE77A77EEC57AF4EEE67ACF
:10D57000F1EE10FA7FF529AD1BE544F2A00303FBA1
:10D580000643B046D3F8742D8AE4D3F87C3DDFED32
:10D59000576A5B1A07EE903AF8EEE77A77EEC57AAB
:10D5A000F4EEE67AF1EE10FA7FF549A9FFF73BB900
:10D5B00044F2A00303FB06433746D3F8742DFFF76C
:10D5C000A3B87346002F40F00D8348F6986148F6E3
:10D5D0009C626158A150012744F2A001721901FB1D
:10D5E00000F144F2A00505FB074744F6F85601EBAD
:10D5F0008202224444F6A0554FF0FF3E47F806E071
:10D600004FF0020C23F0010613F0040302F805C0EA
:10D610000293266100F04A8104F6340104F63802D0
:10D6200004F63C033248334D086046F02006106093
:10D630001D6046F004032361FFF7ADB944F2A00179
:10D6400001FB05F1BA1901EB820244F6F8552144B9
:10D65000224444F6A0504FF0FF364E5123F002030F
:10D66000022111542361FFF7C3B948F6887144F2CF
:10D67000A00254F801E002FB0E4292F8801D01293D
:10D6800001F02D87022901F02B86FDEEC87A17EEF6
:10D69000902AA2F50042C2F38D0202F07F04FCF74B
:10D6A000A4BED3F87C3DDFED116A5B1A07EE903A19
:10D6B000F8EEE77A77EEC57AF4EEE67AF1EE10FA54
:10D6C0007EF501ADFEF7F3BC44F2A00303FB064375
:10D6D000B046D3F8747DFEF75FBC4FF0FF31DFED4D
:10D6E000067A0391FDF73EBD00FEFF460000204391
:10D6F0000000A041CDCC4C3D000000003ACC012000
:10D700000040204448F6887144F2A002665802FBAB
:10D71000064292F8801D012902F0AF8102297FF4B0
:10D72000FBA8D2F8905DD2F8741D07EE905A02F66D
:10D730008450F8EEE77A90ED007A67EE877A090276
:10D74000F5EEC07AF1EE10FAC2F28881D2F87C0DC3
:10D75000411A07EE901A02F55762B8EEE77AD2ED59
:10D76000007A77EE677A1FED1A7AF4EEC77AF1EE57
:10D7700010FA3FF6D1A859077FF5CEA8B6FA86F180
:10D78000490944F2A00202FB014202F68450D2F899
:10D79000903D5B4207EE903AC2F8903D90ED007AE2
:10D7A000F8EEE77AAFAD67EE877AF5EEC07AF1EE84
:10D7B00010FAACBFD2F8783DD2F87C3D44F2A0021A
:10D7C00002FB01414FF0FF32C1F86C3D0023D4F859
:10D7D00024082B60B493B992BE92002E42F03A8195
:10D7E00044F608620123A15844F2A00606FB034355
:10D7F000B9AFD3F86C2D009748F688772B46F8F729
:10D8000045FBE359D4F82408002B0CBF3346002312
:10D810002344BEAAD3F8681D0092B4AB0022F8F7E7
:10D8200035FB2968B49BE659C91A002E42F00781DE
:10D83000DDEDB97AF8EEE77A04F59C43C3ED047A9E
:10D84000012344F2A00202FB034303F6845090ED4F
:10D85000007AD3F8900D134D07EE900AF8EEE77AB0
:10D8600067EE877AF5EEC07AF1EE10FAACBF0020D1
:10D870000720002E18BF002244F6FC56224498517F
:10D88000C2F8741D2369084904F6340604F638000A
:10D8900004F63C0243F0200323613560056011600B
:10D8A000FFF73AB800002044CDCCCC3A48F688794E
:10D8B000214444F8090091F8803D002B3FF4B9AEB3
:10D8C000D1F8683DD1F8782DD1F87C1DD4F8240822
:10D8D00005910DF5E6786EAF19460493009743461F
:10D8E000CDF8B8E1CDF8CCE1F8F7D0FA54F809302A
:10D8F000D8F80000C64E039644F2A00E002B18BFC5
:10D900004FF0000E7346234444F69C524FF0010E34
:10D91000985003F805E00425D4F804C08A95DCF893
:10D92000802236789DF808508DF81C5244F69851A4
:10D9300001325958DCF884328991002E02F01F051B
:10D940000CBF032101219D42069088908DF82C1276
:10D95000079500F045810DF5077E75460FCDDCF883
:10D9600080E20EEB8E0E4FEA8E0E0CEB0E0A4CF898
:10D970000E00CAF80410CAF80820CAF80C302B7838
:10D980008AF8103054F80930079DCCF8805244F2E0
:10D99000A005002B18BF00252B46069A234444F609
:10D9A000A850043244F6AC511A504FF001005854BC
:10D9B0000420D4F804C08590C8F80020DCF8801258
:10D9C0009DF80800DCF884528DF8080244F6A45053
:10D9D00001311B588493002E01F01F000CBF03235C
:10D9E0000123A842064683928DF8183200F0F88091
:10D9F00082AD0FCDDCF880E20EEB8E0E4FEA8E0E7C
:10DA00000CEB0E0A4CF80E00CAF80410CAF80820F5
:10DA1000CAF80C302B788AF81030D4F82408059A0C
:10DA2000CCF88062049900974346F8F72FFA039ADE
:10DA300054F809301278D8F800A0CDF8F8A11546AE
:10DA400044F2A002002B18BF00221346234444F6E0
:10DA5000F05144F6F45243F801A04FF001019954FB
:10DA600067680395D7F88002D7F8841244F6EC5221
:10DA700000F1010E9B589DF808007F93002D0EF0D9
:10DA80001F0E0CBF032301238DF8F4018E454FF0C8
:10DA9000040080908DF8043200F0A2807DAB1D461A
:10DAA000D7F880620FCD06EB8606B60007EB060CB2
:10DAB000B8512878CCF80410CCF808208CF8100065
:10DAC000CCF80C3054F80930C7F880E244F2A001D9
:10DAD000002B18BF00210B46234444F6E450AAF162
:10DAE000040244F6E8511A504FF001005854676898
:10DAF000C8F80020D7F88012039ED7F884027992E4
:10DB000044F6E05501315B597A93002E01F01F0E67
:10DB10000CBF032301239DF808108DF8E0110422A7
:10DB200086457B928DF8F0315AD078ADD7F8806277
:10DB30000FCD06EB8606B60007EB060CB851287829
:10DB4000CCF80C30CCF80410CCF808208CF810007D
:10DB500054F80900C7F880E244F2A003002818BF77
:10DB6000002303F668502044F9F782FA54F809506C
:10DB7000002D41F03B8748F698620626D4F8680DE0
:10DB8000A65044F6086144F6206394F8802D605056
:10DB9000E25404F59C435A6804F50E43C3F8A420EC
:10DBA00004F6845393E8070004F59C43243383E888
:10DBB000070044F61861D4F8780DD4F87C2D605035
:10DBC00044F61C630121E25002910A4644F2A0038C
:10DBD00003FB054503FB0243D5F8902DC3F8902DB8
:10DBE000266926E544F6F85144F6FC526158A150E6
:10DBF0000027F1E44FF0FF31039108EE102AFDF702
:10DC00002FB94FF0FF31039108EE102AFDF744BC05
:10DC10003ACC01207346002D40F0E88148F6986127
:10DC200048F69C626158A1504FF0010E44F2A005E5
:10DC30003A1805FB06F144F6F85001EB820205FBA9
:10DC40000E4E224444F6A0584FF0FF3C4EF800C060
:10DC5000022723F0010013F0040302F80870029376
:10DC600020612DD004F6340104F6380204F63C039A
:10DC7000114D124E0D6040F0200015601E6040F006
:10DC800004032361FEF7C3BA44F2A00101FB05F1CE
:10DC9000BA1901EB820244F6F8552144224444F6B5
:10DCA000A0504FF0FF364E5123F0020302211154D1
:10DCB0002361FEF7D9BA00BF0000A041CDCC4C3D96
:10DCC00048F688772144E65191F8803D002BD6D064
:10DCD000D1F8683DD1F8782DD4F82408CDF8E4C205
:10DCE0000DF5707A1E464AF8C8CDD1F87C3D0496F1
:10DCF0003146B9AE059300965346F8F7C7F8E35995
:10DD0000D54EBE980690002B0CBF2B460023314603
:10DD100023449DF808608DF8486344F69C524FF008
:10DD20000106985003F808600426D4F80480D596BC
:10DD3000D8F8802203910978D39044F698500029AE
:10DD40000E4602F10102D8F884121B58D49302F057
:10DD50001F0E73460CBF032301238E458DF85833E5
:10DD6000CDF81CE000F040810DF5527ED8F880C25D
:10DD7000BEE80F000CEB8C0C4FEA8C0C08EB0C0986
:10DD800048F80C00C9F80410C9F80820C9F80C308C
:10DD90009EF8003089F81030E359079A0698C8F8C1
:10DDA0008022002B0CBF2B460023234444F6A851AD
:10DDB00044F6AC5204304FF0010E585003F802E024
:10DDC0000422D4F80480BE90D092D8F88022D8F8EB
:10DDD0008412CE9044F6A45001321B589DF80800DE
:10DDE0008DF83403002E02F01F000CBF0322012225
:10DDF00088420646CF938DF8442300F0F5800DF558
:10DE00004D7EBEE80F00D8F880C20CEB8C0C4FEAB8
:10DE10008C0C08EB0C0948F80C00C9F80410C9F880
:10DE20000820C9F80C309EF8003089F81030D4F87A
:10DE30002408C8F88062B9AE5346059A0499009642
:10DE4000F8F724F8E359039ADDF8F8E292F800A015
:10DE50009DF808208DF82023002B0CBF2B460023B3
:10DE6000234444F6F05144F6F45243F801E04FF0F5
:10DE700001019954D4F80480CDF824E3D8F8800245
:10DE8000042244F6EC51CB9200F10109D8F8842227
:10DE90005B58CA93BAF1000F09F01F090CBF0323A6
:10DEA000012391458DF8303300F09E809DF80830B5
:10DEB000D8F880628DF80C330DF5487CBCE80F0073
:10DEC00006EB8606B6009CF800C048F806004644FB
:10DED000AEF104007160B260F36086F810C0E359DF
:10DEE000C8F88092002B0CBF2B460023234444F635
:10DEF000E45144F6E85258504FF001019954D4F8D7
:10DF000004C0BE90DCF88012C490013144F6E050A9
:10DF1000DCF884221B58C593BAF1000F01F01F08EA
:10DF20004FF004000CBF032101219045C6908DF8ED
:10DF30001C1359D0C3AEDCF880E20FCE0EEB8E0E70
:10DF40004FEA8E0E0CEB0E094CF80E003078C9F833
:10DF50000410C9F80820C9F80C3089F81000E059FD
:10DF6000CCF8808200280CBF2846002000F66850BC
:10DF70002044F9F77DF8E659002E41F03C8648F63A
:10DF800098620625D4F8680DA55044F6086144F659
:10DF9000206394F8802D6050E25404F59C435A6845
:10DFA00004F50E43C3F8A42004F6845393E8070055
:10DFB00004F59C43243383E8070044F61861D4F841
:10DFC000780DD4F87C2D605044F61C630121E2509A
:10DFD00002910A4644F2A00303FB064603FB0243F8
:10DFE000D6F8902DC3F8902D206948E644F6F851F4
:10DFF00044F6FC526158A1504FF0000E16E644F270
:10E00000A00101FB0747D7F87C0D801A07EE900AA4
:10E01000B8EEE77A77EE457AFDF7DFBEB5EEC07A67
:10E02000F1EE10FA41F1C783E645C1F2B1834FEA40
:10E030004E0EB5EEC07AF1EE10FABDF66EAE07EEFA
:10E04000908AB8EEE76AF7EE006A35EE466A36EE79
:10E05000C66AFDF768BE00BF3ACC01206346002FB8
:10E0600040F0EF8148F6986048F69C622058A05036
:10E07000012744F2A002701902FB01F244F2A0054C
:10E0800005FB074502EB800044F6F85C204444F6AB
:10E09000A0574FF0FF3E45F80CE0022623F00105A3
:10E0A00013F00403C655049325612DD0029E144934
:10E0B000144806F6EC0306F50F62196006F6F40341
:10E0C000116045F02005186045F004032361FDF759
:10E0D000DFBC44F2A00101FB05F5BA1905EB820291
:10E0E00044F6F8502544224444F6A0514FF0FF3640
:10E0F0002E5023F00203022050542361FDF703BD8C
:10E100000000A041CDCC4C3D48F68879A31844F8D6
:10E11000091093F8802D002AD6D0D3F8682DD4F8B2
:10E120002408CDF88CE0114628ADD3F8782DD3F82B
:10E130007C3D06930DF18C0A2B46CDF800A005918D
:10E14000CDF8A0E0F7F7A2FE54F809302868C84ED1
:10E15000039644F2A00E002B18BF4FF0000E73463A
:10E16000234444F69C524FF0010E985003F807E008
:10E170000427D4F804C03F97DCF8802236789DF855
:10E1800010708DF8F07044F6985101325958DCF84F
:10E1900084323E91002E02F01F070CBF03210121A3
:10E1A0009F4207903D908DF80011089700F047813D
:10E1B0000DF1F00E77460FCFDCF880E20EEB8E0EFD
:10E1C0004FEA8E0E0CEB0E084CF80E00C8F8041047
:10E1D000C8F80820C8F80C303B7888F8103054F89C
:10E1E0000930089FCCF8807244F2A007002B18BFBA
:10E1F00000273B46079A234444F6A850043244F6CD
:10E20000AC511A504FF0010058540420D4F804C007
:10E210003A902A60DCF880129DF81000DCF88472D5
:10E220008DF8DC0044F6A45001311B583993002EC0
:10E2300001F01F000CBF03230123B84206463892A9
:10E240008DF8EC3000F0FB8037AF0FCFDCF880E2C8
:10E250000EEB8E0E4FEA8E0E0CEB0E084CF80E00F5
:10E26000C8F80410C8F80820C8F80C303B7888F8C3
:10E270001030D4F82408069ACCF880620599CDF8BD
:10E2800000A02B46F7F702FE039A54F809301278E3
:10E29000D5F80080CDF8CC80164644F2A002002BC1
:10E2A00018BF00221346234444F6F05144F6F452BA
:10E2B00043F801804FF001019954D4F804E003962B
:10E2C000DEF88002DEF8841244F6EC5200F1010A16
:10E2D0009B589DF810003493002E0AF01F0A0CBFC3
:10E2E000032301238DF8C8008A454FF004003590C0
:10E2F0008DF8D83000F0A38032AB1E46DEF8807275
:10E300000FCE07EB8707BF000EEB070C4EF8070098
:10E310003078CCF80410CCF808208CF81000CCF839
:10E320000C3054F80930CEF880A244F2A001002B42
:10E3300018BF00210B46234444F6E450A8F1040220
:10E3400044F6E8511A504FF00100585467682A60AB
:10E35000D7F88012039ED7F884022E9244F6E05537
:10E3600001315B592F93002E01F01F0E0CBF0323C8
:10E3700001239DF810108DF8B410042286453092C8
:10E380008DF8C4305BD02DADD7F880620FCD06EB91
:10E390008606B60007EB060CB8512878CCF80C308E
:10E3A000CCF80410CCF808208CF8100054F80900C0
:10E3B000C7F880E244F2A003002818BF002303F648
:10E3C00068502044F8F754FE54F80950002D41F0ED
:10E3D000108248F698620626D4F8681DA65044F6C6
:10E3E000086044F6206394F8802D2150E25404F52F
:10E3F0009C435A6804F50E43C3F8A420029B03F61D
:10E400003C6393E8070004F59C43243383E807004A
:10E4100044F61860D4F8781DD4F87C2D215044F6C9
:10E420001C630121E25004910A4644F2A00303FB5D
:10E43000054503FB0243D5F8902DC3F8902D2569BF
:10E4400042E644F6F85044F6FC522058A05000270B
:10E450000FE644F2A00101FB0747D7F87C5DAD1A37
:10E4600007EE905AB8EEE77A77EE457AFEF733BCBE
:10E470003ACC01200000000000C07F44B5EEC07A15
:10E48000F1EE10FA41F10282CC45C1F2EB814FEA84
:10E490004C0CB5EEC07AF1EE10FABEF6BAAB07EE50
:10E4A000908AB8EEE76AF7EE006A35EE466A36EE15
:10E4B000C66AFEF7B4BB44F2A00202FB0742D2F8E0
:10E4C000742DFEF756BB0499D1ED007A77EEE66A1B
:10E4D000C1ED006ADEF8742DFEF74BBB44F2A002DA
:10E4E00002FB0742D2F8742DFDF7C9BB0499D1EDA8
:10E4F000007A77EEE66AC1ED006ADEF8742DFDF76A
:10E50000BEBBD2F86C1D012544F2A00202FB0742FB
:10E51000D2F87C2D8A42CCBF0021012179B148F686
:10E520008C7123F024034FF0FF300322236103F0AA
:10E53000200A60501FED318A2273FDF75FBC44F260
:10E54000A00202FB074202F55762D2ED007AB5EE57
:10E55000C07A76EEA77AF1EE10FAC2ED007AC1F237
:10E56000C6801FED3B7AFDF7FDBA4CBF4FF0FF357B
:10E57000002513F0200AE2D1B5EEC07AF1EE10FAD0
:10E58000D2F86C1DC0DAD2F8782DC3DA9142CCBF34
:10E5900000210121C2E744F2A00101FB0747D7F89F
:10E5A0007C5DAD1A07EE905AB8EEE77A77EE667AA0
:10E5B000FDF7CDBFB5EEC07AF1EE10FA41F1CC8097
:10E5C000CC45C1F2B5804FEA4C05B5EEC07AF1EE0C
:10E5D00010FABDF659AF07EE908AB8EEE76AF7EE8B
:10E5E000007A36EEC66A37EEC66AFDF753BF44F2CC
:10E5F000A00202FB0742D2F8742DFDF7F6BE049983
:10E60000D1ED007A77EEE66AC1ED006ADEF8742D8E
:10E61000FDF7EBBED2F86C1D012544F2A00202FB0F
:10E620000742D2F87C2D8A42CCBF0021012179B16A
:10E6300048F68C7123F024034FF0FF350322236149
:10E6400003F0200065501FED758A2273FEF754BB5E
:10E6500044F2A00202FB074202F55762D2ED007AB3
:10E66000B5EEC07A76EEA77AF1EE10FAC2ED007A36
:10E67000C1F217811FED807AFEF7E9B94CBF4FF068
:10E68000FF35002513F02000E2D1B5EEC07AF1EE9F
:10E6900010FAD2F86C1DC0DAD2F8782DC3DA9142A4
:10E6A000CCBF00210121C2E7D2F86C1D012544F244
:10E6B000A00202FB0742D2F87C2D8A42CCBF002187
:10E6C000012179B148F68C7123F024034FF0FF3516
:10E6D0000322236103F0200065501FED9A8A227304
:10E6E000FDF746BF44F2A00202FB074202F5576263
:10E6F000D2ED007AB5EEC07A76EEA77AF1EE10FA96
:10E70000C2ED007A19DB1FEDA47AFDF7DCBD4CBF2A
:10E710004FF0FF35002513F02000E3D1B5EEC07AAD
:10E72000F1EE10FAD2F86C1DC1DAD2F8782DC4DA05
:10E730009142CCBF00210121C3E780F23C84F5EE79
:10E74000C07AF1EE10FA4CBF01220022FDF7C2BDE3
:10E75000B5EEC07AF1EE10FA00F1CA837F00FDF742
:10E7600067BCB5EEC07AF1EE10FA00F1D883520022
:10E77000FEF7E0BB3746FDF7C7BF236948F6887749
:10E7800044F2A00A44F8078023F020030AFB08485B
:10E79000236198F8803D93B9B0EE688AFEF7CFBE4A
:10E7A00044F2A00303FB0646D6F8783DCB1A07EEE9
:10E7B000903AB8EEE77A77EE057AFEF719BCD8F80A
:10E7C000683DD8F87C1D049150ADC549D8F8782D26
:10E7D000D4F82408039155AE1946029300953346A8
:10E7E0004FF0FF3550955595F7F750FBE3590398D7
:10E7F000DDF854910078CDF8D091002B0CBF534632
:10E800000023234444F69C5144F6A05206464FF0A0
:10E81000010043F8019098540420D4F804C0769085
:10E82000DCF88022DCF8840244F6985101325B580F
:10E830007593002E02F01F050CBF032301234FF038
:10E84000000E85428DF8DC318DF8CCE10595A3D022
:10E8500073A80546DCF880E20FCD0EEB8E0E4FEA72
:10E860008E0E0CEB0E084CF80E00C8F80410C8F819
:10E870000820C8F80C302B7888F81030E359059D33
:10E88000CCF88052002B0CBF53460023234444F69F
:10E89000A85009F1040244F6AC511A504FF001009F
:10E8A00058540420D4F804C071905592DCF88012BA
:10E8B000DCF884526F924FF000008DF8B80144F6F6
:10E8C000A45001311B587093002E01F01F080CBF9B
:10E8D00003230123A8458DF8C8313FF45DAF6EAD29
:10E8E0000FCDDCF880E20EEB8E0E4FEA8E0E0CEBB5
:10E8F0000E094CF80E00C9F80410C9F80820C9F830
:10E900000C302B7889F8103050ABD4F82408049AD6
:10E91000CCF880820299009355ABF7F7B7FAE35928
:10E92000039ADDF854E11278002B0CBF5346002304
:10E93000234444F6F051154644F6F45243F801E0FE
:10E940004FF0010199540422D4F804C06C92DCF811
:10E950008002DCF8842202954FF000018DF8A411AA
:10E9600044F6EC5100F101085B586B93002D08F060
:10E970001F080CBF032301239045CDF8A8E18DF8B3
:10E98000B4313FF409AF69AB1D46DCF880620FCDAE
:10E9900006EB8606B6000CEB06094CF80600C9F833
:10E9A0000410C9F80820C9F80C302B7889F8103009
:10E9B000E359CCF88082002B0CBF5346002323443C
:10E9C00044F6E450AEF1040244F6E8511A504FF018
:10E9D000010058540421D4F804C055926791DCF822
:10E9E0008052029EDCF8841265924FF000008DF890
:10E9F000900144F6E05005F101081B586693002E83
:10EA000008F01F080CBF0323012388458DF8A031AF
:10EA10003FF4C2AE64AD0FCDDCF8806206EB860633
:10EA2000B6000CEB060E4CF80600CEF80410CEF83B
:10EA30000820CEF80C302B788EF81030E059CCF846
:10EA4000808200280CBF5046002000F66850204409
:10EA5000F8F70EFBE559002D46D148F698620626D8
:10EA6000D4F8680DA65044F6086144F6206394F883
:10EA7000802D6050E25404F59C435A6804F50E431F
:10EA8000C3F8A42004F6845393E8070004F59C43DC
:10EA9000243383E8070044F6186344F61C62D4F874
:10EAA000780DD4F87C1DE050A150012344F2A0025F
:10EAB00002FB054502FB0343D5F8902DC3F8902DCA
:10EAC0006AE6D7ED007A37EEC77AB04687ED007A6E
:10EAD000DEF8742DFEF7E4B9B046FEF7E1B900BFE9
:10EAE0003ACC01200040204444F6F8530622E2507C
:10EAF0000AFB0546D6F8683DC4F8683D96F8803DA7
:10EB000084F8803D06F59C435A6804F59C435A609E
:10EB100006F6845393E8070004F6845383E807005D
:10EB2000D6F8783DC4F8783DD6F87C3DC4F87C3DF5
:10EB30000023BBE7D2F8906DD2F8741D07EE906AFF
:10EB400002F68450F8EEE77A90ED007A67EE877A65
:10EB50000902F5EEC07AF1EE10FAC0F2A281D2F805
:10EB60007C0D411A07EE901A02F55762B8EEE77A6B
:10EB7000D2ED007A77EE677A1FED267AF4EEC77A47
:10EB8000F1EE10FA3EF6DBAC59077EF5D8ACB5FADB
:10EB900085F1490944F2A00202FB014202F68450C9
:10EBA000D2F8903D5B4207EE903AC2F8903D90ED6E
:10EBB000007AF8EEE77A64AE67EE877A0DF5D279DF
:10EBC000F5EEC07AF1EE10FAACBFD2F8783DD2F88B
:10EBD0007C3D44F2A00202FB01416EAF0DF5E678E8
:10EBE000C1F86C3D4FF0FF320023D4F824083360A5
:10EBF000C9F800303A60C8F80020002D40F04E817E
:10EC000044F608620123A15844F2A00505FB034322
:10EC100048F6887AD3F86C2D00973346F7F736F923
:10EC200054F80A30D4F82408002B0CBF2B460023DC
:10EC300023440022D3F8681DCDF800804B46F7F737
:10EC400025F93168D9F8003054F80A50C91A002D56
:10EC500040F0FF80D7ED007AF8EEE77A04F59C43A8
:10EC6000C3ED047A012344F2A00202FB034303F63E
:10EC7000845090ED007AD3F8900DD14E07EE900AB3
:10EC8000F8EEE77A67EE877AF5EEC07AF1EE10FAE1
:10EC9000ACBF00200720002D18BF002244F6FC5511
:10ECA00022445851C2F8741D2369C64904F634053C
:10ECB00004F6380004F63C0243F0200323612E6082
:10ECC00006601160FEF73BBCD2F8906DD2F8741D5F
:10ECD00007EE906A02F68450F8EEE77A90ED007A3B
:10ECE00067EE877A0902F5EEC07AF1EE10FAC0F20B
:10ECF000C780D2F87C0D411A07EE901A02F55762D0
:10ED0000B8EEE77AD2ED007A77EE677AB3EE057A5D
:10ED1000F4EEC77AF1EE10FA3EF611AC58077EF524
:10ED20000EACB5FA85F35B0944F2A00202FB034284
:10ED300002F6845191ED007AD2F8901D07EE901AF8
:10ED4000F8EEE77A44F2A00167EE877A01FB03430D
:10ED5000F5EEC07AF1EE10FAACBFD2F8782DD2F809
:10ED60007C2DC3F86C2D64AE0DF5D2796EAF0DF528
:10ED7000E67800234FF0FF32D4F824083360C9F856
:10ED800000303A60C8F80020002D76D144F60862C1
:10ED90000123A15844F2A00505FB034348F6887AF5
:10EDA000D3F86C2D00973346F7F770F854F80A3013
:10EDB000D4F82408002B0CBF2B4600232344002248
:10EDC000D3F8681DCDF800804B46F7F75FF831683F
:10EDD000D9F8003054F80A50C91A002D43D1D7EDA4
:10EDE000007AF8EEE77A04F59C43C3ED047A012338
:10EDF00044F2A00202FB034303F6845090ED007A34
:10EE0000D3F8900D704E07EE900AF8EEE77A67EEB1
:10EE1000877AF5EEC07AF1EE10FAACBF0020072039
:10EE2000002D18BF002244F6FC5522445851C2F868
:10EE3000741D2369654A04F6340504F6380004F6A7
:10EE40003C0143F0200323612A6002600E60FEF75C
:10EE500076BBD7ED007AF8EEE77A04F55763C3ED99
:10EE6000007A0023FFE6D7ED007AF8EEE77A04F5A2
:10EE70005763C3ED007A0023BAE7D4F8681D89E729
:10EE8000D2F8780D091A07EE901A02F55762F8EEDB
:10EE9000E77A92ED007A77EE877A37E7D4F8681D43
:10EEA000B2E6D2F8780D091A07EE901A02F5576209
:10EEB000F8EEE77A92ED007A77EE877A5CE642DA4E
:10EEC0002BD45200B5EEC07AF1EE10FABEF632A89D
:10EED00007EE90EAB8EEE76AF7EE006A35EE466AAA
:10EEE00036EEC66AFEF72CB84EDA03D54FF0000CAA
:10EEF00067452CDB7F00B5EEC07AF1EE10FABDF667
:10EF000097A807EE90EAB8EEE76AF7EE006A35EEEA
:10EF1000466A36EEC66AFDF791B84FF0000C6245BE
:10EF2000CFDA7B1903F0070344F2A00203EB430599
:10EF300002FB06F303EB850303F59B4318332344DD
:10EF400040F2FE72BEE74FF0000CFDF7E0BF431940
:10EF500003F0070344F2A00503EB430705FB06F3A8
:10EF600003EB870303F59B431833234440F2FE77FA
:10EF7000C1E7D0ED007A37EEC77AB04680ED007A6F
:10EF8000DEF8747DFDF708B84FF0000CFDF73DB8D2
:10EF9000236948F6887A44F2A00944F80A8023F0ED
:10EFA000200309FB0848236198F8803D93B9B0EE2F
:10EFB000688AFEF76ABB9FED067AFDF784B900BF49
:10EFC00000002044CDCCCC3ACDCC4C3D0000A0413B
:10EFD00000000000D8F87C1DD8F8683D0591BE49B6
:10EFE000D8F8782DD4F8240804930CAD0DAE0F4654
:10EFF000009519464FF0FF3533460C950D95F6F701
:10F0000045FF54F80A303878DDF834800397002B38
:10F010000CBF4B460023234444F69C5144F6A052B7
:10F0200006464FF0010043F8018098540420D4F8BC
:10F0300004E02B90DEF88022DEF88402CDF8A48074
:10F0400044F6985101325B582A93002E02F01F05B6
:10F050000CBF032301234FF0000785428DF8B03029
:10F060008DF8A0700695A2D028A80546DEF880721B
:10F070000FCD07EB8707BF000EEB070C4EF807001C
:10F08000CCF80410CCF80820CCF80C302B788CF895
:10F09000103054F80A30069DCEF88052002B0CBF79
:10F0A0004B460023234444F6A85008F1040244F6DA
:10F0B000AC511A504FF0010058540420D4F804E029
:10F0C0002690DEF88012DEF884520D9244F6A450A9
:10F0D00001311B582593002E01F01F080CBF03239C
:10F0E00001234FF00000A8458DF88C0024928DF884
:10F0F0009C303FF45CAF23AD0FCDDEF8807207EBA0
:10F100008707BF000EEB070C4EF80700CCF8041081
:10F11000CCF80820CCF80C302B788CF810300CADE3
:10F12000D4F82408059ACEF88082049900950DAB96
:10F13000F6F7ACFE54F80A30039A0D9F1278002BB4
:10F140000CBF4B460023234444F6F051154644F6C9
:10F15000F4525F504FF0010199540422D4F804E0B6
:10F160002192DEF88002DEF8842203954FF0000140
:10F170008DF8781044F6EC5100F1010C5B582093A7
:10F18000002D0CF01F0C0CBF0323012394451F9787
:10F190008DF888303FF40BAF1EAB1D46DEF8806261
:10F1A0000FCD06EB8606B6000EEB06084EF80600FD
:10F1B000C8F80410C8F80820C8F80C302B7888F874
:10F1C000103054F80A30CEF880C2002B0CBF4B46EA
:10F1D0000023234444F6E4503A1F44F6E8511A5001
:10F1E0004FF001005854042167681C91D7F88052F1
:10F1F000039ED7F884120D9244F6E05005F1010EFB
:10F200001B581B93002E0EF01F0E0CBF032301236F
:10F210004FF000008E458DF864001A928DF874301E
:10F220003FF4C5AE19AD0FCDD7F8806206EB860668
:10F23000B60007EB060CB851CCF80410CCF8082047
:10F24000CCF80C302B788CF8103054F80A00C7F842
:10F2500080E200280CBF4846002000F66850204499
:10F26000F7F706FF54F80A50002D40F0FD8148F6EC
:10F2700098620626D4F8681DA65044F6086044F645
:10F28000206394F8802D2150E25404F59C435A6881
:10F2900004F50E43C3F8A420029B03F63C6393E8F5
:10F2A000070004F59C43243383E8070044F6186004
:10F2B00044F61C62D4F8783DD4F87C1D2350A1504C
:10F2C000012344F2A00202FB054502FB0343D5F8EB
:10F2D000902DC3F8902D6AE63ACC012000402044DE
:10F2E000D2F8900DD2F8741D07EE900A02F6845001
:10F2F000F8EEE77A90ED007A67EE877A0902F5EE8C
:10F30000C07AF1EE10FAC0F2DC80D2F87C0D411A1E
:10F3100007EE901A02F55762B8EEE77AD2ED007A5E
:10F3200077EE677A1FED137AF4EEC77AF1EE10FAF2
:10F330003EF6ABA959077EF5A8A9BEFA8EF1490998
:10F3400044F2A00202FB014202F68450D2F8903D42
:10F350005B4207EE903AC2F8903D90ED007AF8EEED
:10F36000E77A19AE67EE877A1EAFF5EEC07AF1EE56
:10F3700010FAACBFD2F8783DD2F87C3D44F2A0023E
:10F3800002FB01410DF18C0A28ADC1F86C3D4FF034
:10F39000FF320023D4F8240833603B60CAF8002011
:10F3A0002A60BEF1000F40F0898044F60862012314
:10F3B000A15844F2A00808FB034348F68879D3F823
:10F3C0006C2DCDF800A03346F6F760FD54F80930F7
:10F3D000D4F82408002B0CBF43460023234400220A
:10F3E000D3F8681D00953B46F6F750FD31683B6841
:10F3F00054F80900C91A00284DD1DAED007AF8EE68
:10F40000E77A04F59C43C3ED047A012344F2A00299
:10F4100002FB034303F6845595ED007AD3F8905D23
:10F42000029FD24E07EE905AF8EEE77A67EE877A9F
:10F43000F5EEC07AF1EE10FAACBF002507250028E2
:10F4400018BF002244F6FC5022441D50C2F8741D1F
:10F450002369C74D43F0200007F6EC0107F50F6262
:10F4600007F6F40320610E6016601D60FEF70DB90B
:10F4700077EE277A4CBF4FF0FF350025C3ED007AB9
:10F4800018DA13DAF5EEC07AF1EE10FA4CBF012368
:10F490000023FCF7E9BCDAED007A029BF8EEE77A8C
:10F4A00003F62863C3ED007A0023AFE7DFEDB66A09
:10F4B000FCF7D3BCDFEDB56AFCF7CFBCD4F8681D10
:10F4C00077E7D2F8780D091A07EE901A02F557621D
:10F4D000F8EEE77A92ED007A77EE877A22E7D2F8B3
:10F4E000900DD2F8741D07EE900A02F68450F8EEE3
:10F4F000E77A90ED007A67EE877A0902F5EEC07A36
:10F50000F1EE10FAC0F2E580D2F87C0D411A07EE58
:10F51000901A02F55762B8EEE77AD2ED007A77EEEC
:10F52000677AB3EE057AF4EEC77AF1EE10FA3EF69A
:10F53000ACA858077EF5A9A8BEFA8EF35B0944F281
:10F54000A00202FB034202F6845191ED007AD2F848
:10F55000901D07EE901AF8EEE77A44F2A00167EEEC
:10F56000877A01FB0343F5EEC07AF1EE10FAACBFE7
:10F57000D2F8782DD2F87C2DC3F86C2D19AE1EAFC1
:10F580000DF18C0A28AD00234FF0FF32D4F8240887
:10F5900033603B60CAF800202A60BEF1000F40F0E3
:10F5A000958044F608620123A15844F2A00808FBA4
:10F5B000034348F68879D3F86C2DCDF800A0334684
:10F5C000F6F764FC54F80930D4F82408002B0CBF7B
:10F5D0004346002323440022D3F8681D00953B4690
:10F5E000F6F754FC31683B6854F80900C91A002842
:10F5F00061D1DAED007AF8EEE77A04F59C43C3EDC9
:10F60000047A012344F2A00202FB034303F684556B
:10F6100095ED007AD3F8905D029F564E07EE905A12
:10F62000F8EEE77A67EE877AF5EEC07AF1EE10FA37
:10F63000ACBF00250725002818BF002244F6FC5067
:10F6400022441D50C2F8741D23694B4D43F0200025
:10F6500007F6EC0107F50F6207F6F40320610D6071
:10F6600015601E60FEF711B844F6F8530622E2500A
:10F6700009FB0546D6F8683DC4F8683D96F8803D1C
:10F6800084F8803D06F59C435A6804F59C435A6013
:10F6900006F6845393E80700029B03F63C6383E875
:10F6A0000700D6F8783DC4F8783DD6F87C3DC4F81C
:10F6B0007C3D002305E6DAED007A029BF8EEE77A5E
:10F6C00003F62863C3ED007A00239BE7D4F8681D96
:10F6D0006BE7D2F8780D091A07EE901A02F5576217
:10F6E000F8EEE77A92ED007A77EE877A19E71BDA7F
:10F6F000F5EEC07AF1EE10FA4CBF01220022FCF7C1
:10F7000038BAD1F87C1D9FED1F6A891A07EE901A4E
:10F71000F8EEE77A77EEE67AF4EEC67AF1EE10FAD2
:10F720007CF502AFFCF7F4BE9FED177AFCF71ABA2E
:10F730000EEB050101F0070144F2A00501EB410CBD
:10F7400005FB07F101EB8C0101F59B4118312144C8
:10F7500040F2FE75FEF739BF4FEA4C05FCF794BE48
:10F760000648FAF773F90648FAF770F900002044E2
:10F77000CDCCCC3ACDCC4C3D0000A041143E020093
:10F780009C3D0200000020430000000000C07F44B8
:10F79000711901F0070144F2A00501EB410E05FBD0
:10F7A00007F101EB8E0101F59B411831214440F234
:10F7B000FE7EFEF73EBC4FEA4E0EFCF7AEBAD1F825
:10F7C0007C1D5FED106A891A07EE901AF8EEE77A51
:10F7D00077EEC57AF4EEE67AF1EE10FA7DF568AAD6
:10F7E000FDF75ABA36DA7EF552AE4FF00009FEF751
:10F7F0004BBE44F2A00202FB054644F6F852062333
:10F80000A350D6F8683DC4F8683D96F8803D84F86A
:10F81000803D06F59C435A6804F59C435A6006F601
:10F82000845393E80700029B03F63C6383E80700D8
:10F83000D6F8783DC4F8783DD6F87C3DC4F87C3DD8
:10F84000049AFEF7F2BD09DA7EF5F1AB4FF0000C39
:10F85000FEF7EABB4FF00009FDF7C6B94FF0000C08
:10F86000FCF747BA0EEB050101F0070144F2A005D1
:10F8700001EB410C05FB07F101EB8C0101F59B410C
:10F880001831214440F2FE7CFEF703BE4FEA4C0CD7
:10F89000FDF7BFB90FDA7EF596AE4FF00009FEF71F
:10F8A0008FBE0CDAF5EEC07AF1EE10FA4CBF0122F1
:10F8B0000022FDF7D3B84FF00009FCF7D1BD1FEDD2
:10F8C0004E7AFDF7C4B8B046FCF766BB44F2A0031D
:10F8D00003FB0646D6F8783DCB1A07EE903AB8EE11
:10F8E000E77A77EE057AFCF701BC77EE277A4CBF12
:10F8F0004FF0FF350025C3ED007A1CDA17DAF5EE7C
:10F90000C07AF1EE10FA4CBF01230023FDF729BAAB
:10F9100044F2A00303FB0646D6F8783DCB1A07EE67
:10F92000903AB8EEE77A77EE057AFCF79BBF5FED89
:10F930006A6AFDF70FBA5FED6B6AFDF70BBA35DA4D
:10F940001DD45200B5EEC07AF1EE10FABCF62AAF23
:10F9500007EE908AB8EEE76AF7EE006A35EE466A7F
:10F9600036EEC66AFCF724BFDCED007A37EEC77AC4
:10F9700037468CED007ADEF8742DFCF7C5BE4FF0EB
:10F98000000C6245DDDA0EEB050303F0070344F2D9
:10F99000A00203EB430502FB06F303EB850303F52B
:10F9A0009B431833234440F2FE72CBE74FF0000C28
:10F9B000FCF7E4BEB5EEC07AF1EE10FAE1D45200E5
:10F9C000FCF7F0BE236948F6887544F2A00A675137
:10F9D00023F020030AFB0747236197F8803D002BA3
:10F9E00040F04A81B0EE688AFCF796BF44F2A0026C
:10F9F00002FB054644F6F8520623A350D6F8683DAC
:10FA0000C4F8683D96F8803D84F8803D06F59C4337
:10FA10005A6804F59C435A6006F6845393E807003D
:10FA200004F6845383E80700D6F8783DC4F8783D9F
:10FA3000D6F87C3DC4F87C3D029AFEF7C7B8DDEDF0
:10FA4000B97AF8EEE77A04F55763C3ED007A00233C
:10FA5000FDF7F7BED4F8681DFDF7C6BED2F8780DE5
:10FA6000091A07EE901A02F55762F8EEE77A92ED5E
:10FA7000007A77EE877AFDF776BED2F8905DD2F8FD
:10FA8000741D07EE905A02F68450F8EEE77A90ED76
:10FA9000007A67EE877A0902F5EEC07AF1EE10FA85
:10FAA000C0F2C082D2F87C0D411A07EE901A02F51E
:10FAB0005762B8EEE77AD2ED007A77EE677AB3EE66
:10FAC000057AF4EEC77AF1EE10FA3CF625AF580746
:10FAD0007CF522AFB6FA86F35B0944F2A00202FB82
:10FAE000034202F6845191ED007AD2F8901D07EEA0
:10FAF000901AF8EEE77A44F2A00167EE877A01FBEC
:10FB00000343F5EEC07AF1EE10FAACBFD2F8782DCF
:10FB1000D2F87C2DC3F86C2DAFAD00234FF0FF322F
:10FB2000D4F824082B60B493B992BE92002E40F012
:10FB3000768244F608620123A15844F2A00606FB2F
:10FB40000343B9AFD3F86C2D009748F688772B465E
:10FB5000F6F79CF9E359D4F82408002B0CBF334680
:10FB600000232344BEAAD3F8681D0092B4AB002240
:10FB7000F6F78CF92968B49BE659C91A002E40F0B3
:10FB80004482DDEDB97AF8EEE77A04F59C43C3EDE3
:10FB9000047A012344F2A00202FB034303F68450DB
:10FBA00090ED007AD3F8900D314D07EE900AF8EE03
:10FBB000E77A67EE877AF5EEC07AF1EE10FAACBF1D
:10FBC00000200720002E18BF002244F6FC562244D5
:10FBD0009851C2F8741D2369264A04F6340604F6C7
:10FBE000380004F63C0143F02003236132600260D8
:10FBF0000D60FCF791BE44F6F8520623A35005FBB6
:10FC00000645D5F8683DC4F8683D95F8803D84F810
:10FC1000803D05F59C435A6804F59C435A6005F6FF
:10FC2000845393E8070004F6845383E80700D5F86B
:10FC3000783DC4F8783DD5F87C3DC4F87C3D029A07
:10FC4000FEF7C8B977EE277A4CBF4FF0FF35002595
:10FC5000C3ED007A80F2948180F28E81F5EEC07A55
:10FC6000F1EE10FA4CBF01230023FCF7B6BC00BF35
:10FC7000CDCC4C3D0000A041D7F8683DD7F87C1DA5
:10FC8000D7F8782DD4F8240804919BAEBE4900968D
:10FC9000A0AE4FF0FF3703910293194633469B976E
:10FCA000A097F6F7F3F86359B748DDF8809200782B
:10FCB000CDF8FC92002B0CBF53460023234444F69E
:10FCC0009C5144F6A05206464FF0010043F80190C3
:10FCD00098540420D4F804C0C190DCF88022DCF8E9
:10FCE000840244F698510132002E02F01F075B583F
:10FCF000C0934FF0000E3B460CBF03230123874205
:10FD00008DF808338DF8F8E203973FF46BAEBEAF81
:10FD1000DCF880E20FCF0EEB8E0E4FEA8E0E0CEB6E
:10FD20000E084CF80E00C8F80410C8F80820C8F8EF
:10FD30000C303B7888F8103063590398CCF8800277
:10FD4000002B0CBF53460023234444F6A85009F16E
:10FD5000040144F6AC5219504FF0010098540420AD
:10FD6000D4F804C0A091BC90DCF88002DCF88422B6
:10FD7000BA9100F1010844F6A451002E08F01F08C2
:10FD80005B58BB930CBF032101214FF0000090454D
:10FD90008DF8E4028DF8F4123FF424AEB9AF0FCF22
:10FDA000DCF880E20EEB8E0E4FEA8E0E0CEB0E09A5
:10FDB0004CF80E00C9F80410C9F80820C9F80C3036
:10FDC0003B7889F810309BABD4F82408049ACCF81F
:10FDD000808202990093A0ABF6F758F86359A09F70
:10FDE000002B0CBF534600232344042244F6F05159
:10FDF000B79244F6F4525F504FF001019954624AB1
:10FE0000D4F804C01278DCF880024FF000011646E6
:10FE100000F10108DCF884228DF8D01244F6EC5190
:10FE2000002E08F01F085B5802960CBF0321012129
:10FE30009045B597B6938DF8E0123FF4D3ADB4AECC
:10FE4000DCF880E20FCE0EEB8E0E4FEA8E0E0CEB3E
:10FE50000E094CF80E00C9F80410C9F80820C9F8BA
:10FE60000C30337889F810306359CCF88082002B3D
:10FE70000CBF53460023234444F6E451043F44F6A8
:10FE8000E8525F504FF0010199540421D4F804E086
:10FE9000B291A097DEF88002029EDEF88422B0972D
:10FEA0004FF000018DF8BC1244F6E05100F1010C56
:10FEB0005B58B193002E0CF01F0C0CBF03230123E1
:10FEC00094458DF8CC323FF48DADAFAE0FCEDEF859
:10FED000807207EB8707BF000EEB07084EF807009C
:10FEE000C8F80410C8F80820C8F80C30337888F82F
:10FEF00010306059CEF880C200280CBF5046002058
:10FF000000F668502044F7F7B3F86559002D43D147
:10FF100048F698620626D4F8680DA65044F60861A3
:10FF200044F6206394F8802D6050E25404F59C431D
:10FF30005A6804F50E43C3F8A42004F6845393E8EA
:10FF4000070004F59C43243383E8070044F6186354
:10FF500044F61C62D4F8780DD4F87C1DE050A15012
:10FF6000012344F2A00202FB054502FB0343D5F83E
:10FF7000902DC3F8902D35E5DFED046AFCF726BB24
:10FF8000DFED036AFCF722BB3ACC01200000000041
:10FF900000C07F440000204344F6F8530622E2509C
:10FFA0000AFB0546D6F8683DC4F8683D96F8803DE2
:10FFB00084F8803D06F59C435A6804F59C435A60DA
:10FFC00006F6845393E8070004F6845383E8070099
:10FFD000D6F8783DC4F8783DD6F87C3DC4F87C3D31
:10FFE0000023BEE7D1F87C1D5FED166A891A07EE83
:10FFF000901AF8EEE77A77EEC57AF4EEE67AF1EE4B
:020000021000EC
:1000000010FA7BF5D7AEFBF7C9BEDDEDB97AF8EE95
:10001000E77A04F55763C3ED007A0023BAE5D4F814
:10002000681D8AE5D2F8780D091A07EE901A02F5D4
:100030005762F8EEE77A92ED007A77EE877A3EE53E
:100040002DE9F8432C4D9DF820709DF8246048F66A
:10005000907404FB005443F2FC1C14F80C80B8F1BB
:10006000030F05D014F80C40042C01D0BDE8F88330
:1000700048F6907404FB00F02C1804F54754303413
:10008000002ED4F8446BD4F848CB06F1010606F0F4
:100090001F060CBFB8464FF00208664528D0D4F8BA
:1000A000447B07EB4707FF00284404F644090A9DF8
:1000B00049F8071009EB070C43F2FC114CF27C17CE
:1000C000AE46CCF80420CCF808303EEA250E28BF16
:1000D00096460A9B8CF80C8004228CED040ACCF81E
:1000E0001430C4F8446B40F807E04254BDE8F8838C
:1000F0000248F9F7ABFC00BFA81CFF1F3C3E020002
:1001000070B5D0F86439002B84B021DBD0F8D8204A
:100110000B2A5DD0D0F8D8210B2A5BD0D0F8D8229A
:100120000B2A59D0D0F8D8230B2A57D0D0F8D8248E
:100130000B2A55D0D0F8D8250B2A53D0D0F8D82682
:100140000B2A07D0D0F8D8270B2A08BF072402D0E3
:1001500004B070BD062400EB042494F89061002ED6
:10016000F6D1D0F8D85A94F8E9202A4492F89011A0
:100170006329EDD805EB8102D2F8F421002AE7DDEE
:1001800005EB4105DFED186AB5F84C2400689FEDDA
:10019000170A07EE102AB5F88423029307EE902A77
:1001A000B8EEC77AF8EEE77A27EE267A67EEA67AF7
:1001B000BDEEC77AFDEEE77A0125009617EE103AFC
:1001C00017EE902A0195FFF73BFF84F89051BFE7A7
:1001D0000024C0E70124BEE70224BCE70324BAE7F9
:1001E0000424B8E70524B6E7000000420000000040
:1001F000D0F86439002B00DB7047F0B5D0F8483BED
:1002000093F8602085B0002A45D0D0F84C4B94F884
:10021000603093B3D0F8502B92F860405CBB92F8FA
:10022000702942BB3BBBD0F8D8200C2A00F09B823F
:10023000D0F8D8310C2B00F09882D0F8D8320C2BA3
:1002400000F09582D0F8D8330C2B00F09282D0F8D1
:10025000D8340C2B00F08F82D0F8D8350C2B00F05E
:100260008C82D0F8D8360C2B21D0D0F8D8370C2B74
:1002700008BF07251CD005B0F0BD94F87039002BDD
:100280000CBF134642F00103D0F8502B92F86040A7
:10029000002CF0D1C3E7D0F84C4B93F8702994F8B8
:1002A0006030003218BF0122002BB3D1E5E70625EC
:1002B00090F88030002B00F09681D0F88430002B2D
:1002C000D9DDE84B9FEDE87A53F82530083300F587
:1002D0002B6631F81330D6ED006A00EE103AF8EED6
:1002E000C07AB8EE400A77EEE67AF0EEE77AF4EEFE
:1002F000C77AF1EE10FA07DD00F5276200F66C23ED
:1003000082ED000A83ED000A044600F65820F0F75B
:1003100087FDD4F884209FEDD57AD4F8881086ED37
:10032000000A07EE902AF8EEE76A531EC6EE877AB7
:1003300027EE800AFDEEC07A17EE902A9A42A8BFF7
:100340001A46914297D02B02E1180120C4F8882068
:1003500084F8640081F8E920D4F8D86A3244002097
:1003600092F8905156F82550C1F8EC50D4F8D85076
:1003700084F890014FF0FF31022DC4F89C11C4F8AD
:10038000A01100F0C181032DC4F8940100F0B681E2
:100390000021C4F89811D4F8D8514FF0FF31002053
:1003A000022D84F89002C4F89C12C4F8A01200F048
:1003B0009D81032DC4F8940200F092810021C4F8BD
:1003C0009812D4F8D8524FF0FF310020022D84F853
:1003D0009003C4F89C13C4F8A01300F07981032D96
:1003E000C4F8940300F06E810021C4F89813D4F887
:1003F000D8534FF0FF310020022D84F89004C4F848
:100400009C14C4F8A01400F05581032DC4F8940482
:1004100000F04A810021C4F89814D4F8D8544FF061
:10042000FF310020022D84F89005C4F89C15C4F813
:10043000A01500F03181032DC4F8940500F0268149
:100440000021C4F89815D4F8D8554FF0FF3100209A
:10045000022D84F89006C4F89C16C4F8A01600F08B
:100460000D81032DC4F8940600F0F6800021C4F835
:100470009816D4F8D8564FF0FF310020022D84F89A
:100480009007C4F89C17C4F8A01700F0DD80032D76
:10049000C4F8940700F0D2800021C4F89817D4F86B
:1004A000D8574FF0FF310020022D84F89008C4F88F
:1004B0009C18C4F8A01800F0B980032DC4F8940863
:1004C00000F0AE800021C4F8981823444FF0FF35A7
:1004D000C4F86C5993F86F01012183F8901180B131
:1004E000884200F04C81D4F858096149614B01FB06
:1004F00000F10B44C3F30E4101F00201C4F8583976
:100500002944D4F8D800C4F860190428D4F8D801D4
:100510004FF0000384F85E3084F85F3008BF94F831
:100520009231042804BF94F892020343D4F8D8020D
:10053000042804BF94F892030343D4F8D803042892
:1005400004BF94F892040343D4F8D804042804BFE9
:1005500094F892050343D4F8D805042804BF94F80E
:1005600092060343D4F8D806042804BF94F89207EF
:100570000343D4F8D807042804BF94F8920803432F
:1005800003B14942012992F890112068DFED3A6ADF
:1005900006EB410604F65C1440F0BE80B6F84C341D
:1005A00094ED000A07EE103AB6F8843307EE903A5D
:1005B000B8EEC77AF8EEE77A27EE267A67EEA67AE3
:1005C000BDEEC77AFDEEE77A00244FF0FF3517EE57
:1005D000103A17EE902AB0EEC00A029501940094EA
:1005E000FFF72EFD47E6D0F8D87AC0F88430012214
:1005F00007F28F1480F880200AE0D6F8F421002A50
:100600007FF75DAE0133632BC0F884303FF459AE01
:1006100014F8012F632A07EB82063FF650AEECE791
:1006200094F8021800293FF450AF4BE794F8F617FE
:1006300000293FF447AFC4F8940843E794F8021741
:1006400000293FF42CAF27E794F8F61600293FF471
:1006500023AFC4F894071FE794F8021600293FF46B
:1006600008AF03E7C844020000AA2A4500FF7F47FD
:10067000FD430300C39E26000000004294F8F615D7
:1006800000293FF4F3AEC4F89406EFE694F802159F
:1006900000293FF4D8AED3E694F8F61400293FF4CD
:1006A000CFAEC4F89405CBE694F8021400293FF4C9
:1006B000B4AEAFE694F8F61300293FF4ABAEC4F83D
:1006C0009404A7E694F8021300293FF490AE8BE659
:1006D00094F8F61200293FF487AEC4F8940383E639
:1006E00094F8021200293FF46CAE67E694F8F61114
:1006F00000293FF463AEC4F894025FE694F8021157
:1007000000293FF448AE43E694F8F61000293FF480
:100710003FAEC4F894013BE6B6F8843394ED000A8A
:1007200007EE103AB6F84C3407EE903AB8EEC77AB6
:10073000F8EEE77A27EE267A67EEA67ABDEEC77A5C
:10074000FDEEE77A00244FF0FF35B0EEC00A17EE59
:10075000103A17EE902AB1EE400A029501940094E7
:10076000FFF76EFC87E51D46A2E50125A0E5022501
:100770009EE503259CE504259AE5052598E529468F
:10078000BFE600BFF0B50268C34C48F6907303FBA8
:10079000024343F2FC1185B05D5C042D00F09080B3
:1007A0005B5C052B0DD14FF0FF3348F6907101FBD8
:1007B00002424CF26C1100245452002B01DB05B0B4
:1007C000F0BDD0F86439002BF9DA90F89031002BA5
:1007D0007ED0D0F89C31591C7AD0D0F8A021002AC4
:1007E00076DB00269F1C00F0178190F870590124D9
:1007F000C0F860493102002D00F0CA802344002B6C
:1008000004DB421892F8A4219A420EDC471897F8AC
:10081000EA30012B00F02A8197F8A421012A00F088
:100820003181012C40F0308123464218C2F89C31BE
:1008300003EBC61300EB4303DFED986AB3F8A62180
:10084000B3F8BE3107EE102A07EE903AB8EEC77A39
:10085000F8EEE77A27EE267A67EEA67ABDEEC77A3B
:10086000FDEEE77A17EE102A17EE903A9A42A6D0DC
:10087000661C00F002810144D1F8A011002D40F067
:10088000C88000F65C1595ED000AB0EEC00AD0F8FD
:10089000D85A29449D1A002D064691F890110068F7
:1008A00040F3D08000254FF0FF3701950095029767
:1008B000FFF7C6FB012504FB05F4C6F860497EE797
:1008C000595C4CF27C1505295B597FF476AF6CE7D7
:1008D00090F890324BB1D0F89C325A1C05D0D0F829
:1008E000A022002A01DB01267CE790F890334BB16F
:1008F000D0F89C335F1C05D0D0F8A023002A01DB80
:1009000002266FE790F890344BB1D0F89C345E1C0F
:1009100005D0D0F8A024002A01DB032662E790F876
:1009200090354BB1D0F89C355D1C05D0D0F8A02592
:10093000002A01DB042655E790F890364BB1D0F839
:100940009C365C1C05D0D0F8A026002A01DB0526C9
:1009500048E790F890374BB1D0F89C37591C05D038
:10096000D0F8A027002A01DB06263BE790F8903854
:10097000002B3FF424AFD0F89C385A1C3FF41FAF33
:10098000D0F8A028002AA8BF0726FFF618AF29E74D
:10099000D0F8D84090F85E20042C04BF90F8924123
:1009A0002243D0F8D841042C04BF90F8924222434D
:1009B000D0F8D842042C04BF90F892432243D0F8D8
:1009C000D843042C04BF90F892442243D0F8D84472
:1009D000042C04BF90F892452243D0F8D845042C4B
:1009E00004BF90F892462243D0F8D846042C04BFA6
:1009F00090F892472243D0F8D847042C04BF90F8CF
:100A000092482243C2B19C1C4AD000254FF0FF34CB
:100A1000F4E6B7EE000A3AE73102421892F8D6211E
:100A2000002A3FF4CCAE90F870590124C0F8604918
:100A3000002DADD00023E4E615469A1C38D12B4694
:100A40000124DEE614BF4FF0FF35002507EE905A73
:100A5000F8EEE77A00274FF0FF3E27EE800ACDF848
:100A600008E001970097FFF7EBFA24E74FF0FF3318
:100A7000C7F8A031C7F89C31A1E617EE902A17EE0F
:100A8000103AF8E60023D0E6931E002BC7F89C31FD
:100A9000BFF6CEAE93E600BFA81CFF1F00000042C9
:100AA00043184FF0FF3493F8A42100251319A6E64C
:100AB0000124A3E62DE9F04FD0F864498DB0002C55
:100AC0009DF8585002DB0DB0BDE8F08F8E460968E6
:100AD00001294FD0CC1F012C4CD9042900F01E83D2
:100AE000022900F05F83032900F07883062900F0D3
:100AF000B7820529E7D1002BE5D090F89031002B83
:100B000000F09F84002380F89031012390F8902218
:100B10001AB1002380F89032012390F890231AB183
:100B2000002380F89033012390F890241AB1002319
:100B300080F89034012390F890251AB1002380F8B2
:100B40009035012390F890261AB1002380F8903652
:100B5000012390F89027002A00F0768490F89038CE
:100B6000002280F8902713B1002380F89038F1F725
:100B70002DFBA8E701EB410C0EEB8C0C9CF80660FA
:100B8000002E00F04082002B9DD001230693DEF85A
:100B900014309EF811B00593072900F0D082D0F8E8
:100BA000D83A03EB0B0494F89071632F6AD803EBE7
:100BB0008707D7F8F471002F64DD4FF00009059F17
:100BC000002F00F0488216B122B190F87B20002A55
:100BD00000F04182072965D1002D53D12F46002214
:100BE00080F87B20002F4DD09CF80720002A00F0D1
:100BF0004982012A00F0C683D0F85829E44DE5491E
:100C000005FB02F21144C1F30549A9F11F09B9F12D
:100C1000000FC0F8581935D000F32584C9F1000938
:100C2000B9F1000F40F01C84DB4A9EF8101052F816
:100C30002120C2F3800ABAF1000F00F0CC829EF8A6
:100C400011201A4492F89021632A14D803EB8202EF
:100C5000D2F8F421002A0EDDBAF1000F40F096839D
:100C60006FF0010B03EB0B0292F8902153F8223046
:100C70000593CEF8143000238EF8FE30D0F8D83A21
:100C800003EB0B0494F89021632A3FF61CAF03EBAF
:100C90008202D2F8F421002A7FF715AF059A002AC4
:100CA0003FF411AFD0F8482B92F8601021B992F8B8
:100CB0007019003118BF0121D0F84C5B95F8602005
:100CC00032B995F87029002A0CBF0A4641F001029A
:100CD000D0F8501B91F86050002D7FF4F4AE91F8DD
:100CE000701900297FF4EFAE002A7FF4ECAE0121E9
:100CF00080F86410069900293FF439AFD0F8D85035
:100D000080F890214FF0FF31022DC0F89C11C0F8FF
:100D1000A01100F02F83032DC0F8942100F024834C
:100D20000022C0F89821D0F8D8514FF0FF320021AE
:100D3000022D80F89012C0F89C22C0F8A02200F08A
:100D40000B83032DC0F8941200F000830022C0F83A
:100D50009822D0F8D8524FF0FF320021022D80F8AF
:100D60009013C0F89C23C0F8A02300F0E782032D65
:100D7000C0F8941300F0DC820022C0F89823D0F869
:100D8000D8534FF0FF320021022D80F89014C0F8A4
:100D90009C24C0F8A02400F0C382032DC0F8941452
:100DA00000F0B8820022C0F89824D0F8D8544FF050
:100DB000FF320021022D80F89015C0F89C25C0F864
:100DC000A02500F09F82032DC0F8941500F09482B6
:100DD0000022C0F89825D0F8D8554FF0FF320021F6
:100DE000022D80F89016C0F89C26C0F8A02600F0CE
:100DF0007B82032DC0F8941600F070820022C0F8A8
:100E00009826D0F8D8564FF0FF320021022D80F8F6
:100E10009017C0F89C27C0F8A02700F05782032D38
:100E2000C0F8941700F03E820022C0F89827D0F84E
:100E3000D8574FF0FF320021022D80F89018C0F8EB
:100E40009C28C0F8A02800F02582032DC0F8941833
:100E500000F01A820022C0F898284FF0FF350121D7
:100E6000C0F86C598EF8B8109CF807209AB1D61EBD
:100E70008E4210D98A4200F0F182D0F85819444DC0
:100E8000444A05FB01F10A44C2F30E4101F002019C
:100E9000C0F858290139DEF80060D0F8D870C0F8E1
:100EA0006019072E04BF0121C0F86019042FD0F883
:100EB000D8714FF0000280F85E2080F85F2008BFF4
:100EC00090F892219CF80750042F04BF90F892727A
:100ED0003A43D0F8D872042F04BF90F892733A4383
:100EE000D0F8D873042F04BF90F892743A43D0F826
:100EF000D874042F04BF90F892753A43D0F8D8758F
:100F0000042F04BF90F892763A43D0F8D876042F95
:100F100004BF90F892773A43D0F8D877042F04BFF3
:100F200090F892783A4302B14942042D00F0898149
:100F3000012994F89011DFED196A9CF8067003EB13
:100F40004103A5F10305B3F88423B3F84C3407EE4D
:100F5000902A07EE103AF8EEE77AB8EEC77A67EE15
:100F6000A67AB7FA87F7B5FA85F54FEA57174FEA29
:100F7000551527EE267AFDEEE77A40F0188217EE37
:100F8000902AFDEEC77A082ECDED057A2BD107E029
:100F9000FD430300C39E26002043020000000042E0
:100FA000D0F85869C249C34BDFEDC36A01FB06F1B3
:100FB00017EE906AB61A0B4407EE106AC3F30B41A2
:100FC00007EE901AB8EEC77AF8EEE77A27EE267A9F
:100FD000C0F8583967EE877A94F89011FDEEE77AF9
:100FE00017EE903A1A4400F65C1393ED000A00687D
:100FF00001954FF0FF3302930097B0EEC00A059BB6
:10100000FFF71EF85FE523B3002D3FF45CADDEF87B
:1010100014309EF811B00593072906927FF4BFADF6
:10102000D0F8D83A03EB0B0494F89081B8F1630F31
:101030003FF628AE4FF0000903EB8808D8F8F4819A
:10104000B8F1000F3FF7BBAD4F46002D7FF4CAAD9E
:10105000C5E506929BE507294F467FF4C3ADF4E74B
:101060009EF84E10002940F0DF81002B7FF42BAD5D
:101070009EF8B93093421CBF012380F864308EF88B
:10108000B92020E54FF001094F469EF810208B490A
:101090008B4C51F8221054F82220CDF81CB0C1F32B
:1010A000800AC2F3800283464FF000085046924601
:1010B00088B39EF811603246642411E0002AB8BF5C
:1010C0006222991891F89011632903EB810503D8E6
:1010D000D5F8F411002908DCB24206D0013C04D056
:1010E0003A44622AEADD0022EBE7BAF1000F09D0A8
:1010F000612ADABF22EAE272D2B262228EF81120AD
:10110000DBF8D83A08F10108C845D1D182465846E3
:10111000DDF81CB08FE56FF00106CCE79EF83610C5
:10112000002975D1002B7FF4CEAC9EF8BA309342E3
:101130001CBF012380F864308EF8BA20C3E4002D70
:101140007FF46EAFD0F8483B93F8604024B993F831
:101150007049003418BF0124D0F84C7B97F86030F8
:1011600033B997F87039002B0CBF234644F00103C4
:10117000D0F8504B94F8607037B994F87079002F1C
:101180000CBF1F4643F00107D0F8D83A03EB0B041D
:1011900087F0010994F89081B8F1630F7FF64CAFA6
:1011A0004F461CE59EF81E1000293DD1002B7FF410
:1011B0008AACDEF8BC30003318BF012393421CBF59
:1011C000012380F864301AB13E4B1B680893089ADB
:1011D000CEF8BC2077E46FF0010232E59EF82A10C9
:1011E000002940F0D680002B7FF46DACDEF8BC30D7
:1011F000003318BF012393421CBF012380F86430E1
:101200001AB1304B1B680A930A9ACEF8C0205AE4F0
:10121000002B3FF458AC90F85E300122534080F828
:101220005E3080F864204EE4002B3FF44CAC254B3C
:101230001B680993099BCEF8BC30012380F8643009
:1012400041E494F89021134493F8DC359B077FF533
:101250003AAC9EF8FE30CEF8C8B06FF00102CEF87E
:10126000C420002B7FF42FAC0368174A94F8901128
:1012700048F6907000FB032000F547500EF1CC02B9
:101280003030F6F745FC1EE490F80228002A3FF4BF
:10129000E4ADDFE590F8F627002A3FF4DBADC0F8B7
:1012A0009418D7E590F80227002A3FF4C0ADBBE5BB
:1012B000FD430300C39E260010C07F392043020077
:1012C000D43C020074CE0120A81CFF1F90F8F62623
:1012D000002A3FF4A9ADC0F89417A5E590F80226BE
:1012E000002A3FF48EAD89E590F8F625002A3FF4F8
:1012F00085ADC0F8941681E590F80225002A3FF4E8
:101300006AAD65E590F8F624002A3FF461ADC0F8B7
:1013100094155DE590F80224002A3FF446AD41E5BE
:1013200090F8F623002A3FF43DADC0F8941439E557
:1013300090F80223002A3FF422AD1DE590F8F62232
:10134000002A3FF419ADC0F8941315E590F8022275
:10135000002A3FF4FEACF9E490F8F621002A3FF4AD
:10136000F5ACC0F89412F1E490F80221002A3FF4A1
:10137000DAACD5E490F8F61000293FF4D1ACC0F80F
:101380009421CDE491464FF0FF377EE69EF811B0F0
:1013900068E4002B3FF497AB344B1B680B930B9B1B
:1013A000CEF8C030012380F86430FFF78CBB17EE15
:1013B00090EAFDEEC77A082E17EE902A21D1D0F8D8
:1013C00058392B4E2B49DFED2C6A06FB03F6CEEB8A
:1013D0000203314407EE103AC1F30B4307EE903A93
:1013E000B8EEC77AF8EEE77A27EE267AC0F85819F1
:1013F00067EE877A94F89011FDEEE77A17EE903A4F
:10140000D21A00F65C1494ED000A006801954FF0C2
:10141000FF34B0EEC00A00977346B1EE400A029462
:10142000FEF70EFEFFF74FBB002B3FF44CAB90F8DE
:101430005F300122534080F85F3080F86420FFF76E
:1014400042BB0023FFF762BB90F89028002A7FF48C
:101450008BAB002B3FF437ABFFF789BB29461AE56E
:101460004FF0FF3711E601270FE600BF74CE0120D1
:10147000FD430300C39E260010C07F39F8B5D0F8A5
:10148000503D8B4238D100F5356E0746144602F1C7
:10149000300C764620686168A268E36835460FC55F
:1014A000103464452E46F5D1206828607968144BC5
:1014B000D1F880421A78D1F88432D7F8547D0134BB
:1014C000002A04F01F0414BF012603269C4212D0F8
:1014D000D1F8802202EB820292008B1800200125B5
:1014E0008D545F60C3F808E01D731E7458739873C1
:1014F000D873C1F88042F8BD0248F8F7A7FA00BFD8
:101500003ACC0120543E020070B5114A48F690745E
:1015100004FB00F3D51843F2FC102E5C16B90D48FD
:10152000F8F794FA2E5C022EF9D0285C0128F6D048
:1015300004FB0120134400F5485003F548510830DE
:10154000083140F24462BDE870400AF0C7BA00BFFB
:10155000A81CFF1F783E0200D0F8482B436810B546
:10156000044650680021984282F8801010D0D4F8C8
:101570004C2B51680020994282F8800017D0D4F893
:10158000502B51680020994282F8800007D010BD8E
:101590009442ECD02068FFF7B7FF6368E7E7944216
:1015A000F5D020680221BDE81040FFF7ADBF94429E
:1015B000E5D001212068FFF7A7FF6368DFE700BFE0
:1015C000F8B590F87E30002B00F0A38000F1A4065F
:1015D000876904460FCE3F0204EB070C4FF0000E64
:1015E0000CF5D27584F880E084F87EE084F87FE022
:1015F0000FC50FCE0FC50FCE0FC533682B609CF8FB
:10160000E920D4F88C309A4214D02168434B48F634
:10161000907000FB01331A4443F29831FF2050547C
:1016200043F60C229958013104BF4FF47A51995076
:10163000D4F88C30274487F8E930D4F89020C7F8E4
:10164000EC20002A61D0D4F8D82AD11891F8901152
:1016500063295AD802EB8102D2F8F421002A54DD22
:1016600021682E4AD4F8945048F6907000FB01216E
:101670000B4443F2983643F60C209D550B5801332A
:1016800048D0D4F88C30D4F8D81A2568D4F898000B
:10169000B4F89C60194444F2C87391F8901103FBAC
:1016A000051303F5AC5103F5AF5318311C3302EBAE
:1016B000410102EB430348F6907707FB052543F60B
:1016C0000C27A1F85C0AA3F85C6AEB59013304BF4C
:1016D0004FF47A53EB51D4F8D85AD4F88C102368CD
:1016E000D4F8A000294448F6907591F8901105FBB4
:1016F0000322531843F2E47543F60C21585553580E
:10170000013304BF4FF47A5353502046FFF724FFB0
:10171000F8BDF8BD4FF47A530B50B2E7A81CFF1F79
:101720002DE9F04F2DED028B3A4A3B4B4260DFF83A
:10173000009140F21F12044602808BB003F5A070A6
:101740001A68596809EBC20208335268984211605E
:10175000F6D1324B3149D8691B6A02688969304D2C
:10176000E56013434FF0010A002222766276E261BF
:101770002266626684F810A0036061610A70636982
:10178000284F5A706369284E9A706369FF21D97097
:1017900063695A716369502199716369DA7161698A
:1017A0008B7803F07F038B70636996461222DA70A0
:1017B00004F10C03F046F44601934FF0FF301B494F
:1017C0000AFA0EF500220AE0C3F5C333A0338342C0
:1017D00002D21846F04694460132402A13D031F81E
:1017E000023F05FB03F3B7FBF3F3B342ECD9A3F5D8
:1017F000C333A03B8342EFD2F0469446D3B10132CB
:10180000402A1846EBD1BEF1020F13D00EF1010EA3
:10181000D5E700BF8C3E020074430200B8460200C8
:10182000202F0200008793039F86010016470200C5
:10183000904A02000CF03F03626943EA8813DBB26E
:1018400053706269537943F020035371626953798D
:1018500043F0800353716269937843F0800393707F
:10186000237CBF4A03EB430302EBC3030121DA6885
:1018700053099B0003F1604303F5614302F01F022B
:1018800001FA02F21A60B74B019A5A602022C4F89A
:10189000F420C4F81421B44AB44BC4F8F820C4F8B6
:1018A0000021C4F80821C4F81021B04A1E211F26C7
:1018B00000251D209342E566C4F8EC10C4F804111D
:1018C000C4F8F060C4F80C61C4F8E800C4F8FC0087
:1018D00004F16C0504F1F80704F588764FF0010176
:1018E0000CD138790AF0FEFBBE420BD057F8083F06
:1018F0009E4A1B6893424FF00101F2D03846984748
:10190000BE42F3D19A4BDFF890E2C4F81C5193E841
:101910000300C4F818E10022964F974EC4F82071D6
:1019200004F5967503F1080EC4F82421C4F8286163
:1019300085E803009EE8030004F59A7585E8030036
:101940008E4F84F83C21C4F8AC23C4F8B0233A6825
:101950008B4D8C49C4F8401142F0006204F594703C
:1019600028603A608A6822F00C028A608A6842F035
:1019700004028A604A6A22F004024A62CA6842F09B
:101980000802CA608A6842F003028A608A6842F0EC
:1019900020028A60CA6842F00402CA600A6A12F031
:1019A000400204F58C7801F0A9820A6A22F0400214
:1019B0000A62012773494A6A42F0C0024A624A6ACF
:1019C00070481206FBD4426A02691FB1026A42F0F3
:1019D000400202626B4ADFF8C4C1D76C906C516C54
:1019E0003844176C0144D06B0F443844976B07445C
:1019F00093E803007B0843F40043D362C4F8C06358
:101A00000023422204F57176C4F8B42384F8B83375
:101A1000C4F8BC83C4F828C186E803009EE803002C
:101A200004F5737282E803005748584A0168C4F805
:101A3000443641F000610126C4F8483684F8D46386
:101A4000C4F8D8230160936823F00C039360936873
:101A500043F004039360536A04F5707123F00403A8
:101A600069605362D36843F00803D360936843F01E
:101A700003039360936843F020039360D36843F0BB
:101A80000403D360136A13F040031DBF136A23F0ED
:101A9000400313621E463D4B5A6A42F0C0025A622E
:101AA000596A3A4A11F08001FAD1536A02911369D6
:101AB0001EB1136A43F040031362344B344EDD6CA5
:101AC0009A6C596C186C2A441144DD6B9A6B014472
:101AD000294411444908002741F400414322D962B6
:101AE00004F170003946C4F8C0C3C4F84C26C4F8E9
:101AF0005486782284F850760CF016FE019BC4F8C8
:101B000058360125C4F85C3604F25C6B214BC4F8EE
:101B100064364022C4F86076C4F87076394684F89A
:101B2000B95084F8C15084F8815084F8E05084F8AA
:101B3000C05084F89050C4F868B6C4F86C6604F2DB
:101B400074600CF0F1FD2123626984F8B636937855
:101B500003F0BF039370D4F86006657660B31FE0AE
:101B6000B846020048CE01203C2F0200A50B000021
:101B700008300200B90B00002C2F02003C8004400A
:101B800040CD012000B003403080044000B00B4045
:101B900025090000702F0200642F0200542F02005C
:101BA0000368D9495B688B4204F2646241F038866D
:101BB00040680221F1F71CFED4F8585694F8B43668
:101BC000D24AC4F8C026002104F5D76784F8B53698
:101BD0004022C4F8C866C4F8C476C4F8B856C4F83D
:101BE000BC16C4F8CC1604F5DA600CF09DFD222377
:101BF00084F81237AA68937803F0BF039370D4F87F
:101C0000BC0601236B7358B10368BF495B688B4204
